:020000040800F2
:10000000005000202D53010839F60008153D010865
:1000100037F6000835F6000833F600080000000047
:1000200000000000000000000000000031F60008A1
:100030002FF60008000000002DF600080BEC000869
:10004000CD530108CD530108CD530108CD5301080C
:10005000CD530108CD53010801C00008FFBF0008BF
:10006000CD530108CD530108CD530108CD530108EC
:10007000CD530108CD53010815C00008CD53010828
:1000800089930008CD530108CD530108CD530108D1
:1000900099F60008CD530108CD530108FDBF0008B3
:1000A000CD530108E5BB0008CD530108F5BB00089E
:1000B000D5BB0008C5BB0008B5BB000863530008EA
:1000C000675300085D53000861530008CD530108D1
:1000D000CD5301080DC00008CD53010803C000082E
:1000E00019EC0008CD530108053D0108000000008F
:1000F0000000000000000000000000000000000000
:0C01000000000000000000005FF808F1A3
:100110002DE9F04F684B694EA1B033600023736046
:1001200011F07EFB18B911F09DFB08F0C9F908F039
:1001300069FA634A634D1378634F43F00103137008
:100140000023089309930A934FF4E0130B932B6851
:10015000B87B43F480332B60AB6943F01003AB6191
:100160002B6803F400330993089B01330893099B20
:100170001BB9089BB3F5A06FF2D12B68514913F45A
:10018000003301D0022315E00A6842F001020A6040
:1001900008932B6803F002030993089B013308932B
:1001A000099B1BB9089BB3F5A06FF2D12B689A0786
:1001B00039D501230A93454B45491A6842F010028C
:1001C0001A601A6822F003021A601A6842F00202EA
:1001D0001A606B686B606B686B606B6843F480637C
:1001E0006B603C4B1A68043B22F070425A603A4AFA
:1001F0001160696821F47C116960596841F000411F
:100200005960D96821F40041D9609B681B0449BF3B
:10021000324B4FF4E01313604FF480130B930A9B9F
:10022000012B01D117E0FEE7022B18D168B10B9B1F
:10023000B3F5801F02D14FF4A01305E00B9BB3F57B
:10024000E01F02D14FF400130B930B996B680B4323
:1002500043F4803302E06B6843F460136B602B68F7
:1002600043F080732B602968164B8C01FBD55968CD
:1002700021F003015960596841F0020159606B682F
:10028000104903F00C03082BF9D14B68DFF85480B8
:1002900003F00C03042B03D0082B03D00C4B29E0F4
:1002A000136827E04B684868C3F38343C00303F136
:1002B000020319D40A4A1CE0A77C00087801002038
:1002C0007A300020001002404C280020002002401C
:1002D00000127A000410014048000020001BB70003
:1002E00000093D0004010020496812688C0348BFE2
:1002F00052085343C8F800306B68DFF83091C3F3FD
:1003000003134B441A7BD8F8003020ACD340C8F814
:1003100000303A4A3A4BDFF818B19360394B4FF04E
:10032000000AD360AB69039243F00103AB616B6ACF
:100330003548B3606B6A43F080736B62AB6943F01E
:100340001C03AB614FF6FF7324F82C3D21468DF85A
:1003500056A00FF051FE584621460FF04DFE2B4897
:1003600021460FF049FE2A4920464B6843F00073AE
:100370004B600DF02DF8159B2649039AB3FBF1F362
:1003800025490B60254B4FF47A71C3F800A0D8F8CB
:100390000030DFF89480B3FBF1F32149013B4B605F
:1003A000F02382F823300723C1F808A00B60BB6854
:1003B000DFF880A0CAF8003009F11C0393E80300BD
:1003C000AB6984E8030043F00803AB610823CBF872
:1003D0001030159816A90FF00FFEDAF80030180744
:1003E00030D598F89031012B2CD80E4B98F89121EC
:1003F0009B6813F0805800F0BF8523E000ED00E01B
:10040000000000080005FA05000801400010014046
:100410000000014040420F00341F0020381F002020
:1004200010E000E0780100204C28002018A001080E
:10043000000C0140EC270020B54B002283F89121ED
:1004400008F0ACFA64200EF0D6FBA022B1480021DF
:1004500017F0FDFAB04A536823F4406343F0706329
:1004600043F400635360EB69002243F00703EB6140
:10047000AB6943F4006343F00C03AB61A74B4FF04F
:10048000000B03F10C0102F801B001320C2AF5D186
:10049000FF221A765A769A76DA76A14BA14A594605
:1004A0001A60A1483022DAF8005017F0D0FA594605
:1004B000C5F3801804239D4A9B4811F802E00C22E2
:1004C0004A4302F800E0B8F1000F09D1BEF11E0F57
:1004D00001BF4FF0FF0E03F1FF3302F800E0DBB283
:1004E00001310429E7D1924A97F805A01370914B86
:1004F000914983F800A0914B884AF361C0330B60A7
:100500008F4BA90603EBCA035B7848BF0123136234
:10051000002340F2DC518B4A22F813100133082BE0
:10052000F7D11C220EA8002117F091FA15F40072E1
:100530001DBF854B149403930392BAF10E0F03D0A1
:100540000AF0EF03082B02D101238DF84A30C5F3DE
:1005500040038DF83E30C5F340338DF83830C5F395
:10056000C0338DF83B3015F400638DF8408007D020
:1005700097F8843103F1FF3EDEF1000343EB0E03F5
:100580008DF83C30C5F300438DF84130131C18BF83
:1005900001238DF84230336AB7F84821003318BF81
:1005A00001238DF84330C5F300538DF84430B7F87C
:1005B0004A3105F00100ADF84830B7F85631C5F3BF
:1005C000C001ADF84630C5F38043ED04ADF84E20D0
:1005D00048BF4F4A8DF83F3048BFB2F85021B7F8B6
:1005E000543148BFADF84E20B3F5FA7FADF84C302A
:1005F00084BF0023ADF84E3097F8CC31534A86F8CB
:100600002430002386F8253053709DF84A308DF849
:100610003900002B8DF83A100CBF0023022300B9DB
:1006200001B1013309EB8309D9F824304FF00009F7
:10063000A3F1020A163304934FF6FF723AF8023F11
:10064000934200F0B7819DF83D10DDB21B0ADAB28B
:1006500019B1A91E012940F2A9819DF8401031B1BC
:100660003B48290140583B49884200F09F819DF852
:10067000411031B13648290140583649884200F0CE
:1006800095819DF83E1051B13148334F00EB051074
:100690004168B94203D10189012900F087819DF8A1
:1006A0003B1051B12A482C4F00EB05104168B9426C
:1006B00003D10189022900F079819DF83C1051B1E4
:1006C0002348264F00EB05104168B94203D1018948
:1006D000022900F06B81DDF850E0BEF1000F12D06E
:1006E0001B4FDEF8001007EB0517786888420AD127
:1006F0003989BEF80400884200F05881BEF806002F
:10070000884200F05381022B2AD19DF838302BE02B
:100710004C2800204C1F00200000014078010020E0
:10072000FC230020322A002000240020B0E0010831
:10073000A5110020580A0020682000206028002011
:1007400098C801080E11002018A001089D01002082
:1007500070C301080004004000080140000C014083
:10076000012B04D19DF83930002B00F01F819DF83A
:10077000443033B19DF84A301BB92B1F032B98BF6F
:100780000422C34B9DF838102D015F19A1B1D11E71
:10079000C9B2012908D85B59B3F1804F00F0068136
:1007A000BC498B425DD101E1022A40F0E2805A59F6
:1007B000B94B9A4257D1F9E0012A52D19DF83F2016
:1007C000DFF8E48232B15A59B34B9A4204BF032393
:1007D00088F82730AE4AFF23511991F80DE088F8C8
:1007E0006C3088F86D30486801F1080309894FF0D2
:1007F000000BADF8541002218DF8571088F870B036
:1008000015A9C8F87C708DF856E00692059388F813
:1008100028B0C8F82CB0C8F830B0C8F834B0C8F860
:1008200068B088F86EB088F86FB00FF0E5FB059BF4
:10083000069A997850595A4608F0F7FB38465946B7
:1008400001220BF037FB954B9549C8F88030954B4A
:10085000C8F888B0C8F8843038460A1D0BF072FB1F
:10086000A4E0022A4CD15FFA89F31C2101FB03FCAE
:100870008D4B4FF0000803EB0C0B01238BF870300D
:100880000693834B8BF87190591991F80DE001F1A3
:100890000802486809898BF87280ADF8541002216B
:1008A0008DF857108BF87A8015A9CBF87C70CDF8AD
:1008B0001CC08DF856E005920FF09EFB744B059A14
:1008C00058599178424608F0B0FB069B38461A46C4
:1008D00041460BF0EFFA754A734BDDF81CC0CBF8BC
:1008E000802003EB0C01724A8031CBF88420CBF8D6
:1008F000888038460A1D0BF025FB09F1010955E0F7
:10090000032A39D19DF83F30674DDFF8D8813BB1DC
:1009100095F826B0384608214FF6FF7200231CE0F8
:10092000BDF84C2095F826B0B2F5FA7F0DD9614B91
:100930003846B3FBF2F20821BDF84E3092B208F00F
:10094000C9FB5D4B48F82B000CE05C4B3846B3FB11
:10095000F2F2BDF84E30012192B208F0BBFB584BC9
:1009600048F82B00C36095F82630013385F826300F
:100970001CE0012A3FF422AF042A17D1BDF846201B
:100980004E4B494D93FBF2F23846BDF848300121F9
:1009900092B295F8258008F09DFB95F8253005EB7F
:1009A00088080133C8F8500185F82530049B9A4522
:1009B0007FF442AE96F82520424B86F87021424AD9
:1009C000002792F800901F70A9F11702022A364DF5
:1009D0009A461AD8EB690021D85903EB070813F09F
:1009E00055FC10B1336A7BBB27E0384B07EB030E95
:1009F00098E80F008EE80F009AF8003010370133A6
:100A0000C02F8AF80030E5D1ECE7314B13F839C03C
:100A100003EBC903D3F804808AF800C0B8F1000FD3
:100A2000E0D06745DEDA294A3B0103EB020E43447E
:100A30000FCB01378EE80F00F3E7264B1A68984674
:100A400012F4805F52D11DE0234B244A13F8390081
:100A500003EBC9035E681070002EEED000238342C2
:100A6000EBDAC3EBC3017218D2F800C0DFF878E00C
:100A7000013341F80EC001EB0E079188B9809279DD
:100A8000BA71ECE709F0EF03082B154B53D155E091
:100A900070C3010800040040000800409D8A00085F
:100AA000F8010020898B000878010020659000087B
:100AB000738A000800127A00A98B000840420F00D8
:100AC000998B000818210020580A00209409002062
:100AD00098C80108EC270020A8AE0108F41F0020E8
:100AE000E81100201C210020F51F00209AF800309A
:100AF000012BC7D91A4E06EB031303F1100710366A
:100B0000BE42BFD056F8100C4FF07C5113F02AFAB9
:100B10004FF07C5146F8100C56F8140C13F022FAE2
:100B20004FF07C5146F8140C56F80C0C13F01AFADE
:100B300046F80C0CE3E7B9F10E0F09D11A78B9F1B8
:100B4000180F42F010021A700CD10EF0C3FA09E02F
:100B50001A78B9F1190F22F010021A70F4E700BFE9
:100B60009C0900200EF09AFAD8F80030BD4E5803C8
:100B70005EBFBD4B01221A70BC4A4FF002091378C8
:100B8000214643F0040313704FF40043ADF8543092
:100B900014238DF85630B3698DF8579043F0040351
:100BA000B361B3480FF028FAB24AB34B00201A6081
:100BB0000EF03AF8B14B032793E80300B36984E8D9
:100BC000030043F00803B361159816A90FF014FA57
:100BD000B369182243F48053B361F368A44843F423
:100BE0008053F3602146A0238DF8562005924FF0E4
:100BF000040AADF854308DF857700FF0FDF940231A
:100C00009B482146ADF854308DF856A00FF0F4F90A
:100C1000102397482146ADF854308DF85630049390
:100C20000FF0EAF9F1684FF0070B41F48051F160E1
:100C3000F168059A21F48051F1609149088800F427
:100C4000415040F4457038430880888B20F40060A0
:100C50000004000C8883A1F810B0088880B240F02E
:100C600040000880F16941F48041F161316941F44B
:100C7000804131618DF85770824F8DF8562038468B
:100C80004FF420422146ADF854200FF0B5F94FF44F
:100C9000804238462146ADF854208DF856A00FF01A
:100CA000ABF9049B4FF4805A384621468DF85630F4
:100CB000ADF854A00FF0A0F93369734A43F48043B0
:100CC00033613369484623F480433361138803F466
:100CD000415343F4457343F003031380938B23F490
:100CE00000631B041B0C9383A2F810B013889BB203
:100CF00043F040031380C7F810A00DF059FE002800
:100D000001F0C8824388002B01F0C4825F4F0021AC
:100D100038461022D8F8004016F099FE4FF6FF73BF
:100D2000ADF83430022304F4004A04F400694FF0B3
:100D3000000B1C408DF836308DF837B00DD00124F3
:100D400020A921F84C4D4A480CF0B0FC072387F845
:100D500000B087F801B0BC70FB70BAF1000F0ED084
:100D6000022320A921F84C3D41480CF09FFC0123AF
:100D7000E2183B71BB7107237C71FB71D4B2B9F1EE
:100D8000000F0FD0022320A921F84C3D3D480CF064
:100D90008DFC092301223B73BA73631C07227C7309
:100DA000FA73DCB273683A4843F440437360736982
:100DB000DFF8DC9043F001037361B36943F400731F
:100DC000B3610CF08DFA334B012C1593324B4FF07D
:100DD0000006169394BF334680231A934FF4807312
:100DE0001B934FF480631C93202315A91D93484641
:100DF0004FF4005318941E93179619961F960CF0F3
:100E000051FAD9F80030254A43F00103C9F80030FF
:100E10005368012C23F4702394BF0021012123F493
:100E2000807343EA0123536091681D4B013C0B40E2
:100E300043F4602343F002039360D36AE4B223F4E3
:100E4000700343EA0454D4620123BA19917800294B
:100E50007CD0B85D591C0928C9B2D278DFF83CE0D3
:100E600032D91FE000100240C00E00207A3000206E
:100E700000080140C9E80008843000204CA00108A7
:100E800000300140000C014000380040541D00209B
:100E9000080002404C240140641D00200024014051
:100EA000FDF7F1FFA0F10A04DEF80C9004EB440416
:100EB0004FF0070C0CFA04FC29EA0C0CA2404CEA97
:100EC0000202CEF80C200EE0DEF8104000EB4009E4
:100ED0004FF0070C0CFA09FC24EA0C0402FA09F2A0
:100EE0002243CEF81020062BB94C0ED8013B626B82
:100EF00003EB83034FF01F0E0EFA03FE22EA0E02ED
:100F000000FA03F3134363631FE00C2B0ED8DA1FC0
:100F1000D4F830C002EB82021F2393402CEA030E68
:100F200000FA02F34EEA030323630EE0A3F10D027D
:100F3000D4F82CC002EB82021F2393402CEA030E4C
:100F400000FA02F34EEA0303E3620B460436102E66
:100F50007FF47BAF9E4B9A6842F480729A609A68E5
:100F600042F001029A609A6842F008029A60996819
:100F7000974A090731D5FAE7531E092B3FF662AAB3
:100F8000D9F840002146206058460FF035F84FF45C
:100F90000063CBF810303C200DF02DFE97F8913116
:100FA0009845BFF649AADFF86CB208224FF40063F7
:100FB000CBF8102078200492CBF8143003930DF076
:100FC0000FFE049A039BCBF814207820CBF8103046
:100FD0000DF006FE08F10108E0E7936843F0040312
:100FE00093607B4B9F6817F00407FAD19A6842F42C
:100FF000A0029A60774BB3F85C019946002841F053
:101000004E81B9F95E31002B41F04981B9F9603167
:10101000002B41F04481D8F800309B031FD5C82035
:101020000DF0E9FDAE200FF068F908B10FF06AF994
:10103000694C85F87101C8200DF0DDFD674B00217A
:101040000C222046C5F8743116F001FD0223E3702E
:1010500008F02EFC0DF0AAFD614B0344A360614B28
:1010600000211B680C22B3F856305F480493B9F88E
:10107000644199F8638199F86B61B9F80CA099F80B
:101080000FB016F0E4FC14225848002116F0DFFCE3
:10109000574A0023137095F87831914633B10022F6
:1010A000A5F87A2153B904F04DFA07E0059304F04E
:1010B0009FFA059B002800F00B83F0E7B4F5807FD2
:1010C0000ED0BB2C0ED8612C0ED8292C0ED8132C88
:1010D0000ED8092C0ED8002C14BF062200220AE0DC
:1010E000002208E0012206E0022204E0032202E0DE
:1010F000042200E005223F4905920B88192023F0C5
:1011000040031B041B0C0B800B8823F038031B04CB
:101110001B0C43F030030B800B889BB243F0400361
:101120000B8095F87C1104F0F7F901200DF058FDC3
:10113000059A1A20114604F0EFF901200DF050FD38
:1011400015A804F0B7F99DF95630013303D19DF984
:101150005430013303D0B5F87A319BB21BB1002370
:10116000A5F87A31B4E2214B234A64201A60234A5D
:101170005A60234ADA60234A1A610DF03CFD0423C9
:10118000214A224989F80030062313700B689146E2
:1011900043F001030B6043461D4A0021092B1170E7
:1011A000904601D90B46F7E740F2023101229A40FE
:1011B000114000294CD112F0FD0F49D095F878214B
:1011C00052B30023A5F87A3172BB04F0BBF92BE0CF
:1011D000002401404C280020941C0020D429002029
:1011E000404B4C00201100205C21002038300020B2
:1011F000420F0020003001405D500008B554000847
:101200003154000890C1793D00010020E411002014
:10121000A4300020000C01400692059304F0E8F988
:10122000059B069AA0B1CCE7C34BC44A64201A6060
:10123000C34A5A600DF0DFFC0423C24A88F800302C
:10124000072389F80130136843F00203136003E0B9
:10125000012B01D900239FE70A200DF0CCFC772059
:10126000A02101220DAB03F057FF00285FD01E2103
:101270000122772004F010F84FF42F600DF0B0FC3D
:101280004FF00008A8F160010025C9B2022215AB99
:1012900077208DF854508DF8555003F03DFF9DF8A0
:1012A00055309DF8542043EA0222A74B03F5BF7145
:1012B00028F8012008F10208B8F1100FE2D1B3F8C4
:1012C0008C114FF0010E01F00F0001F47F41A3F8E3
:1012D0008C112B46DFF870C225F001026244B2F88F
:1012E0007E21002A18BF4FF0000E15F0010F03D029
:1012F000D2B25340082202E083EA1223FAE713F441
:10130000004F18BF83F4C053013A4FEA4303F6D1AC
:101310000135102DDED18C4A0143A2F88C11BEF1AB
:10132000000F04D1C3F30333984200F0D580864DFB
:1013300095F88E81B8F1000F40F0D18714200DF0A0
:101340005AFC7720D02101220DAB03F0E5FE0028E6
:1013500000F08D809DF834300322552B85F8A7319D
:10136000A5F8B02140F08380D12101220DAB772078
:1013700003F0D2FE9DF83430772003F00F021B09F2
:1013800085F8A82185F8A931162215ABAA2103F00A
:10139000C3FE9DF854209DF8553043EA0223A5F87A
:1013A00090319DF856209DF8573043EA0223A5F866
:1013B00092319DF858209DF8593043EA0223A5F850
:1013C00094319DF85A209DF85B3043EA0223A5F83A
:1013D00096319DF85C209DF85D3043EA0223A5F824
:1013E00098319DF85E209DF85F3043EA0223A5F80E
:1013F0009A319DF860209DF8613043EA0223A5F8F8
:101400009C319DF862209DF8633043EA0223A5F8E1
:101410009E319DF864209DF8653043EA0223A5F8CB
:10142000A0319DF866209DF8673043EA0223A5F8B5
:10143000A2319DF868209DF8693043EA022341F209
:101440007072A5F8A431012385F88E313F4B1A80C4
:1014500046F678125A803E4A5A603E4A9A603E4AA0
:10146000DA603E4A1A613E4A5A6100F038BF364D92
:1014700095F8B431002B40F0FF8614200DF0BBFB33
:1014800005F2B5137620D021012203F045FE95F830
:10149000B531582B37D105F5DC7388211822762019
:1014A00003F03AFE31227620F42103F0F5FE012309
:1014B0002C4A85F8B431254B9A602B4AA3F800805A
:1014C0005A6045F6D8125A80284ADA60284A1A61CA
:1014D000284A5A6100F0D0BE42F210721B4B1A80AB
:1014E0005A80254A5A60254A9A60254ADA60254A78
:1014F0001A61254A5A610323244A9370114A1368DA
:1015000043F0040313600F4D2B689A0702D50A4B72
:101510001B689847E3B21E4A0B4CBBF1000F58D032
:10152000C3BB40F259612B6813F0020F40F27123E4
:1015300018BF0B467D2137E05C2100204D5000088C
:101540004F540008E411002078010020F406002028
:1015500055530008715200083D53000831520008ED
:10156000714F00086D4F00086F4F00083553000899
:10157000E5510008094D00082D530008D551000819
:1015800025530008C55100084D4B000800010020FC
:10159000342400202B689B0759BF4FF47A731946F7
:1015A0004FF4FA634FF47A719A4505DBBAF57A6F16
:1015B000A8BF4FF47A6A00E09A464B1E5344B3FB2F
:1015C000F1F3013BDBB203FB011184F87C311160C4
:1015D00003E084F87CB1C2F800A0314BB1461B682F
:1015E0009847304A002313709046B9F1000F03D09A
:1015F000B9F1020F40F04386002620AB03F82C6DB2
:101600001E200A210122C4F8D46103F085FD0028C0
:1016100000F068869DF85430482B0CD1224B234AA9
:101620001A60234A5A60234B0222DA702B6843F077
:1016300008032B6002E0304600F054BE1E4B93F8C6
:1016400058210AB11D490A7093F859210AB11C4961
:101650000A7093F85A310BB188F800302B68194D95
:1016600013F0080F19D0BDF91080642698FBF6F42A
:10167000204612F023FC814606FB148000B212F0D3
:101680001DFC114912F06EFC0146484612F062FB47
:101690000E4912F067FC28601DE000232B601AE061
:1016A00038300020AC300020D82300205D00010835
:1016B000C9FD0008000100204C280020420F002036
:1016C000A4300020081F00208988883C00002041A9
:1016D00003200DF0FFFAB34A0A24137843F0020303
:1016E0001370B14B08221A61AF4D1920EB68013C11
:1016F00083F00803EB600DF07EFA01200DF094FA00
:1017000019200DF078FA00200DF08EFA14F0FF0485
:10171000EAD10823A54C2B612368180705D5A44BF3
:101720001B689847A34B01221A70A34BA34D1B685B
:10173000187B12F0C3FBA24912F014FC06F09CFDCA
:101740000646288812F0BAFB314612F00BFC16F060
:101750008BFB9C4B1880288812F0B0FB01469A48FE
:1017600012F0B4FC994912F0B1FC994B94491860FD
:10177000984B994D186912F0F5FB984912F0F2FB5D
:10178000974BFF2118601A22284616F060F9284668
:1017900000222A702268934B012112F0020F18BF19
:1017A000697019701FBF032119700221A9705107B8
:1017B00041BF19784D1C1D70032548BF455412F0D8
:1017C0000A0F0CD01A7804218154511CC9B2052586
:1017D0004554D11C02321970D2B206218154824D77
:1017E00029688E0641BF1A78561C1E70072648BF0E
:1017F00086540A0608D51A7809268654961C0132A2
:101800001E70D2B20A268654784E96F805E0BEF1D4
:10181000080F02D0BEF10E0F08D11A7802F1010CA8
:1018200083F800C04FF00B0C00F802C01A7811F4D6
:10183000803F4FF00C0800F8028002F1010C1CBF41
:10184000DFF8A08102325FFA8CFC83F800C01FBF72
:1018500088F80020604A4FF00E0802F80C804A0712
:1018600048BF1A784FF0120841BF02F1010C83F80B
:1018700000C04FF0100C00F802C01A7811F4806F0D
:1018800002F1010C5FFA8CFC83F800C000F80280C2
:101890000ED096F80882B8F1000F09D0DFF8448125
:1018A000023288F800204C4A4FF0130802F80C80EE
:1018B0001A7811F4007F4FF0140800F8028002F14A
:1018C000010C1CBFDFF81C8102325FFA8CFC83F82C
:1018D00000C01FBF88F800203F4A4FF0150802F8EB
:1018E0000C80BEF1180F14D11A784FF0160C00F8C6
:1018F00002C002F1010C5FFA8CFC4FF0170800F8EF
:101900000C8002F1030C0232D2B283F800C000F85E
:1019100002E00A0341BF1A78511C1970192348BF0D
:10192000835400219822324816F091F810F045FCBB
:10193000304A314B31491A6000234B800B71B6F8A5
:1019400096012F490A6081B22E4A22F81310013302
:10195000122BF9D12B68D9045CBFB6F89C11118009
:101960001B0740F11A8196F89031062B00F20F8187
:10197000DFE803F004047097AECACA002249234A84
:10198000012B0A60DFF890E02148224946D14FF050
:10199000030C8EF800C04FF0070E0B7080F800E0CB
:1019A0000C2343E07A300020000C0140E4110020B9
:1019B000D8230020F8230020742000201C000020E1
:1019C00035FA8E3C982000200AE81C4100401C4655
:1019D0000C08002038300020ED100020BD3786357F
:1019E00070200020EC100020EC2700204C28002064
:1019F0003C230020D4290020A40F002070300020B8
:101A0000D026002028280020C8270020D427002026
:101A1000CC270020FC250020C527002002238EF8BB
:101A200000300323037000230B7007231370834AD5
:101A3000834B40201A600CF0F3FF002800F0A780D1
:101A400001234FF0000A90F9000040218DE80804BE
:101A50007C4A3AE012F032FA7B4912F083FA7B4971
:101A600012F076F912F06AFC0023794A42F823005A
:101A70000133122BF9D1724A764940201160764A1F
:101A800013700CF0CDFF002800F0818001234FF08F
:101A9000070990F9000040218DE808026F4A704B59
:101AA0006FE0704A664B40201A606B4B10221A7030
:101AB0000CF0B6FF00286AD001234FF0000890F91F
:101AC00000008DE80801684A40214FF4E13358E0F6
:101AD000664A5B4B40201A605F4B08221A700CF07C
:101AE0009FFF002853D001234FF0000C90F9000015
:101AF00040218DE808105E4A4FF4E13305F06EFF97
:101B00005C4BC3F8D8013EE053490C22062BDFF8AA
:101B10008C81DFF88CC1DFF88CE157480A7010D057
:101B2000002388F800308CF800308EF800301B233A
:101B30000370524B4FF4E1381A70514B05221A7062
:101B40000EE0002188F800108CF800108EF80010CC
:101B5000212101704949DFF850810A70484A137009
:101B6000484A374B40201A600CF05AFF78B10123E5
:101B70004FF0000E90F900008DE808404346424ABD
:101B8000402105F02BFF003018BF012028B90820A4
:101B900006F064FC2A4B00221A602B682E4A13F4CC
:101BA000804F1FBF082111703848254918BF0860B1
:101BB00042F20101194079B1980441BF0821117026
:101BC00033481F4948BF0860D90741BF0C21117035
:101BD00030481B4948BF086011781806A1F104017C
:101BE000517040F1A3802348DFF8C0A04FF00009F6
:101BF000DFF8BC80C0F8DCA14946152200F5F07082
:101C0000DFF8B0B088F80190C8F80490C8F80890E0
:101C100015F01DFFAAF105034846CBF8003009F086
:101C200000FD1D4B02201B68C8F80C300CF0F8FEBC
:101C3000002841D1802006F011FC6FE07D280108CA
:101C4000D0270020F1290108CDCCCC3F0000B044C2
:101C500070260020C9280108D4270020352B010850
:101C6000A0860100B5280108892A0108A1280108D9
:101C70003D2A010878010020271D0020C3270020ED
:101C8000281D002089D00008A1D00008F9280108EB
:101C9000152901080529010810280020C427002063
:101CA000051D0020041D002090D00300322A0020D2
:101CB000280800204808002090F805E098F8013036
:101CC000C4490C2202FB03125278724504D001333E
:101CD000DBB2042BF4D9002388F80130DBF80030A4
:101CE00098F801201B7890F90000002B4FF00C03AE
:101CF00003FB021314BF4FF0030E4FF0010E00223E
:101D00005B78CDF800E00192022105F067FEB24B4E
:101D1000186000288ED0012009F083FCAF4B1868B2
:101D2000AF4B00F5C5721A6009F022FD2B680DF16A
:101D3000540813F4007F6BD0AA4ADFF8F492039B97
:101D40004FF0100AC9F800309369A74843F0010327
:101D50009361039B0CA91B888DF832A0ADF830303D
:101D600002238DF833300EF047F9D9F800309E4841
:101D70005B880CA9ADF8303004238DF832300EF0BA
:101D80003BF9D9F800104FF00F0E0B7A4FF0010B12
:101D900003F0030203F0FC0303F1804303F58033F7
:101DA000986892000EFA02FE20EA0E009860986889
:101DB0000BFA02F202439A604B688C4A4046536128
:101DC000159300238DF8583003938DF859A08DF8A2
:101DD0005AB011F057F8D9F80020039B527A0DA899
:101DE0008DF8342003228DF835208DF836308DF8AB
:101DF00037B011F029F87E4B7E4A1B683C3B1360DC
:101E000023684FF0FF3243EA0A0323607A4B1A60DB
:101E10007A4B7B4A7B4C13607B4A803313602B6880
:101E20004FF00009D90384F8009040F1C0800FF012
:101E3000FFF840F22A33DFF8FCC14FF0010A1A46DE
:101E400060464946CDF814C0049384F800A015F00C
:101E5000FEFD644A4FF0100B9169634841F00801A0
:101E6000916118218DF8331003218DF832100CA9DF
:101E70000392ADF830B00BF019FC039A6348D169B6
:101E8000634C41F00201D16162490968B1FBF0F194
:101E90002088013920F45C7000FA0BF020FA0BF076
:101EA000208089B21D20A0852185A4F814A0218C52
:101EB00021F0010101FA0BF121FA0BF12184218CAF
:101EC000B4F804E0208B21F0020120F0730000FA46
:101ED0000BF001FA0BF120FA0BF021FA0BF11FFACB
:101EE0008EFE40F0600041EA0A01A4F804E020837D
:101EF000A4F834902184218B21F0080101FA0BF120
:101F000021FA0BF141F008012183B4F844106FEA83
:101F100041416FEA514189B2A4F84410516941EA44
:101F20000A0151613C4A104603920BF0D9F9049B17
:101F3000039A3A4918938023DDF814C01A934FF49A
:101F40008073104615911B9341464FF400531E9326
:101F5000CDF86490CDF87090CDF87490CDF87C9069
:101F6000CDF858C0CDF85CB00BF09CF9A389039A6A
:101F70009BB243F40073A38113680DA843F00203DE
:101F800013608DF834B08DF835A08DF836908DF84B
:101F900037A010F059FF224B1A68224B43F8272034
:101FA0000137202FF7D10DF049FF0DF047FF2B68C7
:101FB0005A0540F18A801C4C1C4BD4F82095042013
:101FC000C3F800900CF02CFD0421C4F824050CF09B
:101FD00003FD31E0C4A00108901C00202011002066
:101FE0000010002000100240000C014000040140DD
:101FF000102800202008002040110020642A002022
:10200000AC120020C10E0020D41C002000366E014E
:1020100000040040040100206C0002403404004031
:1020200054A00108C20E002078010020D811002021
:10203000240800206D030020AF4B84F828050820F9
:10204000C3F800900CF0ECFC0821C4F82C050CF04F
:10205000C3FCAA4F84F83005002138462C2215F025
:10206000F6FC8E237B704FF07C0BE0234FF07D0A53
:10207000FB7087F800B087F82BA0A14F2C2200211D
:10208000384615F0E4FC8A237B701020A023FB70F7
:1020900087F800B087F82BA0C4F834950CF0C0FC8A
:1020A0001021C4F838050CF097FC84F83C0520207A
:1020B000C4F840950CF0B4FC2021C4F844050CF0A1
:1020C0008BFC84F8480507F0F3FA8E4C0027238830
:1020D000322023F040031B041B0C238023884FF481
:1020E000805923F038031B041B0C238023889BB2E8
:1020F00043F0400323809F238DF834308DF83570F2
:102100008DF836708DF837700CF075FD8DF85570C0
:102110007D4F0DAA0423C7F814902046414603F0D2
:1021200023F9C7F810909DF856209DF855301202FB
:1021300042EA03429DF857301A43744B9A42744B5B
:1021400017D008D873498A420CD001F51A410231E0
:102150008A4209D01CE070498A4205D001318A4286
:1021600007D015E0202200E080221A804FF4807210
:1021700002E04FF480721A805A809A8819881202FD
:102180009A604A43DA60654A012182F8491504E001
:1021900000221A805A809A60DA60DF68FFB13F0C33
:1021A000B9464FF0000ABA4512DA0AEB0704641088
:1021B0002004414610220EF04DF8002358F8232049
:1021C000013263D10133042BF8D12746A146EAE757
:1021D00009F086FC514A4FEA0943C2F84C352B6896
:1021E0004F4A13F4002318BF012313700CF0DEFCD8
:1021F0004C4B18607379052B02BF4B4B4FF4C872E0
:102200001A804A4B4FF47A721A80494BC8221A80BE
:10221000484A137843F008031370474A137823F0B1
:102220000203137040F602032A6813406BB143495E
:10223000434B1960434B03211970434B0121197023
:10224000424900230B8042490B80930341BF414B1D
:1022500004221A71DA7844BF42F00102DA70B368DE
:1022600001222B603C4B1A703C4A137863F07F03C9
:10227000137021B0BDE8F08F0423FFF73DB9B9F129
:10228000010F7FF6DBA99946FFF7ABB904F1010A0C
:102290004C469BE701200EF0C5F8FEF737BD304BEA
:1022A00000221A7000B211F009FE2E4911F05AFEF8
:1022B0001590B9F95E0111F001FE2A4911F052FEA4
:1022C0001690B9F9600111F0F9FD264911F04AFEA6
:1022D0002549179015A805F0D9FFFEF79CBE0223EB
:1022E000FFF70AB9B9F1010F7FF6A8A94FF000096D
:1022F00088F80000FFF780B930120020001200209B
:102300003512002000380040000C014018BA2000AF
:102310000C000020152020001740EF00780100205D
:1023200030240020CC080020B60F00209E30002072
:102330009C300020E8110020A6300020C629002093
:10234000D011002034120020F8000020600F00207F
:10235000620F0020941C0020C00E00207A30002064
:102360004C00002035FA8E3C301D0020B54B2DE985
:10237000F04FB3F90610B44B85B01F6801937A890A
:1023800091420EDBB1F5FA6FFC79BFBF8B1A634344
:10239000A2F5FA6493FBF4F4ACBFC4F164046434B2
:1023A00000E06424A94BAA4AB3F896B193F96231CC
:1023B00012689BB2029215460393002240F2E63067
:1023C000A04B4FEA420C33F912E0CBEB0E0303F2C1
:1023D000F316864203D8002BB8BF5B4201E04FF4EE
:1023E000FA73022A2ED0029E96F811611EB1B342F2
:1023F000CCBF9B1B0023642093FBF0F8954E6FF03D
:10240000630A36F818900AFB083A08F1010836F911
:1024100018600FFA89F8C8EB060606FB0AF696FB69
:10242000F0F68D484E4420F80C60BE1836796420D2
:1024300073438A4E93FBF6F364339BB2634393FB7F
:10244000F0F02CE0029890F812611EB1B342CCBFBC
:102450009B1B0023642093FBF0F0DFF82C926FF0BD
:10246000630808FB003A39F91060013039F91000AF
:10247000002BA0EB060000FB0AFA9AFBF8FA03987F
:10248000C6EB0A0A0AFB00FA7348B8BF5B42A0F821
:1024900004A0B8794343714893FBF0F064306B7843
:1024A0004FF06408434393FBF8F36D4E022AB35494
:1024B000EB7A6C4E00FB03F393FBF8F3B3546B7DA4
:1024C000654E00FB03F090FBF8F0674B9854674BA8
:1024D0000ED1DE4583F802800DDB5C4CB4F8982108
:1024E000914214DBB1F5FA6FA8BF4FF4FA610FE027
:1024F000DE459C5404DA36F80C305B4226F80C308A
:102500000132032A05F101057FF458AFE5E71146D2
:10251000891A4FF47A735943C2F5FA62B1FBF2F1AA
:10252000642391FBF3F2DFF874E16FF063073EF888
:10253000120007FB021101323EF9122007B2D21B32
:10254000514391FBF3F30344F380494B424D1B8805
:102550005F063BD5474A484B10881B88181A00B2C3
:1025600011F0ACFC454911F0FDFC074605F084FE76
:102570008046384605F00DFE0746B5F9020011F019
:102580009DFC8146B5F9000011F098FC4146824659
:1025900011F0E8FC39468346484611F0E3FC014659
:1025A000584611F0D5FB11F0A3FE4146288048465D
:1025B00011F0D8FC39468046504611F0D3FC014654
:1025C000404611F0C7FB11F093FE68802C4D2B683C
:1025D000980740F19E8045F207212A4B2A4F1A683E
:1025E0007B69D31A8B4240F394807A610BF0C2F975
:1025F000264BDFF8AC901A789846032AB9F80030D9
:1026000050D10A2B58D90023282088F800300CF02C
:10261000F2FA0BF0AFF91E4B18880BF095F91D4B31
:102620001A68D37890FBF3F0013008281A4BA8BF42
:1026300008201870537980B243433B831379584381
:10264000788339E028280020481100204C280020F9
:1026500020110020261F0020C81100200CFEFFFFC3
:10266000AC1E0020560F0020C41E0020F81D0020C4
:10267000A8120020FA0F0020C011002035FA8E3C6D
:10268000EC27002088300020480F00203412002062
:102690006C1D0020D0110020F80000200E1F00202B
:1026A000D41100200A2B07D803239B4A88F8003056
:1026B000002313703B837B8398F80030974A012BEB
:1026C0000CD002D3022B1BD023E03A8BB9F8003098
:1026D0009A421EDD012388F800300FE0B9F800109F
:1026E0007B8B8B4202DD022313700FE08C4B1B8B24
:1026F0000133994202DD002313700AE0082006E04E
:102700007B8BB9F8002001339A42E3DC07200CF000
:10271000A7FA2D68290575D5824B814F1A68FB6988
:10272000C3EB020845F2072398456BDDB6F9063086
:102730004FF47A71A3F57A7B7B4BFA61D3F8009062
:1027400098FBF1F899F80A30B4F85201012B774E52
:1027500003D040D3022B1FD03FE0754B386A5A7B21
:10276000744B4FF0080E33F8122090FBFEF392B238
:10277000C01A83183B6293FBFEF3BA8440F6E4422E
:102780009BB25343B9F80820C2EB13334B43B9F95A
:10279000062093FBF2F31FE0674BB9F808A01B7803
:1027A000C6F800A05A0718D510F0CBFD20B915F0D7
:1027B000100F18BF4FF0000B0BFB0BF1322391FBF6
:1027C000F3F3B9F906205B445A434FF47A7392FB52
:1027D000F3F3534400E0002333603368D7E90A0180
:1027E00003FB08F84FF47A7398FBF3F810EB08003A
:1027F00041EBE8710023C7E90A01504A11F0BEFD20
:102800004F4B18604F4E3368DB0427D52F0622D577
:102810004D4B1B789D071ED54C4B187804281AD9B0
:1028200000224B4B0521D718951C4FF00A0E122A97
:10283000D154E9B287F801E004D0B0EB510F2A4639
:10284000EFD800E014215A18322002F8010CFF22C0
:102850005A540F2000E00A200CF002FA3D4D2A687D
:10286000002A51D03C4B3D4F186839689846814248
:102870004AD83B4BDFF8F49019785268E1B94FF031
:10288000010A83F800A0B9F80030D35C23B35046A6
:102890000CF0CAF9334B83F800A010F0B1FAB9F884
:1028A0000030CBB92B681B78053B534514D80CF08E
:1028B0007DF92D4B18600FE04FF0000A83F800A05F
:1028C000B9F80030D35C3BB150460CF0ADF9254B64
:1028D00083F800A010F094FA2B68B9F800205B6828
:1028E00022499B5CFE2B02D100230B800CE0FF2BC6
:1028F00002D10CF09FF907E0D8F800000A2505FB8B
:10290000030301323B600A800B4D2B78580731D509
:10291000174B08225A616BE0F800002034120020A7
:10292000480F002088300020D0110020DC1100204A
:10293000541D0020641D0020A6300020407E0500AC
:10294000E0110020E8100020E8110020EE11002026
:1029500068210020481F002010280020401F002070
:102960003C1F0020D7270020EC250020441F00201A
:10297000000C01403268D1075CBF43F001032B70AB
:10298000984B1B781F075EBF2B7823F001032B7039
:10299000D60248BF2B78944A44BF23F001032B7022
:1029A000924B1B6813F0040F02D09149098851B96A
:1029B0009049098809B1980705D48F4B1B880033CB
:1029C00018BF012333B1022313702B7823F00103C6
:1029D0002B7004E02978C90758BF022313700CF04C
:1029E000E5F8864B1B68C01A002801DB10F008FAD6
:1029F00006F05EFE824B1E789846002E00F0AB80FB
:102A0000804E3368002B00F0E78630680CF09EF9AA
:102A1000002800F0E1867B4B7B4C18680CF093F9A2
:102A2000092801D03F2850D14FF0000A5746D4F86A
:102A30000090764DB9F1000F05D0754829684A46D7
:102A400015F052F810B9AA4607B92F46714B103548
:102A50009D42EFD3C7B1D7F800E0DAF800C0236891
:102A60001EF803501CF80300A8420DD15A1C6849F7
:102A700038B92D2B05D8644D2A602025CD548854B3
:102A800002E0CD542260EAE723680BB1574511D02C
:102A900061480DF0B7FF574507D857F8100B0DF0F8
:102AA000B1FF09200DF0A6FFF5E75C480DF0AAFF85
:102AB0004FF0000923689945A7D2554B13F8090038
:102AC0000DF098FF09F10109F4E72368002B40F0AD
:102AD0006886042840F0A1864D4809F0A1FD00F069
:102AE0007BBED9F80000DFF844A10CF02FF940B309
:102AF000DAF800000CF027F9DBF80030024693F812
:102B00004810002935D1242840F09280012283F812
:102B10004820DBF80030DFF810A193F84820062A9F
:102B2000DFD193F8490002F0A5FD8146002800F0AE
:102B3000A3803B6898790DF0B2FE3B68002283F8D1
:102B40004820374B93F83530002B40F018864C3630
:102B5000982E00F04186334BF21892F84A10012962
:102B6000F5D1314FF3583A60304ABB461360914675
:102B7000B7E7012904D14D2814BF00220222C6E77D
:102B8000022904D13C2814BF00220322BFE70329F5
:102B90000CD140284FF0000102D983F84810B8E763
:102BA00058711971D97198710422B0E7042906D1BE
:102BB000997983F849004A409A710522A7E70529C7
:102BC000A7D1587919798842987906D950409871D7
:102BD000481C18710B441A729BE790420CBF0622E6
:102BE000002294E7E8110020D7270020E4110020FC
:102BF0009C300020B60F00209E300020D8270020F7
:102C0000A730002014210020D01C002008AC0108AF
:102C1000A01C0020E8AD010830C7010835C7010835
:102C2000480F00203C230020881200208C12002036
:102C30002B7858073FF56DAF232ADAF800300ED114
:102C4000012188F80010AE49AE480B60AE490292EF
:102C50000B630DF0D7FEAD480DF0D4FE029AAC4BDD
:102C60001B681B78934201BFAA4AAB4B1A60AB4A60
:102C700004BFAB4BDA604CE7DAF8002092F8493039
:102C80004A2B00F038815CD8332B00F09E8421D889
:102C9000292B00F0388409D8252B00F00F84272B2E
:102CA00000F01384232B40F0B4853CE22D2B00F080
:102CB0003B8407D82B2B40F0AC850DF0D3FD607121
:102CC00000F058BD2F2B00F00885312B00F01A853D
:102CD00000F09FBD3E2B00F004811DD8372B00F083
:102CE000C48404D8352B00F0578200F092BD392BF4
:102CF00000F0F8833C2B40F08C85DFF82892D9F85F
:102D000000A00DF0AFFD8AF80000D9F80030187867
:102D10000CF048FC00F02EBD432B00F0838406D855
:102D2000412B40F076854FF0000900F053BC442B56
:102D300000F01C85482B40F06C8508F00FFF00F078
:102D400019BDD02B00F0338368D8CA2B00F0F28075
:102D50001CD84E2B00F00B8410D84C2B40F059851A
:102D60000DF080FD84F8CE010DF07CFD84F8CF01DC
:102D70000DF082FDA4F8D00100F0FCBCC82B00F0DF
:102D80008380C92B00F0348300F043BDCD2B00F0CD
:102D9000198304D8CC2B00F0278200F03ABDCE2B4B
:102DA00000F01983CF2B40F034850DF065FD6FF4F2
:102DB000AF6283189BB2C62B98BFA4F896010DF0A2
:102DC0005BFDA4F844010DF057FDA4F846010DF099
:102DD00053FDA4F848010DF04FFDA4F8D0010DF00B
:102DE00041FD84F8E1010DF03DFD0DF03BFD84F85F
:102DF000E2010DF037FD84F885010DF033FD84F814
:102E000092010DF02FFD474BD3F800900DF034FDEB
:102E100000EB80004000A9F8560063E3D62B00F0D9
:102E20004B820AD8D22B19D0C0F00983D32B25D0DE
:102E3000D42B00F04C8200F0ECBCEF2B41D005D835
:102E4000D82B40F0E6844FF00009FFE0F22B00F0B1
:102E50008682FA2B00F0C88200F0DBBC2B78590781
:102E600000F188840DF0FEFC022884F8A00740F2EF
:102E7000A4822D4B002283F8A0279EE20DF0FCFCDB
:102E80002A4B188000F076BC92F805904FEA590959
:102E9000B9F1120F03D90FF01BFA00F06BBC4FF021
:102EA000000ACA4507D20DF0E7FC214B23F81A00AF
:102EB0000AF1010AF5E7144B012283F8342000F0EF
:102EC00059BCDFF86090D9F800A00DF0D5FCAAF845
:102ED0005A00D9F800900DF0CFFCA9F8580000F086
:102EE00049BC0DF0BFFC84F8D4010DF0BBFC84F8A4
:102EF000D30100F03FBC0DF0BFFCA08100F03ABC54
:102F00001421002065C70108480F002035C70108BB
:102F1000FC230020EFBEADDEF04F00200400FA05D8
:102F200000ED00E0201100204C280020F80F0020C8
:102F300028280020D64B1A689A461278022A6AD1AD
:102F4000DAF8003009F1080B02930DF08BFC10F059
:102F5000B1FFD04911F0BAF8029B43F82B00DAF820
:102F600000B00DF07FFC09F10A030BEB830B10F0AE
:102F7000A1FFC94911F0AAF8DAF80030CBF8040033
:102F800002930DF06FFC10F095FFC44911F09EF80C
:102F900009F10E0B029B09F10109B9F1030F43F886
:102FA0002B00CDD1B9F1070FDAF800B01AD10DF02E
:102FB00059FC10F07FFFB74911F088F8CBF84400B6
:102FC000DAF800B00DF04EFC10F074FFB14911F0CA
:102FD0007DF8CBF84800DAF800B00DF043FC8BF830
:102FE0004C0012E00DF03EFCCB448BF80100DAF807
:102FF00000B00DF037FCCB448BF80B00DAF800B0D2
:103000000DF030FCCB448BF8150009F10109B9F142
:103010000A0FC7D1AEE3DAF800B00DF023FCCB44C1
:103020008BF80100DAF800B00DF01CFCCB448BF8F3
:103030000B00DAF800B00DF015FCCB4409F10109E2
:10304000B9F10A0F8BF81500E5D193E3DFF840A240
:1030500009F1080BDAF8003002930DF00DFC10F0C6
:1030600029FF8E4911F032F8029B43F82B00DAF861
:1030700000B00DF001FC09F10A030BEB830B10F01B
:1030800019FF864911F022F8DAF80030CBF8040075
:1030900002930DF0F1FB10F00DFF804911F016F8CE
:1030A00009F10E0B029B09F10109B9F1030F43F875
:1030B0002B00CBD1B9F1070FDAF800B01AD10DF01F
:1030C000DBFB10F0F7FE754911F000F8CBF8440077
:1030D000DAF800B00DF0D0FB10F0ECFE6F4910F004
:1030E000F5FFCBF84800DAF800B00DF0C5FB8BF81F
:1030F0004C0012E00DF0C0FBCB448BF80100DAF875
:1031000000B00DF0B9FBCB448BF80B00DAF800B03F
:103110000DF0B2FBCB448BF8150009F10109B9F1B0
:103120000A0FC7D126E30DF09DFB132883463FF617
:10313000B2AEDFF85CA1DAF800900DF093FB00234B
:1031400057490C2202FB0312117A814220D11378D5
:1031500009EB8B0989F879300DF084FB89F87A0046
:103160000DF080FB89F87B000DF07CFB4D4A4E4B47
:1031700089F87C001A60DAF800004C4B00211860D6
:1031800079300BF0D9FC4A4B80F001001870F1E265
:1031900001331B2BD4D17EE60DF064FB0B28824655
:1031A0003FF679AE3A4BD3F800900DF05BFB032865
:1031B0003FF671AE062303FB0A9989F8CE000DF0A5
:1031C00051FB89F8C9000DF04DFB89F8CA000DF0DC
:1031D00049FB89F8CB000DF045FB89F8CC000DF0D8
:1031E00041FB89F8CD00C5E25379092B7FF653AE38
:1031F000019BD3F800900DF035FB019B89F800008E
:10320000D3F800900DF02EFB89F801000DF02AFB99
:10321000019B64281B68A8BF642018710DF022FB75
:10322000019B64281B68A8BF642058710DF01AFB2D
:10323000019BFF281B68A8BFFF2098710DF012FBAF
:10324000019B6428D3F8009028BF642089F8070008
:103250000DF008FB019B89F80200D3F800900DF0F7
:1032600001FB019B89F80300D3F800900DF004FBEB
:103270003B68A9F80A005B790A2B40F27B820D4B70
:10328000D3F800900DF0EEFA89F8080072E200BF62
:1032900020110020000020410000C84200007A44B4
:1032A00018A5010890290020F00F0020F40F00203D
:1032B00008000020481100200DF0DEFACB4B23F867
:1032C000190009F10109B9F1080FF5D152E253795A
:1032D0000F2B7FF4E0AD0DF0C5FA072881463FF6CD
:1032E000DAADDFF834A3DAF800B00DF0C5FA0E233A
:1032F00003FB09F9CB44ABF81901DAF800B00DF083
:10330000BBFACB44ABF81B01DAF800B00DF0B4FA0D
:10331000CB44ABF81D01DAF800B00DF0A3FACB44B2
:103320008BF81F01DAF800B00DF09CFACB448BF853
:103330002001DAF800B00DF095FACB448BF82101AA
:10334000DAF800B00DF08EFACB448BF82201DAF8EF
:1033500000A00DF09BFAD144C9F823010AE20DF058
:1033600081FA0F2881463FF696AD0DF07BFAC9EB46
:10337000C909A14489F8D4000DF074FA89F8D50080
:103380000DF070FA89F8D6000DF06CFA89F8D700C4
:103390000DF068FA89F8D8000DF064FA89F8D900C0
:1033A0000DF060FA89F8DA000BF094FEE2E12B7878
:1033B0005B0700F1DF810EF055FA05F081F805F0AA
:1033C00021F9D7E12B78580700F1D481884B4FF4CD
:1033D000C8721A80CEE12B78590700F1CB81854A5B
:1033E000137843F0040328E02B785A07E5D510E260
:1033F0000DF038FA7F4B1A7810B142F0020201E06A
:1034000022F002021A700DF02DFA7B4BDFF80C92BD
:1034100018700DF03BFAC9F800000DF037FAC9F842
:1034200004000DF029FA754B18800DF025FA744B45
:10343000744A1880137843F0020313709AE10DF078
:1034400011FA02900DF022FA83460DF01FFA82461F
:103450000DF01CFA81460DF00FFA0DF00DFA0DF08B
:1034600001FA029BA3B9684B1020C3F800B0C3F85F
:1034700004A004F0D2FF5F4A137843F001031370F5
:10348000B9F1000F00F07681604BC3F8009071E154
:10349000102B40F06F815E4BC3F800B0C3F804A05E
:1034A000B9F1000F02D0594BC3F800905848594B5E
:1034B0000222011D1A7008F015F95BE1A0600DF001
:1034C000E5F9A3681843A06054E10DF0D5F9A4F81C
:1034D0005C010DF0D1F9A4F85E010DF0CDF9A4F86E
:1034E000600147E10DF0BEF984F87A010DF0BAF9F8
:1034F00084F87E010DF0B6F984F87D010DF0B2F983
:1035000084F87F0136E10DF0B7F9A4F880010DF0E1
:10351000B3F9A4F882010DF0A5F984F884010DF047
:10352000ABF9A4F8860125E10DF09CF984F890012F
:103530000DF0A2F9A4F89A010DF09EF9A4F89601F5
:103540000DF09AF9A4F898010DF08CF9DAF8003032
:1035500084F891015B79082B40F20C810DF08CF915
:10356000A4F89C010DF088F9A4F89E0102E192F8FC
:1035700005900323B9FBF3F9B9F10E0F3FF68BACBD
:10358000DFF89CA04FF0040BCB4580F0F3800DF0EA
:1035900069F98AF8A0010DF06FF940F2ED23984225
:1035A00005DD40F6CA039842A8BF184601E040F284
:1035B000EE20A0F2EE20192390FBF3F00BF1010BAB
:1035C0008AF8A1010AF1020ADEE70DF04BF984F84E
:1035D0009201CFE00DF046F904EB090309F101096E
:1035E000B9F1080F83F88801F4D1C3E0FA20002074
:1035F000B60F0020E8110020EE110020EC11002091
:10360000EA1100204E11002050110020601100200E
:1036100058110020FC0F002020110020F011002084
:103620004C2800200DF01EF9C4F8089060710DF0D0
:103630002DF9A3681843A0600DF014F984F89001E7
:103640000DF01AF9A4F85C010DF016F9A4F85E016A
:103650000DF012F9A4F860010DF00EF9A4F8800144
:103660000DF00AF9A4F8820184E053794FF0070ABB
:10367000B3FBFAF2C2EBC2029A1A12F0FF0F7FF408
:103680000AACB3FBFAFA0AF1FF3A5FFA8AFABAF126
:10369000FF0F6FD00DF0E6F85FFA80FB4FFA8BF06A
:1036A0000BF086F9814600283FF4F5AB80F800B0B6
:1036B0000DF0E2F8A9F802000DF0D4F889F8040042
:1036C0000DF0D0F889F805000DF0CCF889F8070066
:1036D0000DF0C8F889F80600D5E7DFF8509209F137
:1036E000400A0DF0C9F8A9F898020DF0BBF889F866
:1036F0009A020DF0B7F809F1040989F89702D1454B
:10370000EFD137E00DF0AEF81F2881463FF6C3AB8E
:103710003B685B79082B7FF4BEAB0DF0ADF809F187
:10372000860904EB890A00F03F00AAF802000DF0B8
:10373000A3F8BAF80230800100F4FE501843AAF84A
:1037400002000DF08FF8000104F829000DF08AF84E
:1037500014F8293000F00F00184304F829000DF088
:1037600081F88AF801000DF063FC03E05D4B012253
:1037700083F8352000200DF0C1F8FFF7DAB95A4B75
:1037800098590BF0DAFA18B932200BF034FAF6E750
:103790000BF05EFC04F06AFE544A554BDA60FFF70A
:1037A000D6B90C283BD00A2842D1524D52480DF0D0
:1037B00029F92846232114F080F908B1401B206024
:1037C0002368002B57D14B4800213022236014F08E
:1037D0003EF998F800302BBB484B1B689B060FD571
:1037E000474B40491B688A6B9A1A002A08DB454AF6
:1037F0001278042A82BF03F5123303F5F8738B6342
:10380000414B9B68002B69D0404805B0BDE8F04FA4
:1038100018470EF05DFDFFF78CB90C2804D13C4829
:103820000DF0F0F83B480DE07F2812D1FFF7EDB81E
:103830000D28BAD07F2809D12E4A013B00213648F5
:103840002360D1540DF0DEF8FFF7DFB82F2B3FF6E1
:10385000DCA8A0F12002D2B25E2A3FF6D6A813B9A6
:1038600020283FF4D2A85A1C2260224AD0540DF0DE
:10387000C1F8FFF7CAB85A1EA95C202901D1134626
:103880009FE71C4A00212360D154244B244DD3F8D8
:1038900000A0D5F800B0DFF85C90584614F01BF992
:1038A000074659463A46484614F01EF91D4A28B9BB
:1038B00019F8073053445B785B0703D01035954205
:1038C000E7D306E0954204D2781CEB684844984759
:1038D00002E015480DF096F8002374E705B0BDE846
:1038E000F08F00BF480F00203C2300200400FA05A1
:1038F00000ED00E0A01C002069D60108E4110020C2
:1039000088300020EE11002038300020840F002085
:103910003AC7010835C7010861C701080C0100203A
:1039200008AC0108E8AD010845C701084C28002093
:103930002DE9F04FA04EA14D3368A14C03F59C43F7
:10394000203323602B889F4A01332B8042F20103EE
:10395000116889B00B4092461BB19B4A1378013322
:1039600013700FF089F9DAF80030DF0405D5974BB2
:103970001B68D80701D40EF04DFF954B37681A68C5
:10398000907AB8B19349137B013831F810001BB11C
:10399000C0F53B60083080B200B2A0F57A70B0F597
:1039A0007A7FA8BF4FF47A7020EAE07010F086FAB0
:1039B000894930E0DAF80030190435D56368804E63
:1039C000FB1A002B30DB07F59C4320337360834BDD
:1039D000D27A5979824B33F81130317A9BB293FB0A
:1039E000F2F3013101F00F02327232445372034696
:1039F0007C4A825C0130134410289BB2F8D11BB280
:103A000093FBF0F000B26428A8BF642020EAE070C5
:103A100010F054FA744910F059FB744910F0A2FAEE
:103A200010F08CFC724B1880DAF80030694E13F4F9
:103A3000807F00F081806F4B9F4204D92B7913B9AE
:103A40005E4B01221A71B5F900E06B4ABEF1140F0A
:103A50001778CCBF4FF0000E4FF0010E574BC7F355
:103A60008007BEF1000F06D04FF0000883F80680F3
:103A700083F8058001E04FF00308E369A87901931A
:103A8000D4F820C0B5F9009069796B883288032892
:103A900048D8DFE800F0020E1B36BEF1000F02D05E
:103AA000328000222BE0002F40F062863280AF711E
:103AB0003AE09CF8000000EB8000814502DC328097
:103AC00001221CE001206FB300F0DABE47B1019A79
:103AD0004FF00208D2897280B280BCF80200F080F8
:103AE0009CF800B09CF80100584400EB8000814530
:103AF00000F34186002F00F03E8632800222AA7138
:103B000012E032800322AA7169716B8077B13A4A60
:103B1000137843F002031370284B00225A710EF001
:103B200079FE03E03280A87169716B80B8F1000FF3
:103B300002D040460BF094F8304FB7F852010FF026
:103B400000FC0197834668B90FF076FF2C4B0022EA
:103B5000C3F800B0C3F804B0C3F808B0294B1A602A
:103B60005A609A60244F3B785B0763D5DAF80030DF
:103B7000D8065FD5244B1B78D9065BD4234B1B7822
:103B800093B1019B93F8D431BBF1000F42D173B1D3
:103B90001F4B1A68636A9B1A002B08DA0EF03AFE74
:103BA000074B83F828B045E0BBF1000F3AD1102055
:103BB0000BF056F801233BE08830002070300020E5
:103BC000880F0020EC270020D4260020E8100020D9
:103BD000D02600202828002000007A44541D002010
:103BE000641D0020910F00200000C84200C07F44E7
:103BF00044110020404B4C00A63000204C280020EF
:103C0000241E0020E41E0020E811002008000020EF
:103C10001028002033B1AD4A4FF47A71126801FBCD
:103C20000323636294F8283023B10BF003F80023D8
:103C300084F82830019B93F8D2310293019B93F8CA
:103C4000D311B3F898E1B3F89AC10023184636F9B6
:103C5000132080087245C4BF60F07F00C0B20133FA
:103C60006245B8BF40F04000042BF0D194F82930F1
:103C7000974A834205D192F82A30F92B04D80133B0
:103C800000E0002382F82A30924B84F829001A7849
:103C9000DFF85C829946DAB9D8F80030DA0708D53F
:103CA000BBF1000F14D13B78DB0711D50EF00AFCF5
:103CB0000EE03B7858070BD5874B1B7843B16B79E7
:103CC00033B911B10EF0A6FD02E0BBF1000FF9D03F
:103CD00094F82A307E4A142BDFF818B240F08F8017
:103CE000029B003318BF0123029399F8003063B39D
:103CF00092F829305F2B11D13B7803F0040303F0D5
:103D0000FF0113B10EF086FD08E00B200491039231
:103D10000AF0A6FF039A049982F82A10029BA3B125
:103D200094F829307D2B10D13B7803F0040303F085
:103D3000FF0213B10EF06EFD07E00B2003920AF0B4
:103D40008FFF634B039A83F82A203B7803F0040328
:103D500003F0FF01002B52D194F829305C4A572B15
:103D600016D15E4B4FF47A721A80DAF800301906D9
:103D700001D507F04DFD5A4B1B685A0742BF594AFF
:103D80000A21118013F0080339D1574A138036E015
:103D9000DAF80000400717D55A2B15D192F82B30CE
:103DA0002BB1012382F82B1082F82C3027E092F8F7
:103DB0002D3083F0010382F82D300BB10C2000E090
:103DC0000D200AF04DFF1AE05D2B00F0D7845B2B2D
:103DD00000F0D6845E2B02D1032000F0D2BC562B1B
:103DE00001D104F0DBFD99F80030002B00F0DE84F7
:103DF00094F829306F2B40F0D4840EF063FBDAF88E
:103E000000305B0736D594F82D30314A93B13B78BA
:103E100058070FD5019BB6F90610B3F898319942AF
:103E200008DDD8F8003013F0010302BF32211186FB
:103E300082F82D30D8F80030D9030CD594F8322010
:103E4000234B22B993F82B200AB932221A86012378
:103E500084F832300EE094F82B301D4A53B13B7891
:103E600003F0040303F0FF0123B9012382F82B10B0
:103E700082F82C30DBF800700023C8F8003007F11E
:103E80007B0607F1CB093278737816F8010C9A4259
:103E90000DD231460AF02CFE48B116F8022C01234F
:103EA00003FA02F2D8F800301343C8F800300436A1
:103EB0004E45E8D10D4B1B78F3B10D4E084F3368DA
:103EC00013F0020F40F03A8332E300BF10280020C5
:103ED000880F002008000020D62700209E300020F8
:103EE000E41100209C300020C0110020A7300020E9
:103EF000E81000202011002007F1CA0607F5897795
:103F00003278737816F8010C9A4222D231460AF0C0
:103F1000EFFDF0B196F804E00C21B37801FB0E41FF
:103F2000B44A013B03EB430313448A6B96F80380C6
:103F30009A42B1480DD08B63002390F86420CB6384
:103F4000012303FA0EF322EA030381F8348080F898
:103F500064300636BE42D3D1A84BDFF8BC921F684E
:103F6000A74B4FF0000B1B680293A64B1B780393E3
:103F7000D9F80030002B00F0C48293F80080B8F12B
:103F8000000F00F0BE82D9F8042002998A1A002A94
:103F90000CDB01F5FA72C9F8042094F864100122D0
:103FA00002FA0BF221EA020284F86420039A002A42
:103FB00000F0A78219F8042C59780432D2B20029F3
:103FC00040F06082904931F91210904AB2F896217F
:103FD00002F1C800814201DD9E7814E0C83A9142A6
:103FE00002DA99784E420EE094F86420012303FA35
:103FF0000BF322EA030384F86430029B03F5FA739F
:10400000C9F804307DE294F8643043FA0BF3DA0720
:1040100000F17782002ECCBF022001200AF042FE80
:1040200008F1FF32744B132A00F26382DFE812F0CA
:10403000140021002E003D0056005D00C1003A0131
:104040009E01CB01FA0161023D004C005D00C10000
:104050003A0193000C017001397838460E44FA2E6B
:10406000A8BFFA2626EAE6763E700AF027FD012070
:1040700019E0797838460E44642EA8BF642626EAF3
:10408000E6767E700AF01AFD02200CE0F9783846D8
:104090000E44642EA8BF642626EAE676FE70996E6A
:1040A0000AF0C4FC03203146B9E179790D2031448E
:1040B0006429A8BF642121EAE17179710AF062FDE7
:1040C000B8F10D0F00F0158239790E2031446429C2
:1040D000A8BF642121EAE1713971A0E1B979052015
:1040E000314481F30801B97199E1DB6E1A78022A33
:1040F00022D1304604930FF0E1FE45490FF0E6FF70
:10410000049B596A05930FF025FE0021049010F0DE
:10411000C7F8059B48B9049A3E49104610F0DEF8EE
:10412000049A059B10B13B4A00E000225A620F201E
:1041300011460AF012FD0AE099780F203144C8298F
:10414000A8BFC82121EAE17199700AF01BFDB8F1FE
:104150000F0F00F0CE81284BD3F86C8098F8003018
:10416000022B1AD130460FF0A9FE29490FF0AEFFFD
:10417000D8F820100FF0EEFD0021064610F090F860
:1041800030B93046234910F0A9F810B1214E00E0B3
:104190000026C8F82060122064E198F8011012206F
:1041A0003144C829A8BFC82121EAE17188F801106B
:1041B00035E1DB6E1A78022A37D1304604930FF0CE
:1041C0007DFE14490FF082FF049B196B05930FF0DD
:1041D000C1FD0021049010F063F8059BF0B9049A2A
:1041E0000C49104610F07AF8049A059BB8B1094AB8
:1041F00015E000BFACA40108880F00204811002082
:1042000010280020D6270020282800204C28002035
:10421000000020410000C842C00F002000221A63A5
:10422000102011460AF099FC0AE0197B1020314455
:10423000C829A8BFC82121EAE17119730AF0A2FCBC
:10424000B8F1100F00F05581B24BD3F86C8098F89C
:104250000030022B1AD130460FF030FEAE490FF07D
:1042600035FFD8F82C100FF075FD0021064610F030
:1042700017F830B93046A84910F030F810B1A64E02
:1042800000E00026C8F82C601320EBE098F80B1033
:1042900013203144C829A8BFC82121EAE17188F858
:1042A0000B10BCE0DB6E1A78022A22D13046049350
:1042B0000FF004FE99490FF009FF049BD96B059399
:1042C0000FF048FD002104900FF0EAFF059B48B96C
:1042D000049A9149104610F001F8049A059B10B118
:1042E0008D4A00E00022DA63112011460AF035FC05
:1042F0000AE0997D11203144C829A8BFC82121EACC
:10430000E17199750AF03EFCB8F1110F00F0F180EF
:10431000804BD3F86C8098F80030022B1AD13046CD
:104320000FF0CCFD7D490FF0D1FED8F838100FF01A
:1043300011FD002106460FF0B3FF30B93046764933
:104340000FF0CCFF10B1744E00E00026C8F83860C2
:10435000142087E098F8151014203144C829A8BF0C
:10436000C82121EAE17188F8151058E0D3F86C8073
:1043700098F80030022B1AD130460FF09FFD6849A3
:104380000FF0A4FED8F828100FF0E4FC0021064638
:104390000FF086FF30B930465F490FF09FFF10B134
:1043A0005D4E00E00026C8F8286009205AE098F821
:1043B000031009203144C829A8BFC82121EAE171AE
:1043C00088F803102BE0D3F86C8098F80030022BAB
:1043D0001AD130460FF072FD4F490FF077FED8F832
:1043E00034100FF0B7FC002106460FF059FF30B92A
:1043F000304649490FF072FF10B1474E00E00026E9
:10440000C8F834600A202DE098F80D100A203144D5
:10441000C829A8BFC82121EAE17188F80D100AF067
:10442000B1FB66E0D3F86C8098F80030022B1DD108
:1044300030460FF043FD39490FF048FED8F84010E0
:104440000FF088FC002106460FF02AFF30B93046F5
:1044500031490FF043FF10B12F4E00E00026C8F89D
:1044600040600B2031460AF078FB42E098F81710C4
:104470000B203144C829A8BFC82121EAE17188F87E
:104480001710CCE7012934D19878264B33F9123034
:10449000B3F5617F05DB40F633029342A8BF1346B4
:1044A00001E04FF46173B8F10C0F22D14FF4966222
:1044B00092FBF0F0A3F5617393FBF0F31A4ADEB2BE
:1044C0001378B34215D0042E34BF33460223137041
:1044D000019A08FB0323154A03F2A27313600DF03F
:1044E0007BF9404631460AF04DFB701CC0B20AF021
:1044F000D9FB94F86420012303FA0BF3134384F8E7
:1045000064300BF1010BBBF1040F09F10C097FF4CE
:104510002FADD2E4880F00200000C84200007A448A
:104520000000204128280020F82000204811002009
:10453000DAF80030DB050FD56B796BB13B68980773
:104540000AD5AC4B1B8813F001050AD10FF074FAA1
:10455000012003F073FF04E0012003F05EFF01235C
:1045600000E00023326851070DD563B1012003F04C
:1045700054FFA04B1B889A0708D40FF05DFA022065
:1045800003F05CFF02E0022003F047FF3B6813F0FA
:104590000A0F26D03368DB060BD5964B1B885D07C8
:1045A0000AD4042003F04AFF934B1B88A4F8703010
:1045B00002E0042003F031FF3368980607D58D4BE5
:1045C0001B88590606D4402003F038FF02E0402043
:1045D00003F023FF33685A0642BF874B1B88A4F8B9
:1045E00072303B689B0608D433681F0540F18E800B
:1045F0004FF4807003F022FF8CE0804B7D4F1B78DE
:1046000013F0020F4DD07E4B1B78042B49D9336831
:1046100013F400780ED03B88DD0636D4102003F06A
:104620000DFF202003F0F9FE7648011D07F05AF82F
:10463000022326E03D8805F01005ADB22DB1102013
:1046400003F0EBFE012584F874803368580511D51A
:10465000A36F6D495A89B1F90030002BB8BF5B4296
:10466000934207DAB1F90230002BB8BF5B429342A4
:10467000C0F20C813B88990608D5202003F0CDFEBE
:10468000002384F87430012500E0002594F87C3084
:10469000B3B90E200AF0E4FA5C4B012283F87C20C7
:1046A0000EE03B8803F03003002B9DD0102003F078
:1046B000B4FE202003F0B1FE002384F8743001E042
:1046C000002D91D000200546514B002423F81540C1
:1046D000504B1A1D03F10A0122F8154000224250E6
:1046E00001444C608A6023F8154003F132015A33CB
:1046F0004250C250014403444C608A605C609A603E
:104700001430002D7FF470AF0125DDE74FF4807089
:1047100003F083FE404B5A791C46082A01D00E2A2A
:1047200002D1402003F079FEDAF800305A0540F15A
:10473000C28094F8083223B9384B1B7813F0040F69
:1047400002E0336813F4002F0BD0354B00221A70AF
:104750003C200DF069FE002800F0AD800CF062F8FE
:10476000F6E704F0A5FF09B0BDE8F04F0DF025BD58
:104770000120FFF78CB90320FFF789B9012000E081
:1047800002205FFA80F9019A09F1FF3382F8A0371D
:1047900003F096FE03F036FF48460AF083FAFFF76F
:1047A0002EBB029A12B17E2B3FF427AB94F829302E
:1047B000972B05D1154B4FF4C872DA85FFF71FBB55
:1047C000A72B06D10D4A137843F004031370FFF7AB
:1047D00016BB0022BB2B079201D1022303E0B72BAB
:1047E00004D14FF6FE73ADF81E3021E0BE2B19D177
:1047F00002231BE0A8120020C0110020E8110020B5
:10480000EE11002050110020C8110020880F002058
:10481000A0300020061000204C280020A6300020E8
:10482000F9230020BD2B1AD14FF6FE73ADF81C30D2
:10483000DBF80020BDF81C10B2F858300B44A2F889
:104840005830BDF81E10B2F85A300B44A2F85A3056
:1048500004F0A4F8002384F82A30FFF7D0BA792BAB
:1048600004D1164AD37823F0010306E07A2B7FF4B3
:10487000C6AA124AD37843F00103D370FFF7BFBA38
:10488000013301469BB20220FFF701B93B889B062A
:104890003FF5FCAE202003F0D1FD094B09481A6812
:1048A0005B68011D4360026006F01CFF064B01259A
:1048B00083F87450EAE609B0BDE8F08F941C00203C
:1048C000F011002058110020880F00209148F0B509
:1048D0000368914A9C8AA4B2E1B211F0010F2ED074
:1048E000198821F400610904090C1980198889B21A
:1048F00041F48061198000211170517899B191784B
:1049000011B9D178FF290ED10121917011790229B5
:1049100001BF198889B241F400611980517941F0D1
:1049200001011982E1E0517901F0FE011982D37889
:10493000FF2B00F0DA80784BFF211970D5E08E074D
:104940003AD5BFF35F8F1479E4B2012C13D15178BB
:1049500089B1917879B1198821F480610904090C31
:104960001980BFF35F8F198B1988947189B241F454
:10497000007119801BE0198BBFF35F8F14796649B2
:10498000022C0AD14C7844B1897831B1198821F4CC
:1049900080610904090C1980A1E014795E49032C97
:1049A00005D14C781CB18978002940F0988099880D
:1049B00089B241F4806197E04D0756D5012191718C
:1049C0005178002937D09178002934D011791C888A
:1049D000022911781DD924F480642404240C1C803D
:1049E0001E8A9568CCB2F6B249B26E54198889B263
:1049F00041F4007119800168A31C13700B8A013403
:104A0000DBB264B22B558B889BB243F480638B80FE
:104A100026E0A4B244F400741C801D8A9668CCB2CF
:104A2000EDB249B275541B8A611C49B2DBB2033442
:104A30007354147014E09178374C09B9217B41B15B
:104A4000198889B241F40071198013780133137009
:104A500006E0198889B241F4807119800123A3709E
:104A600001680B88DB05FCD43FE001F0400101F058
:104A7000FF05E1B114781F8A9668E5B2691C64B23B
:104A8000FFB23755C9B21679117049B2CC1CA64293
:104A900001BF9C8824F480642404240C08BF9C80FB
:104AA00013798B4221D11C4B02351D701DE0270666
:104AB0001BD511784CB2661C0AD0156901312C5DEA
:104AC000C9B21C821479117049B28C420DD106E032
:104AD000D17815701982517809B9117929B9998855
:104AE00021F480610904090C9980137992F900403E
:104AF00001339C4208490CD100238B708B7933B170
:104B000001688B8823F440731B041B0C8B800023EB
:104B10001375F0BDF020002088100020074B98424C
:104B200001D1074A03E0074B984204D1064A138893
:104B300001339BB213804FF0FF30704700300140CB
:104B4000F202002000380040C80600206B4B6C4A7F
:104B50002DE9F04F5E8994694FEA062AB4EB0A0A00
:104B60009C884FF000054FEA04481C894FF0000B69
:104B7000A4FB0A6765EB0B0B04FB0B77F40944EA13
:104B8000476418EB04065C884FF000094FEAE7150C
:104B90004FEAC438DC8849EB050787B0CDE90467E4
:104BA000A4FB0A6704FB0B77340A44EA076418EB9A
:104BB00004064FEA27259C894FF0000949EB0507B9
:104BC000CDE90067AAFB046704FB0B77F40D44EA08
:104BD000472414F5FA664FEAE75545F10007B6F5A4
:104BE000FA6F77F10003CDE90267964666DADDE9F0
:104BF0000489A4FB046704FB05F34FF0050C07EBE5
:104C00004307A6FB0C230CFB07335F104FEA320669
:104C1000B8EB06084FEA920646EA837669EB070985
:104C20009F10DDE90023921B63EB0703CDE900230E
:104C3000DDE90267334A4FF0FF33964277EB030317
:104C4000CDE9048927DA40F6AC520023A4185D416F
:104C500004FB05F3A4FB04456FF0060205EB4305D6
:104C6000664202FB0566A4FB0223334418EB0206EE
:104C700049EB0307CDE904670B26A4FB062306FBDB
:104C80000533DDE900455B104FEA3202A41A65EBFB
:104C90000305CDE90045DDE902450AFB0BF3AAFB5C
:104CA0000AAB0BEB430B4FEADA7242EA4B02A41A4F
:104CB0004FEAEB7365EB0305CDE90245DEF81C40D6
:104CC000009B019DA4FB032304FB05334FEA5258CC
:104CD00048EAC3284FEA6359DDE90423B8EB02022E
:104CE00069EB03039946D30B43EA494300B10360E0
:104CF00009B1029B0B6007B0BDE8F08FF6020020FF
:104D00008810002024FAFFFF2DE9F04FDFF85892B9
:104D100085B00746D9F820000E460FF0CFF88E4C2C
:104D2000804620880FF0C6F84FF05C51054640469B
:104D30000FF018F94FF06451824628460FF012F92F
:104D4000014650460FF004F84FF06251824640464B
:104D50000FF008F94FF06A51804628460FF002F92B
:104D6000014640460EF0F4FF0546B4F902000FF08C
:104D7000A5F8014628460FF0F5F85146054650467D
:104D80000FF0F0F88046B4F904000FF097F80146F0
:104D900040460FF0E7F8014628460EF0DBFF80465C
:104DA0000FF0A6FA6D490546A06140460FF08EF956
:104DB000D9F824308046284601930FF07FF84FF051
:104DC0007C510FF0CFF866490EF0C2FF0546E3892B
:104DD000B4F90A0002930FF071F829460FF0C2F8F7
:104DE00029460FF0BFF84FF058510FF0BBF881463D
:104DF000B4F90800B4F810B0B4F80CA00FF05EF8E5
:104E000029460FF0AFF8014648460EF0A3FF4FF0D9
:104E100058510FF0A7F84FF060510FF0A3F84FF082
:104E20007E510EF097FF8146E0880FF043F801466F
:104E300048460FF097F8002181460FF027FA002826
:104E40007BD1294628460FF08DF803900FFA8BF09E
:104E50000FF034F8039B014618460FF083F84FF02B
:104E600060510FF07FF88346BDF908000FF026F877
:104E7000014628460FF076F801460EF06BFF01461A
:104E800058460EF067FF4FF07A510FF06BF88346EB
:104E900001980FF013F801464FF093400EF058FFC1
:104EA00005460FFA8AF00FF009F84FF08F410FF026
:104EB00059F8014658460EF04DFF4FF066510FF07D
:104EC00051F8014628460EF043FF26490FF04AF8F4
:104ED00049460FF0FBF80546B4F916000EF0EEFF58
:104EE00029460FF03FF829460FF03CF84FF04051AB
:104EF0000FF038F88146B4F914000EF0DFFF0146D8
:104F000028460FF02FF84FF060510FF02BF80146B4
:104F100048460EF01FFF8146B4F912000EF0CEFF96
:104F2000014648460EF016FF4FF076510FF01AF882
:104F3000014628460EF00EFF00E0002017B10FF0EA
:104F4000D7F938602EB140460FF0D2F964235843A8
:104F5000306005B0BDE8F08F300300200000A045B0
:104F600000007A470050C345881000207047704702
:104F70002DE9F041324C334D62892B8DB4F9048018
:104F80009A1A2389B4F902E05A43B4F91230D613BD
:104F9000B4F91420DB02324493FBF2F232440A26C5
:104FA000E2615643A2F57A6202FB02F3B4F90EC045
:104FB00002FB0EFE02FB08F2B4F90C801B130CFB83
:104FC00003FC03FB08F31B1403EB62320232E38899
:104FD000921002F5004253434CF25032B4F9207063
:104FE0004FEAEE2EB4F900400EEBEC2C0CEB8404EF
:104FF000BC40ED6A0234A5EBA4043A4162434FEA97
:10500000D3384EBFB2FBF8F35400B4FBF8F340F6CC
:10501000DE3448BF5B001A12524362430A4C083622
:105020005C43241404EB224202F6CF62361103EBF8
:10503000221300B1036001B10E60BDE8F08100BF32
:10504000080300208810002043E3FFFF024B4FF4C9
:1050500080521A80704700BF1C000020704710B5B6
:10506000224C2368998A89B211F4706F1EBF204ABE
:10507000012082F8300011F4E06F2BD01A8B9A884F
:10508000890522F480624FEA02424FEA12429A8076
:1050900020D41A8892051DD41A88D0050FD51A88F5
:1050A000D105FCD41A8892B242F400721A801A8890
:1050B0009205FCD40F4B18780BF0B4F90AE01A886B
:1050C00092B242F400721A809A8822F4407212045A
:1050D000120C9A802268938A23F470631B041B0CC1
:1050E0009382034B00221A7510BD00BFF0200020F0
:1050F00088100020F4200020054A08B513880133E9
:105100009BB21380034B18780BF08CF9002008BD7C
:10511000E6100020F420002010B51E4C4000C0B264
:10512000A36023611C4B6071E17001200021217399
:10513000607022712075186884F8301040B383883D
:105140009B0515D40388D9050DD447F23053028846
:10515000920502D5013BFAD112E08BB103889BB2D4
:1051600043F48073038083889BB243F4407383804D
:1051700047F23053227D12B1013BFBD100E013B95D
:10518000BDE81040B8E7034B93F8300080F0010011
:1051900010BD00BF88100020F020002007B50021BE
:1051A00001AB03227720FFF7B7FF9DF805309DF88C
:1051B00004001B0243EA00439DF80600184303B0B5
:1051C0005DF804FB08B5FFF7E9FF014BD86108BDA6
:1051D0008810002008B5FFF7E1FF014B986108BD7A
:1051E0008810002007B5F7216B4606227620FFF7CE
:1051F00093FF9DF800309DF801101B0343EA011353
:105200009DF80210094A43EA111353629DF80330D6
:105210009DF804101B0343EA01139DF8051043EAAF
:105220001113136203B05DF804FB00BF8810002067
:1052300007B5F62101AB03227720FFF76DFF9DF83C
:1052400005309DF804201B0243EA02439DF8062026
:105250001343054AB2F92020C2F10802D340034AA1
:10526000D36203B05DF804FB08030020881000201F
:1052700007B5F62101AB02227720FFF74DFF9DF81D
:1052800004209DF8053043EA0223024A138503B047
:105290005DF804FB8810002013B5204B400002ACE1
:1052A000C0B2587104F8012DD970012200211A737F
:1052B00059701A711A751A4A1C6110689C6083F83B
:1052C000301040B38288920515D40288D4050DD4DD
:1052D00047F230520188890502D5013AFAD112E02D
:1052E0008AB1028892B242F480720280828892B2BD
:1052F00042F44072828047F23052197D11B1013A76
:10530000FBD100E012B9FFF7F7FE04E0034B93F87E
:10531000300080F0010002B010BD00BF88100020F6
:10532000F0200020772048210122B5E7772058217E
:105330000122B1E77620F4213122ADE7044B77203A
:1053400093F82020F4219201343202F0FC02A3E70A
:10535000080300207720F4212E229DE7FFF7B6BA3C
:105360007DE6FFF7B3BA7AE670B584894FF47A74B4
:10537000FBB112B11578013207E0FF2505E04FF6C9
:10538000FF76013CA4B2B4420DD00689B607F6D52B
:10539000ADB285810589ED070DD44FF6FF75013C4F
:1053A000A4B2AC42F6D1FFF7B9FB003018BF012020
:1053B00070BD012070BD8589ADB209B10D7001319C
:1053C000013BD5E708B540F2E9330289920704D4DE
:1053D000013B9BB2002BF8D10AE040F2E93389B2DD
:1053E00081810289D20706D4013B9BB2002BF8D100
:1053F000FFF794FB00E08089C0B208BD2DE9F041C1
:1054000017468846084C094E102540F0800165611A
:105410003046FFF7D7FF3046414600223B46FFF7B4
:10542000A3FF2561BDE8F081000801400030014084
:1054300013B5012204460DF107013A20FFF7DEFF04
:105440009DF8073003B10123237002B010BD184A44
:1054500013B51388044623F040031B041B0C138070
:1054600013883B2023F038031B041B0C1380138884
:1054700069469BB243F0400313800622FFF7BEFF4C
:105480009DF800209DF8013043EA022323809DF817
:1054900002209DF8033043EA022363809DF8042034
:1054A0009DF8053043EA0223A38002B010BD00BF7F
:1054B00000300140174A13B51388044623F0400317
:1054C0001B041B0C13801388432023F038031B0498
:1054D0001B0C1380138869469BB243F04003138072
:1054E0000622FFF78BFF9DF800209DF8013043EA6C
:1054F000022323809DF802209DF8033043EA022313
:1055000063809DF804209DF8053043EA0223A380C0
:1055100002B010BD00300140F8B503460F46074CFD
:10552000074E1025194665613046FFF74BFF3046A0
:105530003946FFF747FF2561F8BD00BF000801406D
:1055400000300140284A08B51388802123F0400329
:105550001B041B0C138013886B2023F038031B04DF
:105560001B0C43F03003138013889BB243F04003BD
:105570001380FFF7D1FF962009F03DFB032168203F
:10558000FFF7CAFF962009F036FB03216B20FFF7D7
:10559000C3FF012009F024FB10216A20FFF7BCFFA4
:1055A000012009F01DFB00216C20FFF7B5FF012051
:1055B00009F016FB00211920FFF7AEFF012009F0CA
:1055C0000FFB10211C20FFF7A7FF012009F008FBAB
:1055D0001B201821FFF7A0FF012009F001FB034B5E
:1055E00001221A7008BD00BF00300140F002002007
:1055F0001F4A13B513886B2023F040031B041B0CB8
:1056000013801388802123F038031B041B0C43F004
:1056100030031380138806249BB243F040031380A9
:10562000FFF77AFF962009F0E6FA75200DF10701E1
:105630000122FFF7E3FE9DF80730682B04D0013C00
:1056400014F0FF04EED10EE00C200DF10701012251
:10565000FFF7D4FE9DF80730142B04D3182B04D980
:10566000543B062B01D9002000E0012002B010BD00
:10567000003001402DE9F0474B28A0B0044600F06F
:10568000488600F2B480302800F0D48651D8222811
:1056900000F0958423D8032800F0608114D80128F5
:1056A00000F05081022840F0308704200BF026F9EA
:1056B00043200BF0F4F84C200BF0F1F846200BF0EF
:1056C000EEF84C2000F05ABE042800F05181052865
:1056D00040F01B871A200BF011F9002459E128280B
:1056E00000F0E58515D8242800F0CC85262840F068
:1056F0000C87B44C06200BF001F9B4F85C010BF0F8
:1057000000F9B4F85E010BF0FCF8B4F8600100F0A9
:10571000B6BD2C2800F0DE852E2800F05A862A28F7
:1057200040F0F38601200BF0E9F8A64B587900F021
:1057300025BE3D2800F0F0821ED8362800F02F86C6
:105740000BD8322800F01486342840F0DE8648203A
:105750000BF0D4F8002500F054BC3A2800F0B082D9
:105760003B2800F02584382840F0CF8604200BF039
:10577000C5F8944C00F08CBD452800F0B38627D8BE
:10578000402800F0FE85422840F0BF868D4C102056
:105790000BF0B4F860790BF082F8A0680BF0BAF85F
:1057A00094F890010BF07BF8B4F85C010BF0A9F8C9
:1057B000B4F85E010BF0A5F8B4F860010BF0A1F8A5
:1057C000B4F880010BF09DF8B4F8820100F057BDE9
:1057D000472800F06586C0F05286492840F095863B
:1057E00002200BF08BF8774B988900F048BD7028A9
:1057F00000F0E88258D8692800F042822AD865284B
:1058000000F0FA8015D84D2800F09285642840F009
:105810007C8607200BF072F8E7200BF040F8694B0C
:1058200058790BF03CF800200BF039F8042000F018
:1058300068BE672800F0A78100F2158212200BF0E5
:105840005DF8614B00241B88B3F5806F8CBF082581
:1058500001257AE16C2800F0268217D86A2800F02A
:1058600095846B2840F0518605200BF047F8574B84
:1058700018880BF046F8564B18880BF042F8554B39
:1058800093F86A0000F0010000F078BD6E28514DD9
:1058900000F01D8200F26E8206200BF02FF8A86D3A
:1058A0000BF038F84C4B09E2782800F0798119D8D0
:1058B000742800F0C7830BD8722800F0278473285F
:1058C00040F0238608200BF019F8012400F057BCA3
:1058D000762800F07B8400F2F9832F200BF00EF87D
:1058E0003E4C5DE3A42800F0968414D87B2800F099
:1058F000FD82A02840F009860C200AF0FFFF384BFB
:1059000018680BF007F8374B18680BF003F8364BA4
:10591000186800F0F6BDF12800F07E81FE2800F046
:10592000A184F02840F0F1852A4C04200AF0E6FF1B
:10593000E36BB3F85A000AF0E4FFE36BB3F85800E6
:1059400000F09DBC03200AF0D9FF00200AF0A7FF59
:1059500020460AF0A4FF0C2000F010BD0AF0CEFF94
:1059600001200AF09CFF0A200AF099FF00F051BCC8
:1059700006200AF0C3FF43200AF091FF43200AF0FB
:105980008EFF33200AF08BFF44200AF088FF00F0DE
:1059900075BC164B185D01340AF081FF0B2CF8D151
:1059A0000024134B185D01340AF079FF082CF8D15C
:1059B0000024104B185D01340AF071FF072CF8D158
:1059C00000F0A1BD4C2800201C0000206212002025
:1059D00064120020E4100020B8110020E7A40108A0
:1059E000E8F7FF1FECF7FF1FF0F7FF1F88C401085F
:1059F00094C4010869C40108CD4C0B200AF07EFF55
:105A000020880AF07EFF608880B20AF07AFFC94BD6
:105A10001B68C3F3C000C3F38002800040EA420069
:105A2000C3F340021043C3F3401240EAC20003F044
:105A3000100318430AF065FFBF4B1A88636812F021
:105A4000010F14BF4FF0020C4FF0000C12F0020FC8
:105A500002F0080814BF4FF0040E4FF0000E03F4DC
:105A6000475912F0040F14BF1027002749EA08090C
:105A700012F0400F03F4804814BF2026002649EAA4
:105A8000080912F0100F03F4004814BF4FF400751A
:105A9000002549EA080912F0200F03F4803814BFEA
:105AA0004FF48060002049EA080912F4807F03F473
:105AB000003814BF4FF40061002149EA080912F4CC
:105AC000007F03F480289D4A49EA080903F400286E
:105AD00049EA0809127803F4801849EA080903F032
:105AE000007349EA0303C2F3800243EA020343EA74
:105AF0000C0343EA0E0E4EEA070746EA070645EA9C
:105B0000060540EA050041EA00014FF000000346A7
:105B100014BF4FF400184FF0000841EA0808217A3A
:105B20008B420BD2864A9C5C012202FA04F414EAEE
:105B3000080F1CBF9A4010430133F1E70AF0EAFE58
:105B4000804B93F8A00700F019BC7F4B33F9140089
:105B5000013490FBF5F080B20AF0D3FE032CF4D1AF
:105B6000734CA08C0AF0CDFEE08C0AF0CAFE208DAA
:105B7000764C0AF0C6FE20880AF0C3FE60880AF060
:105B8000C0FEA0887BE310200AF0B8FE0024704B12
:105B9000185D01340AF083FE102CF8D100F0B3BC7C
:105BA00070200AF0ABFE00260E247443604D0136CF
:105BB000EB6B2344B3F819010AF0A3FEEB6B23440B
:105BC000B3F81B010AF09DFEEB6B2344B3F81D01F3
:105BD0000AF097FEEB6B234493F81F010AF05FFE77
:105BE000EB6B234493F820010AF059FEEB6B23443E
:105BF00093F821010AF053FEEB6B234493F8220142
:105C00000AF04DFEEB6B1C44D4F823010AF082FE2F
:105C1000082EC9D100F077BC70200AF06FFE494C05
:105C200004F1700594F8D4000AF039FE94F8D50018
:105C30000AF035FE94F8D6000AF031FE94F8D70049
:105C40000AF02DFE94F8D8000AF029FE94F8D90045
:105C50000AF025FE073494F8D3000AF020FEAC4287
:105C6000E0D100F050BC10200AF048FE0024394B6F
:105C7000185D01340AF013FE102CF8D100F043BC7B
:105C8000354D00242878400000F0FE000AF036FE72
:105C90002B789C4280F03784304B33F814000AF0A4
:105CA00030FE0134F4E72E4C06200AF027FE20884F
:105CB0000AF027FE60880AF024FE2A4B1888DEE2EC
:105CC00004200AF01BFE1A4BD86D00F01ABC072006
:105CD0000AF014FE244B1888FF28A8BFFF20C0B28A
:105CE0000AF0DDFD214B186880F3100080B20AF045
:105CF00008FEB5F860000AF004FE124B93F8852107
:105D00001B4B186822B10A23584380F3100001E0AE
:105D100000F30F0080B2B2E20A4C02200AF0EEFD5E
:105D200094F8D4010AF0BBFD94F8D30126E300BF38
:105D3000E4100020E4110020A8120020A63000206A
:105D4000ED1000204C280020B2110020E02300209C
:105D50000E11002024110020D42700202828002024
:105D6000E2270020C0110020D4110020E011002003
:105D7000DC1100200B200AF0C1FD6B6E00261878A4
:105D80000AF08DFD6B6E58780AF089FD6B6EBE4C83
:105D90003344187901360AF082FD032EF6D1636E82
:105DA000D8790AF07CFD636E98780AF078FD636E0E
:105DB000D8780AF074FD636E58890AF0A2FD636E0C
:105DC000187ADBE2B04C1E200AF098FDE36B002548
:105DD0001B78022B77D1E36B05F1080253F8220000
:105DE000AA490EF0BFF812F03FF8FA28A8BFFA202F
:105DF00020EAE070C0B20AF052FDE36BA44903EB65
:105E00008503D86A0EF0AEF812F02EF8FA28A8BF73
:105E1000FA2020EAE070C0B20AF041FDE36B05F120
:105E20000E0253F822009B490EF09CF812F01CF869
:105E30006428A8BF642020EAE070C0B201350AF0EF
:105E40002EFD032DC7D1072DE36B2AD1586C8F4946
:105E50000EF088F812F008F8FA28A8BFFA2020EA15
:105E6000E070C0B20AF01BFDE36B8849986C0EF03D
:105E700079F811F0F9FFFA28A8BFFA2020EAE070BB
:105E8000C0B20AF00CFDE36B93F84C000EF012F870
:105E900011F0EAFFFA28A8BFFA2020EAE070C0B2A9
:105EA0000BE02B4458780AF0FAFCE36B2B44D87AC9
:105EB0000AF0F5FCE36B2B44587D01350AF0EFFC4A
:105EC0000A2DC0D11FE3E36B2B4458780AF0E7FC9E
:105ED000E36B2B44D87A0AF0E2FCE36B2B44587D49
:105EE00001350AF0DCFC0A2DEDD10CE33C200AF070
:105EF00005FD0024644D04F10802EB6B654953F87D
:105F000022000EF02FF811F0AFFF80B20AF0F9FC7A
:105F1000EB6B604903EB8403D86A0EF023F811F0B1
:105F2000A3FF80B20AF0EDFCEB6B04F10E0253F814
:105F3000220058490EF016F811F096FF013480B295
:105F40000AF0DFFC032CD5D1072CEB6B16D1586C73
:105F500050490EF007F811F087FF80B20AF0D1FC2B
:105F6000EB6B4C49986C0DF0FDFF11F07DFF80B29A
:105F70000AF0C7FCEB6B93F84C000BE02344587815
:105F80000AF0BFFCEB6B2344D87A0AF0BAFCEB6B47
:105F90002344587D01340AF0B4FC0A2CD4D1B2E277
:105FA00014F8010F002800F0AE820AF078FCF7E741
:105FB00001200AF0A3FC344BDB6B1878DEE15020A3
:105FC0000AF09CFC0025304B0C21DC6B324B04EBBF
:105FD000850494F87920013501FB023393F83800E9
:105FE0000AF05DFC94F87A000AF059FC94F87B0002
:105FF0000AF055FC94F87C000AF051FC142DE2D113
:1060000081E2214BDC6B062303FB054494F8CE00B0
:106010000AF045FC94F8C9000AF041FC94F8CA0063
:106020000AF03DFC94F8CB000AF039FC94F8CC005F
:106030000AF035FC013594F8CD000AF030FC0C2D47
:10604000DFD160E24FF00008012600270E4B1A7ADC
:10605000974232DA0933FA5C00240C2363430E4D75
:1060600005F13001595C914207D12B44586B11F076
:1060700032FD82462EB9B14610E001341B2CECD122
:1060800019E0804417E000BFE41000200000204128
:106090000000C84200007A44E8A40108D1450ADAA9
:1060A0000C2303FB04535B6B13F809000AF0F7FBA6
:1060B00009F10109F2E70137C8E7002E00F0238259
:1060C0005FFA88F00AF01AFC0026BEE7CC4D0024E7
:1060D000287A0AF013FC2B7A9C4280F01482C94B78
:1060E0000021E65C0C2202FB01F3C74800F13007F7
:1060F000DA5DB24205D1034493F838000AF0CFFBD1
:1061000002E001311B29EDD10134E4E7BF4C162038
:106110000AF0F4FBB4F896010AF0F3FBB4F844017A
:106120000AF0EFFBB4F846010AF0EBFBB4F84801C3
:106130000AF0E7FBB4F8D0010AF0E3FB94F8E101C0
:106140000AF0ADFB00200AF0AAFB94F8E2010AF085
:10615000A6FB94F885010AF0A2FB94F892010AF0DC
:106160009EFB00200AF09BFBA54B0A20DB6BB3F9DA
:10617000563093FBF0F080B20AF0C3FB88E0E0B247
:1061800001340AF08CFB092CF9D1BCE110200AF093
:10619000B5FB9F4B9F4C187800F002000AF07FFB84
:1061A0009D4B18780AF07BFB20680AF0B3FB60680F
:1061B0000AF0B0FB994B18880AF0A3FB984B18889B
:1061C0000AF09FFB8E4BB3F8680058E00AF04AFBD8
:1061D000074612200AF092FB894C17B9E66E256F2C
:1061E00005E0102F19BF00252E46666FA56F3846B3
:1061F0000AF055FB30460AF08DFB28460AF08AFB70
:10620000E06F0AF087FB00200AF07BFB00200AF019
:1062100078FB0020B2E07A4D002495F880002E46ED
:1062200080000130C0B20AF069FB95F880000AF0E6
:1062300036FB96F880309C4280F06581794D285D70
:106240000AF02DFB05F11003185D0AF028FB05F19B
:106250002003185D30350AF022FB285D0AF01FFB91
:106260000134E6E708200AF049FB00200AF049FB68
:1062700000200AF046FB00200AF043FB00200AF051
:1062800040FB40E104200AF039FB604B986838E19C
:1062900094F87A010AF003FB94F87E010AF0FFFA01
:1062A00094F87D010AF0FBFA94F87F0166E0574C00
:1062B00007200AF023FBB4F880010AF022FBB4F8AF
:1062C00082010AF01EFB94F884010AF0E8FAB4F89F
:1062D0008601D4E74D4C0C200AF010FB94F8900195
:1062E0000AF0DDFAB4F89A010AF00BFBB4F8960153
:1062F0000AF007FBB4F898010AF003FB94F8910147
:106300000AF0CDFAB4F89C010AF0FBFAB4F89E0149
:10631000B5E73E4C04200AF0F1FA94F8CE010AF0F9
:10632000BEFA94F8CF010AF0BAFAB4F8D001A6E7A1
:106330003D4C3E4D20780426043800EB4000C0B2AE
:106340000AF0DCFA237802359E4280F0DC8015F8F2
:10635000020C0AF0A4FA15F8010C013600EB8000DB
:1063600000EB800000F2EE2080B20AF0CAFAE9E702
:1063700001200AF0C3FA254B93F892010AF08FFA34
:10638000C1E008200AF0BAFA0024204B234493F815
:10639000880101340AF083FA082CF6D1B3E0184BD7
:1063A0001A4C93F8C10004F12005C0EBC000C0B244
:1063B0000AF0A4FA94F8E80100231D4AD25C904246
:1063C00000F0A5800C33302BF7D10834AC42F1D16A
:1063D00099E040200AF092FA0C4C04F14005B4F820
:1063E00098020AF08EFA94F89A020AF058FA0434E5
:1063F00094F897020AF053FAAC42F0D183E000BF60
:10640000E4100020ED100020E8A401084C28002032
:10641000E8110020F0110020EE110020EC11002006
:10642000EA11002065110020D4270020EC2900206B
:1064300000240020E0200AF061FA424C04F18005BB
:10644000B4F81A02043400F03F000AF05AFAB4F823
:106450001602C0F386100AF054FA94F814020009E8
:106460000AF01DFA94F8140200F00F000AF017FA6F
:1064700094F815020AF013FAAC42E1D143E0324C31
:106480000D200AF03BFA09F0ADFE0AF008FA208868
:106490000AF040FAE0680AF03DFA05F061FA30E0EF
:1064A0000AF0F4F9054684200AF028FA28460AF092
:1064B00031FA254BDC6805F18003A3428CBF641BD5
:1064C000802405F00DFB28462246694609F0C2FEED
:1064D00005460024AC4216DA1DF804000AF0DFF984
:1064E0000134F7E713200AF009FA0024174B185D6E
:1064F00001340AF0D4F90B2CF8D100200AF00AFA82
:1065000000200AF007FA012018E0002016E00AF047
:10651000C6F9B4F8EA010AF0F4F994F8EC010AF0CB
:10652000BEF994F8ED010AF0BAF994F8EF010AF017
:10653000B6F994F8EE010AF0B2F946E720B0BDE8EA
:10654000F08700BF4C2800200C00002088C4010800
:106550002DE9F347C54C06462378C54F002B00F0C4
:10656000D9813A686368D31A7C2B40F2D381237AAD
:106570006260013323724FF0000808F12400BB4D24
:10658000C0B203F049F805F10A0333F918000DF021
:1065900095FCB84B814618880DF090FC01464846A2
:1065A0000DF094FDB4490DF0DDFC0DF0A1FE08F1F5
:1065B000010800B203F01EF8B8F1030FDDD130205E
:1065C00003F02AF8B5F9100003F014F803F01CF8F2
:1065D0002B7A9A072CD141F288336A689A4218D9EB
:1065E000102003F019F868694FF0640890FBF8F088
:1065F00000B202F0FFFF212003F00EF8686990FB63
:10660000F8F308FB13000028B8BF404200B202F0C4
:10661000F1FF142003F000F8B4F9180002F0EAFFCB
:106620001C2002F0F9FF002002F0E4FF02F0ECFF72
:10663000237ADFF838825B0740F04981022002F0BC
:10664000EBFFD8F81C006423323090FBF3F000B26B
:1066500002F0D0FFB8F926504FF0050A95FBFAF585
:10666000032002F0D9FF854BADB21B78DFF82092F2
:1066700013F0040F0BD030460CF063FE28B9D9F8A4
:10668000003013F0100F18BF002528B205E0D8F82D
:1066900028309889B0FBFAF000B202F0ABFFD9F8CD
:1066A00000309E0765D5DFF8EC91A28D99F8003097
:1066B0004FF0640808FB02325B00B2FBF3F3E68D97
:1066C00006203601B6B246EA0326B6B2C3F3032368
:1066D0001E4302F0A1FF30B202F08CFFE38D99F867
:1066E000001001339BB293FBF1F201FB1233E385FF
:1066F000236B5E4D9B7B012B05D1392002F08CFF73
:10670000B5F92C0019E0AD8D6E235D43152695FB80
:10671000F6F53A20AEB202F07FFFB6FBF8F528B2EC
:1067200008FB156502F066FF3B2002F075FFA8B27A
:10673000451D0A2095FBF0F000B202F05BFF282017
:1067400002F06AFF636B0A2093FBF0F000B202F0E4
:1067500051FF042002F060FFA36A9B8913B107F088
:10676000CDF803E0414B986B80F3100000B202F0CB
:1067700041FFE36B3D4E9D0640F19F8096F840300F
:1067800098071DD5112002F047FFB6F842004FF4DC
:10679000F36568433A4B90FBF3F000B202F02AFF36
:1067A000192002F039FFB6F842004543642095FBFA
:1067B000F0F595FBF0F300FB135000B202F01AFF66
:1067C00094F84030B4F8445013F0020F08BF00258D
:1067D000012002F021FF28B202F00CFF092002F094
:1067E0001BFF002002F006FF264B94F846501A8843
:1067F000B2F5967F0AD91D4B1B7A03F00F03072BC6
:1068000004D842F20F75954228BF1546052002F0C4
:1068100003FF236B5B7B0BB928B216E0A5F12000C8
:106820000DF04CFB18490DF051FC002105460DF010
:1068300037FD10B94FF07C5101E04FF03F41284641
:106840000DF088FA0DF054FD00B202F0D3FE94F87A
:106850004020064B910703D493F84720012A1BD10F
:10686000012384F8473009482DE000BFA81100201B
:10687000102800201C00002000007A44A6300020D0
:10688000A0860100FA0000206666E63FF0110020B5
:10689000EC270020F80000201D6BAF4968680DF060
:1068A00061FB0DF025FDAC490090A8680DF05AFB86
:1068B0000DF01EFD0190684605E0A84A92E803002D
:1068C0008DE80300684602F0B7FE02F09DFE237AD1
:1068D000282B1FD1A24B00221A723B684FF47A700A
:1068E000B3FBF0F83C26172002F096FEB8FBF6F555
:1068F000B5FBF6F006FB1050000200B202F07AFE83
:10690000182002F089FE06FB158000B202F072FE2C
:1069100002F07AFE94F85030914D002B00F0408147
:1069200008F044F96B6D8F4AC31A9342064640F251
:10693000C280002385F85A3085F85C30AB8DDAB21E
:106940001B0A85F8762085F8773085F86C2085F865
:106950006D30D5F884203B689A1AD5F88830D97BF9
:106960004FF47A734B439A420ED37F4B1B68C5F8A2
:10697000843095F88C30013B012B9FBF102385F8A4
:106980005A30022385F85C30626B0A20A36B92FBBD
:10699000F0F293FBF0F384F87420121284F875205F
:1069A00084F8783094F840201B1284F8793094F8F9
:1069B000463092076A4984F8A73003D42D2381F822
:1069C000A83077E0D4F848906848DFF8ACC199FB6C
:1069D000F0FA0CFB0A924FF0060E042B0EFB02F2AB
:1069E0008CBF3323322381F8A830614BE76C92FBD4
:1069F000F3F197FBF0F003FB1122642592FBF5F213
:106A00000CFB007C0EFB0CFE84F89920121284F81B
:106A10009A209EFBF3F203FB12E393FBF5F30AEBE0
:106A20008A0A4FFA81F80AEB8A0A08EB8A0189B2CE
:106A300084F8971000EB8000090A84F8981000EBA6
:106A4000800051B201EB800292B284F89C20120ABD
:106A500084F89D2084F89E30B4F842201B1284F8FC
:106A60009F302423534393FBF5F5B4F8BA300A2240
:106A700084F8A0301B0A84F8A130B4F844304FEAFF
:106A8000D979B3FBF2F303F5FA739BB284F8A23021
:106A90001B0A84F8A330B4F8BC30FF0F84F894507C
:106AA000C5F3072584F8969084F89B7084F8955078
:106AB00084F8A930666594F8BE80294DB8F1000FBE
:106AC0000DD1D5F8C40008F041F9012807D90228F2
:106AD000284F00F0388202F07FFD0123BB70D4F80C
:106AE000C8001F4D00285BD095F8BE703FB140F63E
:106AF000B732D5F8D030F31A93420BD850E00123C7
:106B0000D5F8C400022185F8BE3008F013F985F8E5
:106B1000D47043E095F8CC305BB9D5F8C4000121BE
:106B2000C5F8C83085F8BE3008F004F902F054FD0D
:106B300034E0013BDBB285F8CC3095F8D41095F801
:106B4000D520DBB94B1C013285F8D43085F8D5202F
:106B5000D5F8C40020E000BF8096184B68A6010855
:106B6000A81100203F0D03001028002080969800F7
:106B700040420F001C000020806967FF034613F8A5
:106B8000017B01327818394685F8D400D5F8C40065
:106B9000C5F8C83085F8D52008F0DBF8C4F8D06017
:106BA00094F8D6309C4DF3B1D5F8D830DBB1D5F898
:106BB000DC30C3B1C5F8E0301B68984AC5F8E43052
:106BC000D5F8E8301344187AFEF754FDD5F8E030D4
:106BD000987909F064FED5F8E8300133092B88BFB5
:106BE0000023C5F8E8308E4D94F8EC202E688A4BCF
:106BF000002A00F0E281D3F8F020002A00F0DD81C5
:106C000093F8F430013B012B00F2D781D4F8F00067
:106C1000814F08F09BF8E0B1D7F8F00008F093F846
:106C200097F8F53080467E2BD5F800900ED10223E0
:106C30001B2887F8F43009D1D7F8F00008F086F85F
:106C400020B90123C7F8F89087F8FC3084F8F58064
:106C5000DCE7D7F8F8202B689B1A41F658329342AC
:106C60001DD9032387F8F430A7E16E4A32F81300E8
:106C700010B903464FF403600133B0F5C06FDBB2C7
:106C800075D01DD9B0F5006F7AD031D9B0F5036F4A
:106C90003ED184F8FD30E36B5F4F99063FD494F802
:106CA000FC1094F8FD30002900F04A812A68921BFC
:106CB000012ADAD984F8FD30002384F8FC307CE125
:106CC000B0F5007F42D007D8B0F5807F47D0B0F54F
:106CD000887F00F08380E6E7B0F5806F00F0A68043
:106CE000B0F5826F00F0EB80B0F5047FDBD123E0DC
:106CF000B0F5E26F00F08280B0F5E46F00F08380C1
:106D0000B0F5E06FCFD184F8FD30B4F90A107EE021
:106D1000B0F5046F6BD0B0F5026FC4D1FAE097F80C
:106D200040309A07BBD5B7F8421024234B43642167
:106D3000123393FBF1F1FDE084F8FD303A4B364F0E
:106D40001B689B07ABD5BB8D0A21F2E084F8FD30B0
:106D5000354B314F1B681905A1D5796BEAE084F8F2
:106D6000FD30E36B2C4F5A0799D57969E2E084F83E
:106D7000FD302D4B284F1B681B0590D5B96BD9E012
:106D8000E16B254A8F0684F8FD3088D592F84010D3
:106D9000880784D5D90710D5D36C192283EAE3710B
:106DA000A1EBE37101EB5101B1FBF2F1002BACBFA0
:106DB00041F0004141F040410DE0936C192283EA1B
:106DC000E371A1EBE37101EB5101B1FBF2F1002B97
:106DD000B8BF41F080414FF400608AE084F8FD3094
:106DE000E36B0D4F5B077FF55AAF3969A2E084F87A
:106DF000FD30B4F91830642159437AE084F8FD304D
:106E0000B4F90C1003E0B4F90E1084F8FD302C2313
:106E100091FBF3F16DE000BFA811002068A6010806
:106E20001028002078C80108EC27002084F8FD30E5
:106E300094F8FE30624A0133DBB2032B88BF012392
:106E400082F8FE3042F2107394F8FE1059435D4B05
:106E50001B78D80748BF01319A0748BF02315F0746
:106E6000B4F8003148BF0431D80748BF0A319A0747
:106E700048BF14311F0648BF2831D80548BF283104
:106E80005A0748BF64311F0748BFC831980548BF3B
:106E900001F5C8719A0648BF01F57A71DF0648BF4F
:106EA00001F5FA61580648BF01F57A614FF4806038
:106EB00002F05EFB424B002283F8FC20EFE6E16B20
:106EC000DFF8FC8011F0200784F8FD3017D098F827
:106ED000402012F0020F14BF4FF47A71002112F01B
:106EE000010F14BF4FF4FA6300230B4494F84610CB
:106EF000194402F03DFB002384F8FC30CFE6324B0E
:106F00001B6819067FF5CBAE394602F031FB88F8D5
:106F1000FC70C4E684F8FD30E36B294F9A067FF5D8
:106F2000BEAE97F840309B077FF5B9AEB7F8443056
:106F30006421594302F01CFB002387F8FC30AEE6C5
:106F400084F8FD3039E0BB7823B1C5F8C06087F81C
:106F50000280C4E5D5F8C030F31AB3F57A6FFFF4B8
:106F6000BEAD0123D5F8C400BB7007F0ECFE0746A8
:106F7000D5F8C40007F0E7FE7F067FF4B0AD8A289D
:106F800002D08E280CD0AAE5EB6B98067FF5A7AD52
:106F900095F8BE30002B7FF4A2AD05F18D0306E01D
:106FA00095F8BE30002B7FF49AAD05F15803C5F873
:106FB000C8302D2385F8CC3091E502B0BDE8F087CC
:106FC000A8110020A6300020EC270020F8B50446C8
:106FD0000E46174600252046202110F06EFD04467F
:106FE000D0B10134204610F0CBFDB0F5617F05DB58
:106FF00040F634039842A8BF184601E04FF4617090
:10700000A0F56170192390FBF3F00DB9307000E02A
:1070100070703B7801333B700DB90125DBE72046EA
:10702000F8BD7FB504780646E4B9364B19211868D7
:1070300000EB840090F87B5090F879204D4305F5E3
:10704000617590F87A30009590F87C00414301F525
:10705000617101912C482146013401F06BF8142C28
:10706000E3D14CE010F08CFD1328054641DC254BA4
:10707000701C1C68202100238DF80F3010F01DFDBE
:107080001E35064670B10136304610F079FD1928DC
:107090009FBF04EB850358709DF80F30013398BFF4
:1070A0008DF80F303046202110F007FD064670B1F4
:1070B0000136304610F064FD0D289FBF04EB8503B8
:1070C00098709DF80F30013398BF8DF80F3004EBA6
:1070D00085043046E11C0DF10F02FFF777FF9DF8A4
:1070E0000F30042B0BD0601C0021042210F0AFFCE9
:1070F00005E0064806490022132301F01BF804B0FE
:1071000070BD00BF2011002068C901087DC90108B9
:107110009CC90108014809F075BC00BFA2C901085B
:107120002DE9F04304788FB00546002C59D17B4BF4
:107130000021142209A807AED3F8008010F087FCC4
:1071400007223046002110F082FC00231A46A700D7
:1071500005A8059308EB070583807149B5F802E09F
:1071600031F813C01CEA0E0F0AD00E310DF1380CA5
:10717000595C02F1010E624402F81C1C5FFA8EF2A7
:107180000133072BE9D100210B46664AB5F802E02E
:1071900011F802C01CEA0E0F0AD006320DF1380CAD
:1071A0008A5C03F1010E634403F8242C5FFA8EF32A
:1071B00001310629E9D118F807308DE841006A78D5
:1071C0005949029209A81A0903F00F0300F09DFF24
:1071D0002146564809AA013400F0ACFF202CA6D164
:1071E00099E010F0CDFC1F28044600F38680284665
:1071F0002021E4B210F061FC1F2C02D9FFF78AFFB6
:1072000089E0464B451C1B68002103EB84042046A3
:10721000042210F01CFC0027454B09AE304600212B
:107220000A2217F803905FFA87F810F010FC002389
:1072300015F8012B32B10A2B04D04A4502D0F25482
:107240000133F5E74A455FD108F1FF33032B09D835
:10725000DFE803F01005023F0DF1230134E00DF1EA
:1072600023011EE0304610F08BFC2378C0B243EAC5
:10727000001006E0304610F083FC237800F00F0089
:107280001843207031E00133062B0AD0244800F166
:107290001B069E5D9642F6D103445A7D63881343D4
:1072A000638011F8012F02B30023EFE70133072BAE
:1072B0000AD01B4800F10E069E5D9642F6D130F8CA
:1072C000132063881343638011F8012F6AB10023F0
:1072D000EFE7304610F054FC0F2804DC304610F085
:1072E0004FFC607001E0002363700137052F93D1DC
:1072F000012409F09DFE74B980E70E4900221F2386
:107300000D4800F017FF06E020460021042210F08F
:107310009EFB0024EDE70FB0BDE8F083AC12002027
:107320007CA6010891A60108B0C90108BFC90108DF
:107330009DA601089CC901087DC901082DE9F041FD
:10734000047807467CB9344D2146B5F8BC21B5F820
:10735000BE313248013400F0EDFE042C05F1040585
:10736000F2D1BDE8F0812E4910F07AFBB0B92A4B7A
:107370004FF47A714FF4FA62A3F8BC11A3F8BE215E
:10738000A3F8C011A3F8C221A3F8C411A3F8C62121
:10739000A3F8C811A3F8CA21BDE8F081384610F05F
:1073A000EFFB032805462ED83846202110F085FB38
:1073B000044630B10134204610F0E2FB01270646B6
:1073C00000E007462046202110F077FB10B9BDE809
:1073D000F0419FE6013010F0D3FB012FF7D140F2CE
:1073E000DC53A6F2EE229A42F1D8A0F2EE229A42A3
:1073F000EDD88642EBDA084B6E3503EB85039E80B1
:10740000D880BDE8F0810748074900220323BDE882
:10741000F04100F08FBE00BF4C280020CBC901080E
:10742000DEC901087DC90108B1D701082DE9FF4176
:1074300004780546002C34D16E4809F0E3FA6E4D0D
:10744000686900210CF022FF002840F0CF8021461F
:107450006A4800F06FFE6869694600F0F1FC014679
:10746000674800F067FEA869694600F0E9FC01463C
:10747000634800F05FFEE869694600F0E1FC014600
:107480005F4800F057FE286A694600F0D9FC0134D5
:1074900001465C4800F04EFE0C2C05F11005CFD1E2
:1074A000A4E05949052210F01FFB38B9524B0022C5
:1074B00003441030C0285A61F8D197E02846534958
:1074C000042210F011FB04462846002C3FD1202155
:1074D00010F0F3FA002800F08980451C284610F0CF
:1074E000FAFA07464A4B53F824601EB9494809F096
:1074F00089FA7BE028463146FAB210F0F5FA0134F9
:107500000028EFD13C4B0021C2181030C028516137
:107510009E46F7D1404B03EBC402D2F804C0984614
:10752000BCF1000F04D131463C4800F003FE53E0AB
:10753000002718F834309F42F5DA3B010EEB0305C3
:10754000143563440FCB013785E80F00F1E710F0E5
:1075500017FB0B28064643DC2846202110F0ADFA25
:10756000054648B10135284600F0D4FB224B0124E2
:1075700003EB0613586100E004462846202110F072
:107580009CFA054640B10135284600F0C3FB1A4B72
:10759000013403EB061398612846202110F08DFA80
:1075A000054640B10135284600F0B4FB124B0134CA
:1075B00003EB0613D8612846202110F07EFA10B99B
:1075C000FFF7A8FD12E0013000F0A4FB0A4B032CEA
:1075D00003EB06163062F3D11148FFF727FF05E0F1
:1075E0001048114901220C2300F0A4FD04B0BDE8AD
:1075F000F08100BFE4C901084C280020FFC9010840
:1076000005CA01080DD50108DEC9010809CA01082B
:10761000E8AD01080ECA010898C801081DCA010892
:1076200064C701087DC901089CC90108F0B5047848
:1076300087B0064614BB514B19201968062303FB7B
:10764000041191F8CA5091F8CE20454305F56175B3
:1076500091F8C930009591F8CB50C831684300F5D6
:10766000617001900879029049794548039121465B
:10767000013400F05FFD0C2CDDD17DE010F080FACC
:107680000B28044672DC3D4B701C1D682021002332
:107690008DF8173010F011FA064680B101363046E9
:1076A00010F06EFA03289FBF062303FB045383F8F0
:1076B000CE009DF817309CBF01338DF8173030464F
:1076C000202110F0FAF9074680B10137384610F052
:1076D00057FA0D289FBF062303FB045383F8C90004
:1076E0009DF817309CBF01338DF81730062666438E
:1076F000A9193846CA310DF11702FFF767FC20219E
:1077000010F0DBF9074670B10137384610F038FA4F
:1077100014289FBF9DF817307619013386F8CC00E6
:1077200098BF8DF817303846202110F0C6F978B18F
:10773000013010F025FA0D289FBF062303FB0453E8
:1077400083F8CD009DF817309CBF01338DF81730BA
:107750009DF81730062B0FD0062202FB04500021A3
:10776000C93010F074F9FFF7D5FC05E0054806496B
:1077700000220B2300F0DEFC07B0F0BD201100203A
:1077800029CA01087DC901089CC90108F0B5027821
:1077900087B08AB94A4C04F1200694F8E821002306
:1077A000484950B2595681426DD00C33302BF7D135
:1077B0000834B442F1D180E0002204920592451CC5
:1077C00010F0DEF9C4B260B207F0F2F8074618B163
:1077D0008DF81040012400E004462846202110F0D6
:1077E0006CF9054638B10135284610F0C9F9013465
:1077F000ADF81200E4B200262846202110F05DF911
:10780000B0B3451C284610F0BBF900222E495FFAA0
:1078100082FE51F82230834204D00132082AF5D189
:10782000002300E0734651F82320824220D1022E2B
:107830000FD0032E12D05A1E012ED2B204D0042A29
:1078400013D88DF814300EE0042A0ED88DF81530B8
:1078500009E0052B09D88DF8173004E09A1E052A97
:1078600003D88DF816300134E4B20136042EC3D1AA
:10787000052C03D807B0BDE8F0404BE404AB03CBC4
:107880003860796019E094F8ED010F4B94F8EC51F1
:1078900053F82000B4F8EA21009094F8EF0153F86F
:1078A0002000019094F8EE0153F8200053F82530A1
:1078B0000290064800F03EFC7AE707B0F0BD00BF3A
:1078C0004C28002000240020ACC2010849CA01084D
:1078D000F7B5047805464CB9204601A90BF020FD08
:1078E0000134FFF7F5FF0E2CF6D150E010F048F907
:1078F000C6B20D2E47D8681C202110F0DEF80346D2
:1079000050B15B780130682B07D0732B01D1012770
:1079100004E0FFF7FFFB3AE000E00027202110F031
:10792000CCF81C4C06F1D005C8B1013010F028F994
:1079300040F2ED2380B2984205DD40F6CA0398423A
:10794000A8BF184601E040F2EE20A0F2EE20192276
:1079500090FBF2F004EB450304F81570587014F82E
:10796000153004EB45046278012B4FF0190303FB3B
:1079700002F331460CBF7322682203F2EE2306485D
:1079800000F0D8FB03E005480E2100F0D3FB03B064
:10799000F0BD00BF4C28002068CA01087ACA01085F
:1079A00010B50446204607F0C8F918B90A2007F0B8
:1079B00022F9F7E710BD002207490C2303FB02134D
:1079C0005968814204D10022C2621A725A6070471B
:1079D0000132042AF0D17047002400202DE9F04F35
:1079E000064687B088469DF8407011461A469DF8B5
:1079F000443000250C206843594C00EB040E00571E
:107A0000A146B04205D19EF808A0BAF1000F04D0FB
:107A1000A2E00135042DEDD19EE0022E00F08C8015
:107A200005DC002E40F0988000934E4886E0142E2E
:107A30000AD01E2E40F09080504601F041FA39469F
:107A4000044607F077F97DE0474F484CBB690322B5
:107A500043F00403BB614FF4805B204605A98DF819
:107A600016200392ADF814B08DF8176005F01EFED5
:107A7000C4F814B0C82007F0BEF8C4F810B0BB6951
:107A8000039A43F00403BB614FF4C053204605A999
:107A9000ADF814301C23364C8DF816208DF81730B5
:107AA00005F004FE334A4FF4802353614FF0010B7D
:107AB000636304F13400082384F8393084F83AB061
:107AC0000BF0E0F92C4B2D4AC3F800A0FB6905A888
:107AD00043F40003FB612A4BDA6002238DF8153072
:107AE0008DF814608DF816A08DF817B00BF0ACF976
:107AF0002A238DF814309DF817308DF815B08DF8C5
:107B000016A01BB105A80BF09FF904E01D4B4FF424
:107B10008062C3F884201C4B1C4A1D49136002225A
:107B20001A721C4B1C4A13601C4A1B681160984750
:107B30001B4B63601B4C06E01B4800933B4604F064
:107B400085FA044644B10C2303FB059526712046B3
:107B500085F808806C6000E0002007B0BDE8F08F79
:107B600000240020003801400010024000080140BD
:107B7000AC12002000040140D80042420005FA0582
:107B800000ED00E000E100E0DC220020D82200202F
:107B900020000020C8000020D4200020D020002099
:107BA000A4A60108B012002000480040F0B501244E
:107BB000B0FBF4F58D4201D34C43F9E70026D4B174
:107BC000B0FBF4F504FB1500B4FBF1F41EB9002D75
:107BD00001DC002CF3D1092D03F1010EEFB204DD1D
:107BE000002A14BF3725572500E030253D441D707D
:107BF00001367346E3E71C70F0BDF0B50124B0FB1D
:107C0000F4F58D4201D34C43F9E70026D4B1B0FB23
:107C1000F4F504FB1500B4FBF1F41EB9002D01DCF2
:107C2000002CF3D1092D03F1010EEFB204DD002A7F
:107C300014BF3725572500E030253D441D7001361F
:107C40007346E3E71C70F0BD03685A1C02601970AC
:107C500070472DE9F843089E002B074688461446D6
:107C6000334614BF4FF030094FF0200913F8012BB1
:107C70000AB9254603E0002CFBDD013CF6E7002DA8
:107C800004DD38464946C047013DF8E7354624EA59
:107C9000E474A01B284415F8011B11B13846C047F5
:107CA000F7E7BDE8F883024B186807F052B800BF49
:107CB000780F0020F8B507460C46486800211546A5
:107CC0001E460CF0E3FA58B128460CF0F7F81049BC
:107CD0000CF048F901464FF07E500CF0F7F9606067
:107CE000616830460CF036F8014630460CF0EEF98B
:107CF00025680646294638460CF02AF801463046E3
:107D00000CF030F9014628460CF024F82060F8BD4C
:107D1000DB0FC9402DE9F04102780346202A00F12B
:107D20000100F9D0092AF7D02D2A02D10346414D8E
:107D300004E02B2A08BF03464FF07E551C46002660
:107D4000234614F8012BA2F13007F9B209290DD806
:107D5000394930460CF006F9064638460CF0AEF8C4
:107D6000014630460BF0F6FF0646E9E72E2A17D10A
:107D7000314F234614F8010B3038C2B2092A0FD80C
:107D80000CF09CF839460CF0A1F9014630460BF096
:107D9000E1FF2949064638460CF0E4F80746E8E7D3
:107DA0001A7802F0DF02452A39D15A782D2A02D1F9
:107DB0000233012704E02B2A14BF013302330027CA
:107DC000013B002413F8012F303AD1B2092903D81E
:107DD0000A2101FB0424F5E7B4F59A7F28BF4FF48C
:107DE0009A74A0464FF07E53B8F1070F07D9184692
:107DF00012490CF0B7F8A8F108080346F4E704F0BC
:107E0000070434B118460C490CF0ACF8013C0346A9
:107E1000F7E719462FB130460CF058F904E04FF05F
:107E20007E5130460CF09EF8014628460CF09AF838
:107E3000BDE8F081000080BF0000204120BCBE4CA6
:107E400030B5054687B00C4603A800210C220FF080
:107E5000FEFD284600210CF041FA20B128462849B1
:107E60000BF078FF03E0284625490BF071FF254908
:107E70000CF078F80CF03CFA054680EAE0706946B0
:107E8000A0EBE5700BF04CFA002DACBF20232D23A6
:107E900068468DF80C300FF01EFE012807D1302304
:107EA0008DF80D308DF80E308DF80F300CE0022873
:107EB00005D130238DF80D308DF80E3004E0032805
:107EC00004BF30238DF80D30694603A80FF0E6FD9E
:107ED00003A80FF000FE0338C5B22A4603A92046C6
:107EE0000FF024FE00236355204607490FF0D6FD0E
:107EF00003AB204659190FF0D1FD204607B030BD25
:107F00006F12033A00007A4491CA010870B5064620
:107F1000B6FBF2F40846154614B12046FFF7F6FF0B
:107F200005FB1464024B1B5D00F8013B70BD00BFF4
:107F300093CA01082DE9F04F81468A4616461C4631
:107F400089B000253178002900F0DB80252902D096
:107F50000136484674E072784FF00008302A0CBFB2
:107F6000B278B71CA2F1300312BF4FF0000BF71C20
:107F70004FF0010B092B19D8A2F13003D9B209290E
:107F800005D80A2202FB083817F8012BF4E7A2F102
:107F90006103052B02D8A2F1570305E0A2F14103CA
:107FA000052B03D8A2F137030A2BEADD6C2A30D166
:107FB0003A787E1C642A00F083800BD8252A3DD0B5
:107FC00003D8002A00F09D80BCE7582A0CD0632A11
:107FD00019D0B7E7732A22D002D86E2A37D0B1E77A
:107FE000752A5CD0782AADD1271D2068A2F15804EB
:107FF00062424FF01001624155E02CD9582A32D02C
:10800000632A2AD13E4648462178271DD0470135AC
:108010000FE0642A63D00ED9732A14D13E46236838
:1080200048460093514642460023FFF712FE271DA3
:1080300005443C4686E7252ADFD13E4648462521B1
:10804000D04701357EE70AD86E2A06D13E4623681E
:1080500004341D6076E7002A53D03E4672E7752A45
:1080600026D0782AF9D1A2F1580304F1040C5A421F
:108070002068CDF80CC04FF010015A4105ABFFF756
:1080800095FDDDF80CC03E46644605AB00934846BE
:10809000514642465B46FFF7DCFD054452E7206847
:1080A000271D0A21002205ABFFF7A7FD3C46ECE7A0
:1080B00004F1040CCDF80CC020680A210022DDE791
:1080C0002068271D002808DA2D238DF8143040423F
:1080D0000DF115030A210022E6E705ABFAE7206857
:1080E00004F1040C00280ADA2D238DF814304042E4
:1080F0000DF11503CDF80CC00A210022BFE705AB36
:10810000F8E7284609B0BDE8F08F0EB40FB505AB0F
:1081100053F8042B0190064901A80393FFF70AFFC7
:10812000019B00221A7004B05DF804EB03B07047A5
:10813000497C00080FB413B50B4904AB08680B4920
:1081400053F8042B09680193FFF7F4FE0446084B2B
:10815000186806F0F2FD0028F9D0204602B0BDE80C
:10816000104004B0704700BF7C010020780100205F
:10817000780F002080EAE073A3EBE0738B4206DB0C
:10818000002801DD401A704702D0084470470020E3
:10819000704770B504460CF0ABF82030402857D833
:1081A00020462C490CF09AF828B120462A490BF0B9
:1081B000CFFD0446F4E7204628490CF071F828B1B9
:1081C000204625490BF0C6FD0446F4E72046244925
:1081D0000CF084F830B1224920460BF0B9FD01467D
:1081E0001F480AE020461F490CF05AF840B11C49CC
:1081F00020460BF0AFFD01461A480BF0A9FD0446DE
:10820000214620460BF0AEFE0546204629460BF0DF
:10821000A9FE1549064628460BF0A4FE13490BF0AB
:1082200097FD014628460BF09DFE11490BF092FD8B
:10823000014628460BF096FE0E490BF089FD0146DB
:1082400030460BF08FFE014620460BF083FD70BDDB
:10825000002070BDDB0F4940DB0FC940DB0F49C078
:10826000DB0FC93FDB0FC9BF9A7C2E36FAAF4F39FF
:108270003587083CA4AA2A3E08B503490BF06AFDDD
:10828000BDE8084085E700BFDB0FC93F2DE9F04F8F
:10829000056885B0814628460C46FFF7EDFF80460D
:1082A0002846FFF776FFD9F8045006462846FFF720
:1082B000E3FF07462846FFF76CFFD9F8089005460C
:1082C0004846FFF7D9FF82464846FFF762FF41461E
:1082D000814650460BF046FE4146834648460BF029
:1082E00041FE5146019030460BF03CFE494602905B
:1082F00030460BF037FE3946039050460BF032FE05
:108300004946206007F100400BF02CFE29466060D2
:10831000A56002980BF026FE014601980BF01AFDAD
:108320002946E06003980BF01DFE014658460BF00D
:108330000FFD3946206106F100400BF013FE29467F
:10834000606158460BF00EFE014603980BF000FDED
:108350002946A06101980BF005FE014602980BF03A
:10836000F9FC4146E06138460BF0FCFD206205B0A7
:10837000BDE8F08F2DE9F04107688AB0466885684E
:108380000446084601A9FFF781FF019938460BF022
:10839000E9FD0499804630460BF0E4FD0146404675
:1083A0000BF0D8FC0799804628460BF0DBFD014610
:1083B00040460BF0CFFC0299206038460BF0D2FD0E
:1083C0000599804630460BF0CDFD014640460BF046
:1083D000C1FC0899804628460BF0C4FD0146404682
:1083E0000BF0B8FC0399606038460BF0BBFD0699B2
:1083F000074630460BF0B6FD014638460BF0AAFCA6
:108400000999064628460BF0ADFD014630460BF0B3
:10841000A1FCA0600AB0BDE8F081074B10B51A8836
:108420001C4622EA00009042188002D0012006F08B
:1084300039FC208810BD00BFA8120020064B10B5E3
:108440001A881C4610439042188002D0012006F082
:1084500029FC208810BD00BFA8120020024A9368A2
:1084600023EA0000906070474C28002008B5104BAC
:108470001A780023D9B2914207D20E49002051F850
:108480002310013309680880F4E7322006F0B3FBBB
:10849000094B1B685A0309D5084B9B685B0305D43D
:1084A000BDE8084040F2DC5006F0A5BB08BD00BFA7
:1084B000182100201C210020EC2700204C2800203F
:1084C0004B4A68232DE9F341137040F2CC7353807B
:1084D000BE231371EF2382F8C937002319461646CD
:1084E00082F8CA37F25C0133514040F2CC729342B9
:1084F000F8D13F4B3F4A83F8CA173F4B04275A60D5
:1085000002F188325A600020013F17F0FF075ED069
:10851000394B3422394CDA6004F17848A8F5FC383C
:10852000C8F3090353B100234FF4005056F80880F4
:10853000019304F097FF0428E6D11CE04FF43020AB
:1085400004F090FF0428DFD12B4D4FF430202B692D
:1085500043F002032B616C612B6943F040032B61F4
:1085600004F080FF41F6FD732A69042803EA020340
:108570002B61D8D0C8E7204D4FF400502B6943F051
:1085800001032B611FFA88F3238004F06BFF04289A
:1085900013D1A31C0193019B4FEA1848A3F8008054
:1085A0004FF4005004F05EFF41F6FE732A69042880
:1085B00003EA02032B6106D0A6E741F6FE732A699F
:1085C00013402B61A0E70E4B04349C42A4D10A4A0D
:1085D0000428136943F08003136102D109F020F9E4
:1085E00010B90A2006F076FB02B0BDE8F08100BFAA
:1085F0004C280020230167450020024000F80108B4
:10860000CCFF01082DE9F04109F00AF910B90A2060
:1086100006F060FBBB4CBC4940F2CC7220460FF028
:108620000BFA94F8A0374FF4CC71022B84BF0023CF
:1086300084F8A03794F8A027B44D01FB02F303F5AA
:10864000367020442344286093F82C0301FB024237
:10865000022803F54A7384BF0020187192F82C3366
:10866000AB4A13700C2202FB0343AA4A03F2A27323
:10867000136046F20902A3681A401AB9A14A43F4EA
:1086800000539360A368DF0703D54FF40050FFF752
:10869000E5FEA3685E0409D50820FFF7DFFE4FF46E
:1086A0000050FFF7DBFE0120FFF7D8FEA368180794
:1086B00006D54FF40050FFF7D1FE0120FFF7CEFEA4
:1086C000A368990413D54FF40040FFF7C7FE8D4B04
:1086D00093F88431012B03D14FF40060FFF7BEFE05
:1086E0004FF48030FFF7BAFE4020FFF7B7FEA368D3
:1086F0005A0603D54FF48030FFF7B0FE022006F093
:1087000057F9854E40B1438833B133689B0303D595
:108710004FF40030FFF7A2FE94F8D221794B2AB132
:1087200093F8D62112B1002283F8D621336803F4DE
:108730001073B3F5107F03D14FF40070FFF78EFE76
:108740004FF0000C6746754E754B1E6004EB0C0332
:10875000B3F8EAE14FEA5E0101F077314FEA9E0398
:1087600003F03333C1EB0E00C11A4FEADE0303F00E
:108770001133CB1A03EB231303F00F32FF2392FBC9
:10878000F3F31EF00108C3EB032318BF0137A2EB7C
:10879000030318BFFFB2012B0ADD022B40F0AE80AD
:1087A000B8F1000F00F0AA801EF0BC0F00F0A68008
:1087B0000CF1080CBCF1200FC8D1013F012F00F2D1
:1087C0009D8009F009F83022002156480FF03FF94A
:1087D000554F564BD5F800801F60554B002108F1CE
:1087E0007900C3F8008006F0A7F9524B80F0010031
:1087F0001870514B07F126021A60504B07F1C40262
:108800001A6098F8000006F0CDFE28684C4B00F581
:10881000C5721A6002F0ACFF4A4B07F18A021A6077
:10882000494B00221A809A71484B2D6807F12A02A1
:108830001A60474B05F219121A60464B05F289126D
:108840001A60454B07F108021A60444BDFF8488173
:108850001F60434B07F192021A6007F19C03C8F8AE
:108860000030404BB4F866011E600BF023FBC8F8E3
:108870000800B4F868010BF01DFB95F85C3008F1B6
:10888000040288F8043095F87830C8F80C0088F8AD
:10889000053094F8D531286E88F81030324BC8F87E
:1088A00014501A60314B05F164021A6030490BF024
:1088B00059FB01464FF07C500BF008FCB5F816410F
:1088C0002C4B186020460BF0F9FA01462A480BF0B1
:1088D000FDFB2A490BF046FB294A2A4B15602A4A20
:1088E000186005F168031360284A05F21115156038
:1088F000274A1760274A1360BDE8F08109F09EFC03
:108900005FE700BF4C28002000F80108201100207C
:10891000F820002048110020EC270020D429002056
:10892000D0260020BC0F002090290020F00F00204E
:10893000F40F0020080000205008002098060020B6
:1089400000100020A80F002070300020A408002094
:10895000D81C00207C0A0020EC1F0020F01F002003
:1089600090090020540A002074200020B420002028
:10897000DB0F4940B0200020000061444C3D0F4413
:108980001C0800208C090020100800207C09002011
:108990008409002018070020E812002008B5FFF71E
:1089A0008FFDFFF72FFEBDE80840012006F07AB9E1
:1089B000426A806A131A58425841704741717047A1
:1089C00043799B070AD5436A8269D154436A016996
:1089D0000133B3FBF1F201FB123343627047437979
:1089E00013F001031FBFC36803F1FF32C369006ABC
:1089F0001DBF181A1040C0B218467047437910B511
:108A000013F0010304460DD0FFF7E9FF58B1236AC4
:108A10006269E168D05C0133B3FBF1F201FB123310
:108A2000236210BD184610BD90F83B3210B57BB9DB
:108A300090F83A3290F83942A34209D2B0F8401285
:108A400001229A400A430133A0F84022DBB2F3E747
:108A500010BD8379DB0748BFB1FA81F1D0F834311A
:108A600048BF49095A681B8909B1136170475361AE
:108A7000704710F80A3C0133DBB20A2B84BF10F8B0
:108A8000131C054A00F80A3C82BF002322F811306B
:108A900000F80A3C704700BFB8260020354A70B580
:108AA000136C90681944344B1B78D94040F68C23E2
:108AB000081A98429160D060516013463BD91278F1
:108AC00093F9451010468A420BD1111F082908D886
:108AD00093F84610182901D8013103E083F84420A7
:108AE00002E0002183F8461093F944402149A24254
:108AF00019D191F84740B4B10C310024944206DA00
:108B000051F8046F1D4D25F814600134F6E70C2868
:108B100005D01A49002421F810400130F7E7184821
:108B200001780131017083F84520002201211A707B
:108B300083F8471070BD92F84710C9B140F2DA517E
:108B4000A0F2EF248C4208D811780B2905D80B1D10
:108B50000131117042F8230070BD002283F84720D4
:108B6000084B03F13002002143F8041F9342FAD16D
:108B700070BD00BFA00100209F010020B82600208A
:108B8000D8060020AC010020024A136C01331944BE
:108B900011647047A0010020024B53F820301B687D
:108BA000198070471C210020074BA1F57A7153F8FA
:108BB00020301A681B8959434FF47A7391FBF3F103
:108BC00089B21180704700BF1C2100201FB501230E
:108BD000ADF80830ADF80410002301A9ADF80A3053
:108BE000ADF80C30ADF8062004F04DFC05B05DF892
:108BF00004FB38B5A0F513746379A579DB0745D577
:108C000094F8383205F00105F3B1226B1068838DBA
:108C1000C3F34E03838494F83C3223B1B4F8423258
:108C20000133A4F84232917A6A00FFF7CFFF0123A3
:108C300084F83B32002384F8393284F83A3284F8DD
:108C40003832A4F8403238BD94F83B322046012B2C
:108C500004BF94F8393284F83A32FFF7E5FE94F80D
:108C60003B22236B3AB9012284F83B221868997A97
:108C700005FA02F207E0002284F83B2295421868C8
:108C8000997A08BF0222BDE838409FE738BD10B589
:108C9000A0F5127494F83C22BAB9A36A616A9942A9
:108CA00028D0591CA069A162C35C2069DBB25B00BB
:108CB00043F400738142A4F83E324FF00A0384F873
:108CC0003D3228BFA262012312E094F93D327BB10C
:108CD000B4F83E1220464B08A4F83E3201F00101E0
:108CE000FFF7B7FE94F83D32013B84F83D3201E0D6
:108CF00084F83C3294F83832002B4ED194F8393253
:108D00000133DBB2092B84F8393203D12046BDE8A8
:108D1000104089E60A2B40D194F83B322BB9B4F8C5
:108D2000403243F00103A4F840326379D9071CD5DF
:108D3000B4F84002820501D4C30705D4B4F8443224
:108D40000133A4F8443210E0E36AC0F347000BB1EA
:108D500098470AE0E3696269D054E369E168013346
:108D6000B3FBF1F201FB1233E361012284F83822F4
:108D700094F83B220023012A84F839320DD1A279DC
:108D800084F83B32236B12F0010F1868997A0CBFFC
:108D900002220022BDE8104018E710BDF0B5046DB6
:108DA0008279A389467923F4005312F0020F4FEA27
:108DB00003434FEA13430CBF00214FF4005112F05C
:108DC000040FA38114BF4FF4806E4FF0000E16F015
:108DD000010F8768054614BF04200020B307238ACB
:108DE00048BF40F008029BB223F4405343EA01031A
:108DF0002382A18948BF90B289B221F4B05121F0F9
:108E00000C014EEA010140EA0102A281A38A87B067
:108E100023F440731B041B0CA38201A804F0D8FAAE
:108E2000039B049E254A944218BF1E46A38919221B
:108E300072431BB2002BB4BF7E00BE00B2FBF6F63D
:108E40006427B6FBF7F00001010907FB1163A28953
:108E500012B2002AB7BFD9001A013231B1FBF7F2C2
:108E6000A7BF3232B2FBF7F302F007021043A8BFEC
:108E700003F00F03AA79A8BF184380B212F0010FC4
:108E800020812B6D06D00D498B4202BF0420A1F535
:108E90003051086112F0080F9A8A0BBF22F00802C5
:108EA00092B2120442F0080208BF120C9A829A8908
:108EB00092B242F400529A8107B0F0BD00380140EE
:108EC0002DE9F04F4E4C4FF4147585B08046914615
:108ED0001E4605FB0045274620B94A4B2B63103B35
:108EE000C5F834314FF4147303FB08F3464AFC18F9
:108EF000FA5003226271224603F59C733B44E162FF
:108F0000A36100214FF48070D4F8343134324FF033
:108F1000010B62612162E161A162616284F83C122D
:108F200084F83912A4F84212A4F84412C4F8089044
:108F3000A671E060206184F838B284F846825868EF
:108F40001B890222ADF80C3003A910238DF80E30D6
:108F50008DF80F20019207F04FF8236B019A597B8F
:108F600058681B898DF80E1003A9ADF80C308DF8E8
:108F70000F2007F041F828465946FFF76AFD3220D6
:108F800005F039FE214BD4F834A11B681A46B2FB18
:108F9000F9F1B1F5803F03D3012AF8D95208F6E779
:108FA0001B4A5046B3FBF2F289B2D2B202F082FF02
:108FB0004FF4147000FB08F0164B07EB000800F5A7
:108FC00012703C180022C8F848325046214602F080
:108FD000B9FFD8F8307016F0010F0CBF0222002242
:108FE0003868B97AFFF7F2FD0B4B3846C8F84C32B7
:108FF000211D002202F0A6FF284605B0BDE8F08F33
:109000000013002090C301087CAB0108040100207C
:1090100040420F008F8C0008F38B000803460A467D
:1090200090F84602D96A9B794AE71FB50123ADF84B
:1090300008300023ADF80C30ADF80A30084BADF81D
:1090400004101B7801A9012B08BF0323ADF80620EB
:1090500008BFADF80C3004F016FA05B05DF804FB5B
:109060009C01002038B510F80E2C044650F8043C42
:1090700052B9012200F80E2C20F80C1C997A1868BD
:109080000222BDE83840D0E730F80C2C20F80A1C4A
:10909000891A89B220F8081C074A10F80F0C00251D
:1090A00022F8101004F80E5C1868997A2A46FFF727
:1090B000BCFF04F8065C38BDB8260020044B53F80A
:1090C00020301BB107289CBF1B681980704700BF68
:1090D000C80200202DE9F7438E460546DFF8A0922E
:1090E000114699F850420068164698467246631C2D
:1090F00089F8503202F08AFE2B8901A9ADF80430BC
:1091000018238DF80630686802238DF8073006F0C2
:1091100073FFAB7A09F51577240127442A6849467D
:109120000C2B00F2F680DFE813F00D00F400F400E1
:10913000F4005100F400F400F4008A00F400F4009C
:10914000F400C200138CDFF83CC223F001031B04BF
:109150001B0C1384138CB2F804E0108B624520F0D2
:1091600073004FEA00404FEA10409BB21FFA8EFE98
:1091700040F0700014D00CF5006C624510D00CF576
:10918000406C62450CD00CF5806C624508D00CF543
:10919000806C624504D023F0020343F0030307E030
:1091A00023F00E032EF4407E43F003034EF4807E42
:1091B000A2F804E01083A2F834801384138B23F008
:1091C00008031B041B0C43F0080336E0138CDFF884
:1091D000B4C123F010031B041B0C1384138CB2F8CE
:1091E00004E0108B624520F4E6404FEA00404FEA6D
:1091F00010409BB21FFA8EFE40F4E04008D00CF500
:10920000006C624504D023F0200343F0300307E0F4
:1092100023F0E0032EF4406E43F030034EF4806EF2
:10922000A2F804E01083A2F838801384138B23F48F
:1092300000631B041B0C43F40063138369E0138C6D
:10924000DFF840C123F480731B041B0C1384138CC0
:10925000B2F804E0908B624520F073004FEA0040C2
:109260004FEA10409BB21FFA8EFE40F0700008D00B
:109270000CF5006C624504D023F4007343F4407392
:1092800007E023F460632EF4405E43F440734EF431
:10929000805EA2F804E09083A2F83C801384938B54
:1092A00023F008031B041B0C43F0080330E0138C6D
:1092B000DFF8D0C023F480531B041B0C1384108CE4
:1092C000B2F804E0938B20F4005023F4E6431B042F
:1092D00000041B0C000C62451FFA8EFE43F4E043B1
:1092E00040F4405003D00CF5006C624503D12EF4DD
:1092F000804E4EF4804EA2F804E09383A2F84080A2
:109300001084938B23F400631B041B0C43F4006351
:1093100093832B7B43B1B2F844306FEA43436FEA47
:1093200053439BB2A2F8443013889BB243F001032D
:109330001380AB7A0C2B19D8DFE803F00718181844
:109340000B1818180F18181813000B1902F1340015
:109350000AE00B1902F1380006E00B1902F13C009B
:1093600002E00B1902F14000C3F8540238460C44E5
:10937000A4F85C62C4F8582203B0BDE8F08300BFD3
:1093800000130020002C0140084A13689B020BD5F3
:10939000074B002119704FF6FE7306490868034019
:1093A0000B604FF400135360704700BF0000024091
:1093B000A53000206C0002400028114AB8BF40428E
:1093C00090FBF2F330B50F4C3C2504FB03006843DF
:1093D0000D4D90FBF2F22D682D7B25B903EB830335
:1093E00003EB830301E0C3EB031302EB830304FBF2
:1093F00002020B804FF47A7392FBF3F24A8030BD85
:1094000080969800806967FFD8110020022803D059
:10941000431E584258417047064B1B681B7823B1C6
:10942000054B1868C0F3C0407047044B1878C0F370
:109430008000704798060020E8100020A630002029
:10944000A0F17D03012B70B504460D460A4E05D8E8
:1094500030687D2105F07DFC84F0200430682146D1
:1094600005F077FC35B12B881C4404EB142404F080
:10947000FF042C8070BD00BF9812002010B50A4C6C
:109480005E280146206805D15D2105F062FC206858
:109490003E2105E05D2903D105F05BFC20683D21FC
:1094A000BDE8104005F055BC1416002037B51A4B26
:1094B0001A4C1B491B4A20B11B480088B0F5805F3D
:1094C00021D209881278154D9B79ADF804108DF8DA
:1094D000062001A8291D04228DF807300EF09CFA01
:1094E000C0B101986860532008F0BCFCA08808F067
:1094F000EBFCA07908F0E8FCE07908F0E5FC0A4B09
:1095000000221A8006E0098812789B79A180A27156
:10951000E371E8E703B030BD70300020141600207E
:10952000A8120020E8110020F82500202DE9F843BA
:1095300005460E460D4B002493E88003B44213DA2F
:109540007B1933F9140008EB050333F9142009EBF8
:10955000050333F9143001341344022293FBF2F370
:10956000C01A08F0C0FCE9E7BDE8F88354240020E5
:1095700030B585B004AC002524F8025D0091ADF84B
:10958000060021461020FFF75BFF9DF806002146EC
:10959000FFF756FF9DF807002146FFF751FF9DF8A2
:1095A00000002146FFF74CFF9DF801002146FFF720
:1095B00047FF9DF802002146FFF742FF9DF8030098
:1095C0002146FFF73DFF9DF80E002946C043C0B27B
:1095D000FFF736FF05B030BD10B5054C206805F02B
:1095E000B5FB18B1206805F0AEFBF6E710BD00BF73
:1095F0006C12002010B50446C0B2FFF73FFFC4F361
:109600000720BDE8104039E7024B5E21186805F0DD
:10961000A0BB00BF1416002038B50546054C5E21DE
:10962000206805F096FB20682946BDE8384005F023
:1096300090BB00BF1416002013B5044601A90068B2
:10964000FFF7BAFE1320FFF7E7FFBDF90400FFF7AD
:10965000D1FF1B20FFF7E0FFBDF90600FFF7CAFFAF
:109660002320FFF7D9FF2368002BB4BF53204E20DF
:10967000FFF7C0FF01A96068FFF79EFE1220FFF709
:10968000CBFFBDF90400FFF7B5FF1A20FFF7C4FFB9
:10969000BDF90600FFF7AEFF2220FFF7BDFF6368AC
:1096A000002BB4BF57204520FFF7A4FF02B010BD28
:1096B000674B73B51878FFF7A9FE664D04462B7803
:1096C000834220D0C8B1644B1B68E3B193F900001A
:1096D00002230093614B04211B6800225B78003356
:1096E00018BF012301934FF41653FEF777F95C4B33
:1096F000186040B101232B7005E0594E3068FEF729
:109700005AF934602C70574B574D1878FFF77EFE8E
:109710002B780446834218D088B1544B1B68A3B100
:109720000022012493F9000008214FF4964300948D
:109730000192FEF753F94E4B186028B905E04C4EE4
:109740003068FEF738F934602C704A4B4A4D18786F
:10975000FFF75CFE2B78044683422E4643D0002858
:1097600038D0464B1A68002A3DD0D37992F90000D0
:10977000002B4FF00202424C08BF0223009200224D
:1097800054F8233001921021FEF728F93D4B05468D
:10979000186040B33C4C94F84A30022B0BD094F83C
:1097A0009620022A01D14C3405E023B1002A04F1AD
:1097B0004C0418BF0024354B1C6044B120460021E6
:1097C0004C220EF044F90223256084F84A3001232C
:1097D000337008E02B4E306807F024F83068FEF74D
:1097E000EAF834602C702A4B2A4D1878FFF70EFEE9
:1097F0002B780446834229D000B3274B1B682BB338
:10980000264A93F900001268032352782021002A87
:109810000CBF08220922009301924FF461430022F9
:10982000FEF7DCF81E4B186080B11E4A012313704E
:109830002B701D4B1A681D4B1A6007E0184E3068DC
:10984000FEF7B9F8174B34601C702C7002B070BD75
:10985000A0060020A81100209C060020D81100209E
:1098600014160020A8060020F8110020A4060020ED
:109870006C120020B40600207E120020B0060020EA
:10988000ACC20108801200203C230020841200207A
:10989000C006002094120020BC060020B80600205C
:1098A000981200209C12002010280020A0120020F6
:1098B0002DE9F74305F07AF9924CA368C31A002BFF
:1098C000C0F2618300F5433303F5A073A3608E4BB0
:1098D0001D78237BC5F38005EB1A18BF0123257380
:1098E0004DB1002B00F04F83884B5A789A700122BB
:1098F0005A701A702BE0854A2BB1D37843F00203DB
:10990000D37093785370D67806F0020101F0FF030C
:1099100039B97E498968411A002903DB06F0010341
:1099200000E0012303F00107784917707BB1F207CB
:109930000DD50A7905230132D2B2B2FBF3F303EB62
:109940008303D31A724ADBB20B71D35C4B706F4E38
:10995000DFF8088233787BB3F37823F00203F370E7
:109960006C4B0344AE20B36006F0C7FC08B106F0B0
:10997000C9FC88F80000002800F00583B02006F03C
:10998000BCFC402006F0B9FC002006F0B6FC10201C
:1099900006F0B3FC4FF48067013F0020BFB206F031
:1099A00083FC002FF8D1384606F01BFD72785A4B25
:1099B00053F8220006F098FC98F80030002B00F0D5
:1099C000E2827378062B00F2B382DFE813F007001F
:1099D000B102180078006B018801ED014F49504A2F
:1099E000504B5148FEF791FB012006F0FAFC4E481F
:1099F00006F07AFC022006F0F4FC4C48ADE14C4F36
:109A00003B689B0735D5DFF858810A23B8F800106A
:109A1000DFF85091B1FBF3F203FB121399F8001039
:109A200092B29BB2009140484249FEF76EFB00F0B3
:109A300019FB012006F0D5FC3B4806F055FC3E4BD7
:109A400099F800201868B8F80030067902FB163142
:109A500064234B43C17802208E1B5643B3FBF6F6BA
:109A6000F6B206F0BEFC3146152000F0BFFA032620
:109A700000E001263B681F0540F15A822F4B304918
:109A80001F68642397FBF3F2096803FB12730091CC
:109A900025482C49FEF739FB00F0E4FA304606F081
:109AA000A0FC214806F020FC03F028FF0746701CAC
:109AB00006F097FC1520394600F098FA38E20120AC
:109AC000214F06F08EFC214806F00EFC3B689807FB
:109AD0004AD51F4A1448B2F90210B2F90030009179
:109AE000B2F904201B4901921B4AFEF70EFB00F05D
:109AF000B9FA022006F075FC0B4806F0F5FB0326C8
:109B000033E000BF14160020A6300020941C002073
:109B1000B8CA0108404B4C0094AB0108BDCA01080B
:109B2000C6CA010869C4010821160020CDCA01086F
:109B3000EC270020D2CA0108D0110020DC1100203F
:109B4000E0110020EACA0108E4110020FFCA010860
:109B5000B211002015CB010824CB0108E902002036
:109B6000D4110020F800002002263B68D9071AD53E
:109B70007B4A7C48B2F90210B2F900300091B2F988
:109B8000042079490192794AFEF7BFFA06F10108EB
:109B900000F068FA304606F024FC5FFA88F8714855
:109BA00006F0A2FB46463B681A0718D5704A6D4876
:109BB000B2F90210B2F900300091B2F904206A49FA
:109BC00001926C4AFEF7A1FA771C00F04BFA30467E
:109BD00006F007FCFFB2634806F086FB3E46664A85
:109BE0006149B2F90030B2F902205E480092634A3E
:109BF000DFF8B091B2F90020771C0192604AFEF7BD
:109C000084FA00F02FFA304606F0EBFB554806F0D8
:109C10006BFB5449D9F80000FEF712F951480DF0DA
:109C20005AFFFFB2C1B2092909D84B1CDBB221444B
:109C300020224A730021E21891731946F3E7DFF8F6
:109C40002481D9F804004144FEF7FAF800F00AFA3A
:109C5000384606F0C6FB404606F046FB4146D9F8BA
:109C60000800FEF7EDF840460DF035FF0236F6B27B
:109C7000C7B2092F09D87B1CDBB2274420227A7394
:109C80000021E21891731F46F3E73E4BB3F9000041
:109C90000AF014F908EB0701FEF7D2F800F0E2F938
:109CA000304657E00026384F3B78B34240F24081BF
:109CB0000E2E00F03D817008013006F092FB304618
:109CC00009F008FB3B78B34206D9202006F0F1FAF0
:109CD000701CC0B209F0FEFA0236F6B2E3E72B4E72
:109CE0002B4996F8A0271F48FEF70FFA012006F02F
:109CF00078FB1C4806F0F8FA264B27491F781948CC
:109D00003A46FEF702FA022006F06BFB154806F011
:109D1000EBFA0C2303FB0766204996F8A32796F875
:109D2000A2371048FEF7F1F900F09CF9032006F085
:109D300058FB0C4806F0D8FA96F8A81796F8A6270C
:109D400096F8A737074800911549FEF7DEF900F0AD
:109D500089F9042006F045FB024806F0C5FAE7E061
:109D6000081100202116002015CB010828CB01087E
:109D7000E023002091E00108E2270020C01100202C
:109D80002CCB010898200020D42700204C2800204C
:109D900030CB0108F82000203CCB01084DCB010856
:109DA0005ECB01088C200020784B1B681B0640F11D
:109DB000BB80636AA16A764A8B421CBF936292F8A9
:109DC0002C304FF001011CBF013303F003034FF0AF
:109DD000000018BF82F82C3006F00FFB94F82C30EE
:109DE0006C4A0026D05C06F064FA0220012106F0DD
:109DF00004FB694B3620F35C0136C3EBC30393FBD2
:109E0000F0F0C0B2062828BF06206038C0B206F0C5
:109E100050FA102EEDD1614B61491B78614813F067
:109E2000020F614B1A7814BF59234E23FEF76DF9C8
:109E300000F018F9022006F0D4FA5A4806F054FA55
:109E40005A495B4B4E680A68564892FBF3F25949EF
:109E500096FBF3F3FEF759F900F004F9032006F03E
:109E6000C0FA504806F040FA534B54491A884D48FE
:109E7000FEF74BF900F0E3F8042006F0B2FA494887
:109E800006F032FA4E4B4F491A884648FEF73DF924
:109E900000F0D5F804210A2006F0AFFA414806F098
:109EA00023FA4949226B3F48FEF72FF9474E00F04D
:109EB000C6F8052006F095FA3A4806F015FA7268D9
:109EC000B36843493748FEF720F900F0B8F8052198
:109ED0000A2006F092FA334806F006FA3369F2686F
:109EE0003C49D21A2F48FEF710F900F0A8F80620D6
:109EF00006F077FA2B4806F0F7F9B2683649294898
:109F0000FEF703F900F09BF806210A2006F075FA27
:109F1000244806F0E9F93149152222480DF006FEE1
:109F200000F08DF8072015E7F37843F00203F37093
:109F30004DBB2B4B00219B791220032B97BF294A45
:109F40003F259B181D7F06F058FA284606F0B1F908
:109F50001320002106F051FA234B1B78002B14BF6D
:109F60005220212006F0A5F91420002106F045FA20
:109F700094F83450074B585D013505F0030506F0A1
:109F800098F984F8345003B0BDE8F083EC27002042
:109F90001416002070CB010895110020E811002054
:109FA00075CB010821160020EE110020F0110020D1
:109FB0008096980086CB0108EA11002093CB010817
:109FC0004C1100209BCB0108A2CB010828080020DF
:109FD000A9CB0108B2CB0108B9CB01085803002076
:109FE0007030002094AB0108D6270020642928BFD8
:109FF0006421F8B501FB00F5642495FBF4F40646F2
:10A00000E4B20027FBB2A34204D29F2006F051F92C
:10A010000137F7E7B4420BD2142195FBF1F5C4EBFD
:10A020008410663DC4EB80002844C0B206F041F9BC
:10A030000134E4B2B44201D29A20F7E7F8BD08B582
:10A0400007480DF048FDC0B209280246044B04DC65
:10A0500001302021C0B29954F6E700221A5408BDFD
:10A060002116002008B507480DF035FDC0B21428B0
:10A07000044B04D8421C20211954D0B2F7E7002227
:10A080001A5408BD211600202DE9F74F04F08EFD6B
:10A09000A64C804626686568A768861BF643451B64
:10A0A000C71BED43FF43F60FED0FFF0F2EB93FB96E
:10A0B000002D00F08782B9462CE04FF0000929E01E
:10A0C000B14627E003EB8A0BBBF802301A050ED429
:10A0D00013F4805F1DBF964A9BF801101268954AE1
:10A0E000954B14BF52F82120126843F82A20BBF880
:10A0F0000230D80516D499050AD5904B1B7813F079
:10A10000040F0CBF8E4A8F4A8B4B126843F82A20EB
:10A1100009F10109207B5FFA89FA8B4982450B68B6
:10A12000D0D326E0894A5046594606F011FF884BA5
:10A130001B885A0603D550465946864A16E05807EA
:10A1400003D550465946844A10E0190703D55046B6
:10A150005946824A0AE09A0703D550465946804A32
:10A1600004E0DB07D4D5504659467E4A06F0F0FE9F
:10A17000CEE7DFF808E20093BEF906307822A3F5B7
:10A180007A7353434FF47A7293FBF2F3F34603F27C
:10A190002B13019300225FFA82FE864517D2009BA3
:10A1A00003EB820EBEF802E01EF4806F0DD040F289
:10A1B000671ADFF88491019B39F822E09E449EFBE8
:10A1C000FAFC0AFB1CEE29F822E00132E3E74DB36A
:10A1D00008F5C333A0336360637B544A13BB9373A6
:10A1E000614B1B6813F0020F0AD0DFF894E19EF870
:10A1F00000E0BEF1000F03D04FF0010E82F80EE038
:10A20000DA0506D5594B5B791BB1A37B43F00203FA
:10A21000A3734A4B1B7813F0050F02BFA37B43F0D7
:10A220000403A37394F80EE0BEF1000F03D13F4B7B
:10A230005B7B002B4FD094F80DC01CF0010FACF1EC
:10A240000C031DD1BCF1030F07D8DFF8E8901EF016
:10A25000040F3B4A08BF4A4600E0364AACF1040C02
:10A26000BCF1070F05D8DFF81CC11EF0010F18BFA5
:10A270006246DBB2032B0ED81EF0020F3C4B06E009
:10A28000DBB2032B06D82F4B2A4A1EF0020F18BF51
:10A290001A4600E0274A4FF0000C5FFA8CF3834225
:10A2A0000DD20B6803EB8C035B881B0642BFD2F810
:10A2B0000090214B43F82C900CF1010CEDE785B197
:10A2C000BEF1000F08D0637B184A0133DBB2142BB8
:10A2D00006D1002304E025B1637B002BF3D100E01D
:10A2E0005373002E52D0234A3223B2F90250B2F9EE
:10A2F0000020002DB8BF6D42002AB8BF524295FB26
:10A30000F3F592FBF3F2EDB2D3B2AB4238BF2B467A
:10A31000194A13B192FBF3F300E013464344236060
:10A32000E37B024A83BB01232FE000BF4C160020D1
:10A33000D41C002030C40108C20E0020A63000202A
:10A3400098C2010888C20108AC120020B4AB010811
:10A35000A8120020BAAB0108C0AB0108C6AB0108C7
:10A36000CCAB0108D2AB0108EC27002070300020F4
:10A37000A0C20108C8110020400D030028280020B9
:10A3800034120020A8C201080023D3738F4D904BD4
:10A390002D78E27BADB9002F00F00F818D4B267B2D
:10A3A0001A788D4B02F0040293F800C08B4BD2B2A6
:10A3B000D3F800E00B680021894D03EB86060F46B9
:10A3C000B5E01AB9874A1A61002508E0864AFAE71B
:10A3D0000A68AB00D6187688760604D40135EBB24D
:10A3E0008342F5D3D7E7814EB6F90060192E25DDFB
:10A3F00012F803E094F814C00EF00F09E145266945
:10A400000CDCDFF8CCC19CF815C0BCEB1E1FDEBF16
:10A41000D6F800C0DFF8D8E143F80EC012F803E028
:10A4200094F816C00EF00F09E14533DBDFF8A0C148
:10A430009CF815C0BCEB1E1F2CDC26E0193629DA6F
:10A4400012F803E094F814C00EF00F09E1452669F4
:10A450000CDCDFF87CC19CF817C0BCEB1E1FA2BF50
:10A46000D6F800C0DFF888E143F80EC012F803E028
:10A4700094F816C00EF00F09E1450BDBDFF850C170
:10A480009CF817C0BCEB1E1F04DBD6F800E0584E4A
:10A4900043F806E0554EB6F90260192E1BDD12F89E
:10A4A00003C094F814E00CF00F09F14526690CDCA8
:10A4B000DFF81C9199F81590B9EB1C1FDEBFD6F898
:10A4C0000090DFF82CC143F80C90D25C02F00F0C26
:10A4D000F4451EDD82E7193680DA12F803C094F8DD
:10A4E00016E00CF00F09F14526690CDBDFF8E0906F
:10A4F00099F81590B9EB1C1FDEBFD6F80090DFF875
:10A50000F0C043F80C90D25C02F00F0CF445FFF65B
:10A5100065AF94F817E0BEEB121FA2BF3668344A4D
:10A520009E505BE75888000504D404330435B342D9
:10A53000F8D122E04AB101EB0C0A06209AFBF0F9AF
:10A5400000FB19A001280DDC01E057B9012793F8A1
:10A5500001900EEB89003EF829A090F80290C07897
:10A5600003E01746002081468246013125F802ACFF
:10A5700085F800906870C9B2D7E7174A1378013B95
:10A5800013F0FF0308BF06231370124B1B785B0701
:10A5900041BFBBF906304FF47A72A3F57A7303EB2F
:10A5A000C30348BF93FBF2F3124A46BF0133DBB249
:10A5B000012392FBF3F34344A36003B0BDE8F04FE3
:10A5C00005F03CBC03B0BDE8F08F00BFD6270020EB
:10A5D0004C160020A630002044000020D41C00208F
:10A5E000C40E0020A4C2010830C40108C811002014
:10A5F000C20E0020400D0300344B354A1B68126820
:10A6000010B51A60334A11685960516892689960B0
:10A61000DA60314A116819615168926859619A612A
:10A620002E4A1168D9615168926819625A622C4A9F
:10A6300011881985518859859188D2889985DA853C
:10A64000284A118819865188598692889A86264AFE
:10A650001188D986518892881987194621F83A2F8E
:10A66000224A10780022824206DA214C34F8124045
:10A67000013221F8024FF6E71E4A1288A3F864203F
:10A680001D4A1288A3F866201C4A1188A3F86C1092
:10A6900051889288A3F86E10A3F87020184A3B21C5
:10A6A00012689A66174A126892FBF1F2B2F5967F29
:10A6B000C8BF4FF0FF325A67134A1288A3F87820B8
:10A6C000124A5289A3F85E2010BD00BF5424002016
:10A6D00088300020801E00208C1E0020981E002044
:10A6E000C811002008110020B211002018210020FC
:10A6F000241100206C1D00206C0F0020E02300209E
:10A70000BC11002000000020441100200E11002088
:10A7100070B5472007F0A6FB174B1B681B0307D536
:10A72000164B174A5B6810681B68C01A07F0CCFB11
:10A73000144E154C154D307807F0C6FB2368286879
:10A74000C01A07F0D0FB63686868C01A07F0CBFB3B
:10A750000F4B188807F0B8FB0E4B188807F0B4FBB6
:10A760000D4B188807F0B0FB337823742B68A36077
:10A770006B68E36070BD00BFD82500205424002022
:10A7800088300020EE11002040240020F01100202D
:10A79000EC110020EA1100204C1100200A4A138815
:10A7A00001331380094A136801331360084A138880
:10A7B00001339BB2202B01BF00231380054A13886D
:10A7C00008BF013313807047F8250020E0250020E2
:10A7D000E4250020E625002038B53A4B05461B78D5
:10A7E0000C46083B012B6BD8452007F03BFB284665
:10A7F00007F038FB0C2D23D004D80A2D0AD014D82A
:10A8000035B138BD0E2D4BD02ED3FF2D50D038BDD5
:10A81000206849E0207807F025FB62796378002AF8
:10A8200014BF80200020184300E0207807F01AFBB6
:10A83000A07807F017FBE07807F014FB20793BE0E5
:10A84000B4F9000007F036FBA07807F00BFBE078C6
:10A8500007F008FBB4F9040007F02CFBB4F906007C
:10A86000BDE8384007F026BB637820788BB180F0D4
:10A87000800007F0F7FAA468E0B207F0F3FAC4F337
:10A88000072007F0EFFAC4F3074007F0EBFA200EB9
:10A8900012E007F0E7FA6068BDE8384007F023BB34
:10A8A000206807F011FB6068BDE8384007F00CBB7A
:10A8B000054807F05BFA0020BDE8384007F0D2BA3F
:10A8C00038BD00BF30240020F2CB01082DE9F04F45
:10A8D000BF4B8BB018880193002840F0A380BD4E79
:10A8E000FEF7E4FDFFF788FE34684920254607F0AF
:10A8F000B9FAB94B04F11C08186807F0E5FA55F8E5
:10A90000040B07F0E1FA284607F04AFC04F11000B6
:10A9100007F046FC1027B14D01232A68BB401342C3
:10A9200003D0D8F8000007F0DEFA0137132F08F142
:10A930000408F0D1AA4F04F1280007F021FCB7F871
:10A940004431B4F92E00B846C01A07F0BDFA2B689E
:10A9500013F4805F08D0A34BB4F864001B88181A66
:10A96000C0F30D0007F0B0FA2B68990403D5B4F8D2
:10A97000660007F0A9FA2B685A0503D504F16C00AC
:10A9800007F0FEFB2B681B0502D5A06E07F0ABFAA3
:10A990002B685F0402D5606F07F0A5FA2B681804D6
:10A9A00003D5B4F8780007F08FFA274604F1300099
:10A9B00007F0E6FB04F1360007F0E2FBB8F844319B
:10A9C00037F93C0F4FF00108C01A07F07DFA864BAB
:10A9D0001B78984509DA37F9020FB4F93C3008F1D1
:10A9E0000108C01A07F07FFAF1E72B68990505D531
:10A9F000B4F95E00A0F2DC5007F075FA32687B48CB
:10AA00007260B260121A9110794A4A43531C0322B1
:10AA100093FBF2F202EB42029A1A7C2303FB02033D
:10AA2000336068E2734B744A1B6811688B4206D02E
:10AA30000AA941F8203D00201360FFF7CDFE684AC7
:10AA4000019B92F8C6171B8892F8C7070B44013B7D
:10AA5000B3FBF0F200FB12338B4280F017825D4FA4
:10AA60000120FEF723FDFFF7C7FD50203E687D68FB
:10AA700007F0F8F9BA683B6810681B687A68034405
:10AA80001068A3EB400007F02EFA6A68736802A80A
:10AA90009B1A0293AA68B3689B1A0393EA68F36847
:10AAA0009B1A049307F07CFB2A6933699B1A029373
:10AAB0006A6973699B1A0393B369AA699B1A049321
:10AAC0000023194602AA52F8212002F120003F2853
:10AAD00042D802F108000F2806D80232032A04D90E
:10AAE000002B08BF012300E0022301310329E9D133
:10AAF000012B02980ED0022B21D0039B00F0030003
:10AB000003F003039B0043EA0010049B03F00303DC
:10AB100018430CE000F00F0040F0400007F0A2F9ED
:10AB20000498039B00F00F0040EA0310C0B207F046
:10AB300099F906F11C0B05F11C0810246FE000F0D8
:10AB40003F0040F0800007F08DF99DF80C0007F001
:10AB500089F99DF81000EAE702224FF0000802ABE5
:10AB600053F822304FEA880803F18001FF2910D9F9
:10AB700003F50041B1F5803F02D248F0010808E03A
:10AB800003F50003B3F1807F34BF48F0020848F0BA
:10AB9000030812F1FF32E2D268F03F00C0B207F0C2
:10ABA00061F902AC0DF1140A08F00303022B2078BE
:10ABB00007D0032B22D0012B29D107F053F960785D
:10ABC00025E007F04FF9607807F04CF9A0781EE017
:10ABD000E425002054240020E0250020D825002072
:10ABE0004C280020D42500201821002060240020BB
:10ABF000DF7BEFBDEC250020E825002007F032F9CF
:10AC0000607807F02FF9A07807F02CF9E078043489
:10AC100007F028F954454FEAA808C5D189E7B84993
:10AC200001220B68A2401A428A4606D0DBF80000D7
:10AC3000D8F80030C01A07F056F90134132C0BF184
:10AC4000040B08F10408EAD106F1260005F12601FB
:10AC5000002331F9024F30F9022F121B02AC44F8E5
:10AC600023200133042BF4D103214FF000094FEAD4
:10AC700089035FFA83F902AB53F821206AB102F12C
:10AC800008000F2802D849F0010906E08032FF2AA7
:10AC900094BF49F0020949F0030911F1FF31E6D2EE
:10ACA0004846002407F0DEF8A0460DF1080B09F035
:10ACB0000302022A16D0032A1DD0012A38D1B8F186
:10ACC000000F05D1DBF8004090462401E4B22FE0EC
:10ACD000DBF800004FF0000800F00F00204307F001
:10ACE000C1F825E0B8F1000F0CD0DBF80000C0F38C
:10ACF0000310204316E0B8F1000F08D19BF80100C3
:10AD000007F0B0F89BF8000007F0ACF810E0DBF8B3
:10AD10000000C0F30330204307F0A4F8DBF8000084
:10AD2000C0F3071007F09EF8DBF800402401E4B2FE
:10AD30000BF1040B06AB9B454FEA9909B7D1B8F16B
:10AD4000010F02D1204607F08DF8DAF8003013F435
:10AD500080541FBFB6F86420B5F864100124521A5D
:10AD600018BF02929A040AD50AAA02EB8401B5F828
:10AD70006600B6F866200134121A41F8202C5805F6
:10AD800013D502AA02EB840C06F16A0E05F16A00E3
:10AD900000223EF9021F30F9028FC8EB01014CF886
:10ADA00022100132032AF4D10334190508D50AAA66
:10ADB00002EB8400A96EB26E0134521A40F8202CC6
:10ADC0005A0408D50AAA02EB8400696F726F013435
:10ADD000521A40F8202C18040BD50AAB03EB84025E
:10ADE000B5F87810B6F8783001345B1A42F8203C98
:10ADF00000E0FCB1012C03D1029807F074F819E0CF
:10AE0000631E002002AA52F823204000C0B20AB1FB
:10AE100040F00100013BF5D507F024F84FF00008A1
:10AE200002AB53F8280008B107F05DF808F10108FB
:10AE3000A045F5DB30200321FEF778FB3620032107
:10AE4000FEF774FB2F4B3C201978FEF76FFBDAF806
:10AE50000030990506D5B6F95E00B5F95E30C01A26
:10AE600007F041F83A6828487B687A60121A911016
:10AE7000264ABB604A43531C032293FBF2F202EBC7
:10AE800042029A1A7C2303FB02033B60204B1B689F
:10AE90001A0630D51F4C204D22682B689A420BD1E0
:10AEA00062686B689A4207D1019B1B88102B11D1F5
:10AEB0001A4B1B885B060DD1482006F0D3FF206893
:10AEC00007F011F8606807F00EF823682B606368DC
:10AED0006B600EE0124A104B11782A7C914208D127
:10AEE000104A99681068884203D15268DB689A4218
:10AEF00001D0FFF70DFC06F027FF0BB0BDE8F08F87
:10AF0000D82500201821002060240020DF7BEFBD21
:10AF1000EC2700205011002040240020E6250020CE
:10AF2000EE110020F01100202DE9F84F0C9EC2EB2D
:10AF3000030B394C0B9B002914BF4FF0060A4FF04E
:10AF4000040AF61A636805460133904613D1236854
:10AF500053455ED2314A032B98BF294652F823202D
:10AF60002F4806F06DFF63680022013363602D4BAC
:10AF700005461A7013E0002511E02B4A127895421D
:10AF800040DA0B9BE3B109FB06F2995C01228A408F
:10AF9000264909680A4213D1636801336360D4F813
:10AFA00004900A9B1C4F9945E7DB2BD10A2006F041
:10AFB00059FF3B6801333B604FF0FF337B6021E07A
:10AFC000184A117821B12C2006F04CFF013501E020
:10AFD0000121117009FB0BF3226808EB030752B93A
:10AFE00058F8030006F0C2FE97F9041005444B1C04
:10AFF000D2D00F4802E03A440E48117906F020FF03
:10B000000544C9E7206850452CBF00200120BDE859
:10B01000F88F0020BDE8F88FF0250020D8AB01089C
:10B02000FDCB01086416002008010020D82500206F
:10B030000CCC01089FCB010810B508F03FFF0021A0
:10B04000044609F04BF908B1204601E004F1004044
:10B05000054909F03BF8054908F084FFFDF70CF9B4
:10B06000034B186010BD00BF8096184B35FA8E3C1C
:10B070006C000020F8B59C4B04461B68187818B18A
:10B08000012800F06A819AE2242C984D0CD006D851
:10B090000A2C00F0D9800D2C00F0D68048E12A2C33
:10B0A00006D02C2C04D043E128706870A87050E1C1
:10B0B0008F4B69782F7800208C4A58542FBB197811
:10B0C000D770472921D1597850291ED1997847291D
:10B0D00007D1D978472904D11979412901D1012112
:10B0E000D1709978824A522903D1D1784D2900F044
:10B0F000688299787E4A472907D1D178532904D1AB
:10B100001279562A04BF0322EA70EA78774E022A9F
:10B1100039D0032A4CD0012A40F08580BA1E072A74
:10B1200000F28180DFE802F004080F131A257F2A5D
:10B1300008F04AF8686076E01B78532B73D16B688F
:10B140005B426B606FE008F03FF8A8606BE01B7833
:10B15000572B68D1AB685B42AB6064E01B78302B47
:10B16000644B1A788CBF42F0020222F002021A707D
:10B1700059E0002008F088F8287354E0002008F017
:10B1800083F8E8814FE0072F06D0082F4BD101202C
:10B1900008F07AF8708246E0012008F075F841F274
:10B1A000184358434FF47A73B0FBF3F030823AE01F
:10B1B000022F07D0032F0AD1002008F065F84E4B6C
:10B1C000187030E0002008F05FF830752BE02AD9C5
:10B1D0003A1F9210337D0132D2B2013B02EB83035E
:10B1E000DBB2102B1FD8F91EC2F1010201EB820263
:10B1F000D2B2012A0BD0042A11D100205E1E08F021
:10B2000043F83E4B002298553D4B9A5507E03D4A86
:10B210005E1E0020935508F037F83B4B98553B4A8B
:10B22000136801331360314B2A2C18BF9A7807F149
:10B2300001074FF000000CBF012254402F706870CE
:10B240000CBF5A759C7084E0687D002848D0304B54
:10B2500013F8012D2F495A708B42F9D1244A234CFF
:10B2600013785278402B85BF373B1B011B01DBB2A3
:10B2700098BF03F0F003402A8CBF373A303AD2B27D
:10B280001344AA78DBB29A4227D121230B702249BA
:10B29000E0780B68012803F101031E4A0B600AD015
:10B2A00002281CD172231370228A1C4B1A80628AD6
:10B2B0001B4B1A8013E0672313700E4B1B789F07FC
:10B2C0000ED5184B62681A60A2685A60227B164B32
:10B2D0001A70E289154B1A8002E03F230B700020A0
:10B2E00000236B7535E000BF480800206816002079
:10B2F00018280020E811002064110020951100207A
:10B3000085110020651100207511002038160020DD
:10B310006C0300205803002044160020EA1100208E
:10B320004C110020F0110020EE110020EC11002043
:10B330006B78687D0E2B9FBFA54A591C5170A54A9A
:10B3400098BFD454A24A18B993785C40947000E036
:10B350000020003018BF0120F8BD9D4B0022997DD0
:10B36000082900F22C81DFE801F0050B0F15202BD6
:10B37000475D6700B52C40F02281DA75012239E083
:10B38000622C08BF022235E003229A751C765C7697
:10B390009C7614E104229A755A7E997E2244D2B298
:10B3A0005A760A449A76DC7609E105229A755A7E25
:10B3B000997E2244D2B25A760A449A769C83FEE061
:10B3C00006229A755A7E997E2244D2B25A760A444F
:10B3D0009A769A8B02EB0424A4B2B4F5AC7F82BFB8
:10B3E0007B4A0121D17500229C83DA83002C40F036
:10B3F000E68007229A75E2E05A7E997E2244D2B214
:10B400005A760A449A76DA8BB2F5AC7F3EBF704921
:10B41000891881F820400132998B92B29142DA83E7
:10B42000E7D9CCE008229A755B7EA34200F0C78082
:10B43000674B0122DA750DE0674D9A7515F8012DFD
:10B440006A70664A9542F9D1997E614AA14206D056
:10B450003F232B70624A536801335360AFE0614869
:10B46000016801310160D07D10B13E232B70A6E050
:10B4700021212970D17E062941D004D8022907D084
:10B48000032923D0F8BD122959D0302967D0F8BD3F
:10B490005021546A297054494C60946A0C60116BB5
:10B4A0004FF47A7491FBF4F1504C218092F87811AA
:10B4B0004F4A19B1117841F0020102E0117821F0F0
:10B4C00002011170012283F8792169E0532129706A
:10B4D00092F82510CE0705D592F82420D51E6A4291
:10B4E0006A4100E0024602F0010183F87811002A67
:10B4F00056D13F490A7822F002020A7050E04F21EB
:10B50000297092F82B10CC0705D592F82A20D11E6D
:10B510004A424A4100E0024602F0010183F87811F4
:10B5200022B933490A7822F002020A7093F84F10C8
:10B53000304A1170B3F84C102F4A118030E0562178
:10B54000546B29702D490C8042F21074916B91FB61
:10B55000F4F12B4C2180012182F87A1120E049215D
:10B56000297092F82410274A102988BF10211170E1
:10B57000254914780022A2420ED20E7A234D565548
:10B580004E7A234D5655CE7A224D565511F80C6FF2
:10B59000214D56550132EEE720490A6801320A6012
:10B5A00093F879310A4A002B3AD092F87A31BBB33A
:10B5B000002182F8791182F87A111846F8BD00202E
:10B5C000F8BD1279432A7FF494AD0222EA7090E527
:10B5D00068160020182800206C0300205803002063
:10B5E0002808002044160020F0110020EC11002053
:10B5F000E8110020EE110020FA000020EA110020DE
:10B600004C110020641100208816002065110020D4
:10B61000751100208511002095110020381600209A
:10B62000F8BD0449044B0968002218705A619961F9
:10B630001A7770471028002028080020F8B5101A43
:10B640000D461F4608F03AFC0446781B08F036FC0D
:10B65000174B079E196808F085FC214605462046D1
:10B6600008F080FC29460746284608F07BFC014686
:10B67000384608F06FFB0CF05BFE0E4908F072FCD8
:10B6800008F05CFE069B2946186004F100400CF0AF
:10B69000C3FC094908F066FC084908F05BFB08F0A8
:10B6A00027FE0028BCBF00F50C40A0303060F8BD7C
:10B6B0006C0000202C7D8E3FA00CB34500A00C46F2
:10B6C00044F25063984203DDA0F50C40A038704767
:10B6D000034B9842BCBF00F50C40A030704700BF40
:10B6E000B0B9FFFFF7B50368174C184D23600B681E
:10B6F000174E63600068FFF79FFC95E80300154B49
:10B700000196009394E80C00FFF798FF3668124BFF
:10B7100060681E606B68114FC01A08F0CFFB104BB9
:10B72000196808F01FFC08F0E3FD2A6823687860B8
:10B730009B1A3B600B4B1E600B4B1B68DA880B4B54
:10B740001A8003B0F0BD00BFEC210020F0110020F2
:10B75000F8210020F421002034220020FC210020C8
:10B760006C0000202C220020001000202822002045
:10B7700070B50446407908F09DFB1E4908F0A6FC10
:10B780001D4D1E4E2860E07B08F094FB194908F01F
:10B790009DFCEE606860A07908F08CFB184908F009
:10B7A00095FC184D2860207C08F084FB114908F0B6
:10B7B0008DFC6860A07E08F07DFB134908F086FCD4
:10B7C000EE60A860E07908F075FB0D4908F07EFC9A
:10B7D0000E4D2860607C08F06DFB064908F076FC91
:10B7E0006860E07E08F066FB074908F06FFCEE60D9
:10B7F000A86070BD0000C842042200200000FA4486
:10B80000000020411422002000007A443822002049
:10B8100010B50C4C23789B0713D50B4B1B78042BCE
:10B820000FD90A4A0A4B1068526818605A60FFF72D
:10B8300003FC084B1A88084B1A80237843F0010355
:10B84000237010BDE8110020EE110020F01100203F
:10B8500050110020C011002048220020164B13B5C3
:10B860001B681B0325D5154B154C1B7815498DF806
:10B870000030154B20681B788DF8013008F072FB02
:10B8800008F05CFD11498DF80200606808F06AFB61
:10B8900008F054FD8DF80300A06808F04FFD0C4B34
:10B8A0008DF804001B780A2069468DF80530FEF7F4
:10B8B00093FF02B010BD00BFEC270020DC27002062
:10B8C0000028002000002041FC27002000007A44CE
:10B8D000E0270020054A137883F001031370044A1F
:10B8E00000231360034A1360B8E700BFE02700207D
:10B8F000F8270020F4270020094A1378184413463B
:10B90000C0B210F0800F18BF80381070054A197847
:10B910001378994201BF00231370014A13707047D6
:10B920004D2200204C22002010B50A4B0A4A1B78F9
:10B9300042609C18094A046012789A4225BFD31AC3
:10B940000B60C3F1800300232EBF4B600B604A6085
:10B9500010BD00BF4D2200204E2200204C220020AE
:10B960001FB5684602A9FFF7DFFF044B02981B686A
:10B9700003440398184405B05DF804FBC406002096
:10B980002DE9F04F814689B0029300230391049280
:10B990000193049A934207DA039A019952F82320FB
:10B9A000013311440191F4E7029B019D002B57D113
:10B9B00004F018FC002853D102987FE00222414E87
:10B9C0008DF81C201A0C4FF480578DF81D2006208E
:10B9D0001A0A8DF81E208DF81F3004F02BFC7761B9
:10B9E00006213948F9F7EEFC384B01223761C84689
:10B9F0001A70776126463448002107AA0423F9F714
:10BA0000B3FC039F4FF0000A049B9A451DDABC4625
:10BA100057F8043B4FEA8A0B002B48D0B34235D38A
:10BA200033462948002159F80B20CDF814C0F9F706
:10BA30009BFC59F80B30DDF814C0334449F80B3047
:10BA4000DCF800309E1BCCF800601E4B4FF4805297
:10BA50001A611F4A2D1B13681C44029B14605BB3C0
:10BA600055B31B4B1B68DCB22A19B2F5807F194A0B
:10BA700088BFC4F58074D26898BF2C4693429DD38A
:10BA8000154A00231370154A137015E0D8F80020EA
:10BA90000D480021F9F768FC57F8043CD8F800205D
:10BAA000F61A1344C8F80030002347F8043C0AF1A2
:10BAB000010A08F10408A7E7019B581B09B0BDE87B
:10BAC000F08F00BF000C014000380040C10600208C
:10BAD000C40600200C0000204C2200204D22002033
:10BAE00030B50B4C0B4D22782B7885B09A420CD098
:10BAF000684602A9FFF718FF0123684602A902223F
:10BB0000FFF73EFF00232B70237005B030BD00BF50
:10BB10004D2200204C22002030B50E4D0E4C2A78CC
:10BB2000237885B09A4211D0684602A9FFF7FCFE3F
:10BB3000002302A902226846FFF722FFFFF7DCFE7E
:10BB400020782B781B1A5842584100E0012005B09C
:10BB500030BD00BF4D2200204C22002070B50F4C9C
:10BB60000F4E4FF4805545F2082004F063FB062188
:10BB700065613046F9F726FC0A4B01222561304603
:10BB80001A70C7216561F9F71DFC074A002325617A
:10BB90001370064A1370064A136070BD000C014012
:10BBA00000380040C10600204C2200204D22002019
:10BBB000C40600200148024900F0E4B80008004033
:10BBC000C41F00200148024900F0DCB80004004016
:10BBD0009C1F00204FF08040014900F0D3B800BF07
:10BBE000741F00200148024900F0CCB8002C01402D
:10BBF0004C1F00200148024900F0C4B8002C01404D
:10BC00004C1F0020026D70B515880446ADB2A90620
:10BC100013D5036B8BB9C36A1BB1908880B2984768
:10BC20000BE0E169928840694E1CD2B2E661425451
:10BC3000E169E268914228BFE3612B0613D5636A8C
:10BC4000A26A9A42236D0AD0511CA069A162825C4B
:10BC50009A802369994206D30023A36270BDDA68F3
:10BC600022F08002DA6070BD026B0346C16810B535
:10BC7000406942B11A6C8C1A013A08BF0A46005D4D
:10BC80001A64C0B210BD1A6A805C01328A4228BFB1
:10BC90000022C0B21A6210BD436B13B190F8440089
:10BCA0007047836A406A1B1A584258417047036BB9
:10BCB00013B15B68016C01E0C369016A8B423CBF50
:10BCC000C2689B18581AC0B27047836A8169426B78
:10BCD0001944D160416A994297BF0169CB1ACB1AC6
:10BCE000536096BF0023536083624FF0000380F8D7
:10BCF0004430136888BF816243F0010313607047CA
:10BD0000436A8269D154436A02690133934228BF6E
:10BD100000234362436B1BB11B68DB0705D4D4E7E8
:10BD2000026DD36843F08003D360704738B50D4B84
:10BD30000D4D99680D4B1A681C465288114203D06C
:10BD400002F034FF286007E002F030FF2B689842D1
:10BD500082BFC01A064B186023685A68054B5A61A7
:10BD600038BD00BF000C0140E4170020240800206B
:10BD700000000020000401404171FDF70FB8816010
:10BD8000FDF70CB82DE9F04105460E46078A838978
:10BD90009BB21F40002F37D0B7FA87F24FF0004315
:10BDA000D340DB4399B21F40A2F11B032982042B2D
:10BDB000F0D8DFE803F0221F1C190300746A24B1D5
:10BDC000013C0023A4B2736201E0AC8DA4B2D6F8AA
:10BDD0002080B8F1000FDDD0D8F800304046214671
:10BDE0009847D8F80480F4E73068A98E08E07068B6
:10BDF000298F05E0B068A98F02E0F068B5F840101F
:10BE0000036889B29847C5E7BDE8F081254B10B5B6
:10BE10005A43254B254C1B680139B3FBF2F20388CA
:10BE2000013AA04289B292B29BB212D004F50064EA
:10BE3000A0420ED0B0F1804F0BD0A4F59834A042B0
:10BE400007D004F58064A04203D004F58064A042CA
:10BE500002D123F070039BB2154CA04206D004F52A
:10BE60008064A0421CBF23F440739BB203800F4B3D
:10BE70008185984202850FD003F5006398420BD06C
:10BE800003F54063984207D003F58063984203D0DE
:10BE900003F58063984201D1002303860123838246
:10BEA00010BD00BF40420F0004010020002C0140E3
:10BEB0000010004073B505460068FFF7A7FF2A6829
:10BEC0000124138800269BB243F001031380EB7A10
:10BED00001A88DF804308DF805408DF806608DF8C6
:10BEE000074006F0B1FFEB7A1B2B0BD1192301A8F9
:10BEF0008DF804308DF805408DF806608DF8074008
:10BF000006F0A2FF02B070BD0C4B800A98420CD024
:10BF100004D8B0F5801F0CD101207047084B98421F
:10BF200005D04933984206D003E002207047032031
:10BF30007047FE2070470020704700BF01001000CE
:10BF4000020010002DE9F8430468074620468846A1
:10BF50009146FFF7D9FF03284BD8BA7A9108B8F178
:10BF6000000F06D1A589AEB202258D4026EA05054F
:10BF7000A5810A2303FB00131F4A42F823800433E0
:10BF800042F82390B8F1000F07D0BD7AA189AD081F
:10BF90000223AB400B439BB2A3812823434303F10D
:10BFA00020011144EFF31286502585F3128803F126
:10BFB0000C051C331544134455F8047F17B10F606A
:10BFC000296804319D42F7D100230B60F3B283F35B
:10BFD0001188282303FB0020036A23B1A3899BB2A5
:10BFE00043F0010304E0A38923F001031B041B0CAD
:10BFF000A381BDE8F88300BF4C1F002096E695E6BC
:10C0000094E60148FEE500BFE81700200048F9E586
:10C010003C1800200B4B4FF400525A604FF6FE7351
:10C020000948D0F88C2011680B401360C26FD0F81B
:10C0300080309A4201D0583047E6012380F89C3086
:10C04000704700BF00000240E41700202DE9F043D4
:10C050001E469C4B8DB09842894690469DF8507084
:10C060005ED1994B994AC3F860809A6503F1AC029E
:10C07000DA6603F5D6721A674FF480725A669A66CA
:10C08000934AC3F8A800C3F88C20A2F54842403A6E
:10C09000C3F8A0208F4B9A6942F480429A615A6992
:10C0A00042F001025A6102238DF803303A074FF43F
:10C0B0000073ADF8003001D51C230FE0B30706D59F
:10C0C0001823854869468DF8023003F095FFF5077F
:10C0D0000AD54FF48063ADF8003048237E486946A6
:10C0E0008DF8023003F088FF01240E23002501A8FB
:10C0F0008DF804308DF805408DF807408DF8065016
:10C1000006F0A2FE252301A88DF805408DF8074012
:10C110008DF804308DF80650704C06F095FE50E016
:10C120006F4B984240F0C980674B684AC3F80C8057
:10C130005A6003F52B729A6103F56B72DA614FF462
:10C1400080721A615A61674A5865DA641A65614BF0
:10C150003C07DA6942F48022DA619A6942F0080207
:10C160009A614FF002038DF803304FF48063ADF80D
:10C17000003001D51C230FE0B00706D518235A481C
:10C1800069468DF8023003F037FFF1070AD54FF406
:10C190000063ADF800304823534869468DF80230FB
:10C1A00003F02AFF27238DF804300022012301A881
:10C1B0008DF805308DF806208DF8073006F044FE26
:10C1C0004A4C0025012384F844302562E561A562CC
:10C1D0006562C4F82C906671C4F80880A771204687
:10C1E000FCF7DCFDF20731D5206B002826D0E36C8C
:10C1F000039501934FF480530A9380230693E368D9
:10C200000595049320230993636907950293089584
:10C210000B9501F065F801A9206B01F043F8226B42
:10C22000216D136843F0010313608B8A9BB243F0C6
:10C2300040038B8253689BB2236407E04FF6DF72A2
:10C24000236D1A80DA6842F02002DA60B3072CD539
:10C25000606B28B3A36C002501934FF480530A93BD
:10C260008023069323690295049310230393059575
:10C270000795089509950B9501F032F8606B01A9B7
:10C2800001F010F8636B1A6842F002021A60226D26
:10C290005D605D60938A9BB243F08003938204E00B
:10C2A000226DD36843F08003D360226D20469389CA
:10C2B0009BB243F40053938100E000200DB0BDE831
:10C2C000F08300BF00380140E4170020F0AB010804
:10C2D0004400024000100240000801403C180020C9
:10C2E0000048004004480040000C0140E8170020CE
:10C2F00038B500240B4D6059254404F083FB696870
:10C3000011B10948FBF716FFA96811B10748FBF7FF
:10C3100011FF0748103404F075FBB4F5F07FE9D144
:10C3200038BD00BF08AC010830CC010836CC01088C
:10C3300069D6010870B5054628460BF0CCFB0646C9
:10C3400058B91A4B1A485A791A4BBDE8704003EB9A
:10C350008203D3F8DC11FBF7EDBE284616493246BE
:10C360000BF0C2FB60B9154804F04CFB144C54F8B8
:10C37000041F19B11348FBF7DDFEF8E7124805E08A
:10C380000024124B53F8241021B91148BDE8704025
:10C3900004F038BB284632460BF0A6FB01340028D7
:10C3A000EFD1024B0B4D5C71C6E700BF4C2800205B
:10C3B0003CCC010808AC010848CC01084DCC010870
:10C3C000E4AD010860CC010869D60108E8AD0108B8
:10C3D0000ECA010864C70108F0B585B004460BF029
:10C3E0007AFB082826D1621EE01D1F4912F8013F82
:10C3F00009681944497801F00301022908BF203B6C
:10C4000082421370F1D1254604F1080715F8016B3B
:10C41000164831460BF051FB20B1284631460BF04F
:10C420004CFB10B1FAF776FE1CE0BD42EED120467F
:10C4300005F030FF0E4804F0E5FA00230D4A04A988
:10C440001A4492F888210A440849595C0133082BA0
:10C4500002F80C1CF2D10023074801A98DF80C301A
:10C46000FBF768FE05B0F0BD0C010020B4E0010848
:10C4700064CC01084C2800200DD50108264B274C20
:10C480001D6880B52068FBF78BFA2846FBF788FA11
:10C49000206841798A0703D441F0020102F04AFC86
:10C4A0001F4B08221A611F4B1A681F4612F4003FE7
:10C4B0001FBF06236371E37923F001031CBF43F020
:10C4C0000203E371206802F041FC90B1144E08238E
:10C4D0007361124B186802F036FC8046FEF7CAFD05
:10C4E00008B104F0FFFD2846414602F032FC082363
:10C4F0003361284602F02AFC38B12846266802F04B
:10C5000022FC0146304602F024FC3B689B03D9D54F
:10C51000FDF7CEF9D6E700BF14210020901C0020C3
:10C52000000C0140EC2700202DE9F04705460BF0F8
:10C53000D2FA2F4E0446D6F8088090B92D4804F060
:10C5400061FA2D4B53F8241049B10123A34013EA9B
:10C55000080F02D02948FBF7EDFD0134F1E7284828
:10C5600022E02846274922460BF0BEFA58B9264851
:10C5700004F048FA254C54F8041F0029EFD01F4856
:10C58000FBF7D8FDF7E72B784FF000092D2B03BF01
:10C59000013504F1FF344FF0010A4FF0000A164B49
:10C5A00053F8297027B91A48BDE8F04704F02ABAB1
:10C5B0002846394622460BF097FAA8B9012000FA1E
:10C5C00009F0BAF1000F03D0FBF748FF114803E070
:10C5D00040EA0800B060104804F014FA3946BDE89B
:10C5E000F0470E48FBF7A6BD09F10109D7E700BFE8
:10C5F0004C2800206ACC010850AE010860CC01082C
:10C6000069D6010848CC010874CC01084CAE010879
:10C610000ECA010880CC010889CC01080CD501089C
:10C6200010B5084804F0EEF9074B00241C741C6494
:10C63000064B1C7002F032FD04F058FC044B1C60E9
:10C6400010BD00BF91CC0108901C0020A730002035
:10C650001421002070B5064600240A4BE518AA886C
:10C6600016420AD0E1580848FBF764FD284600212D
:10C6700004F059F9054804F0C5F91434B4F5486FCD
:10C68000EBD170BDF8B40108BDCC010869D6010832
:10C6900008B50848FBF74EFDFFF760FA03F0A2FD6E
:10C6A00018B9642002F0A7FAF8E70348BDE808408B
:10C6B000FBF740BDC7CC0108D4CC01082DE9FF41F0
:10C6C0000A48068885684488B0F80480C768FFF780
:10C6D00047F9CDF800800290019731462A4623465B
:10C6E0000348FBF727FD04B0BDE8F0810C000020F3
:10C6F000DCCC0108F0B504788BB005460CB1002401
:10C7000036E04A4B19680E2303FB0411B1F91D51A1
:10C71000B1F91921B1F91B31009591F8205101F5BA
:10C720008C70019591F8215101F59071029590F965
:10C730000700039091F902103D480491214601340D
:10C74000FBF7F8FC082CDCD16DE02D2B14D1072C65
:10C750001BDC28460BF014FA0AAB661C03EB4404FE
:10C7600024F8100C15F8013F303B092BFAD9344658
:10C770002B78002BE9D104E0A3F13002092A09D873
:10C78000E5E7082CBDF8182009D00BB0BDE8F04053
:10C79000FAF7C0BC202BF8D101352646E7E7072A77
:10C7A000F3D840F2DC55BDF81A00204BA0F2EE2180
:10C7B00089B2A9421B68E8D8BDF81C10A1F2EE248A
:10C7C000A4B2AC42E1D8BDF81E7004B23EB2A6429B
:10C7D000DBDB0DB2AE42D8DCA542D6DBBDF924408E
:10C7E000642CD2D1BDF8266034B2112CCDDCBDF85A
:10C7F0002050B42DC9D8BDF82240B42CC5D812B2EF
:10C800004FF00E0E0EFB0233A3F81B116421A3F8A8
:10C810001901A3F81D7183F8205183F8214183F891
:10C820001F1183F822610BB0F0BD00BF2011002062
:10C8300039CD0108F0B504468FB020460BF04BF916
:10C84000C5B21DBBAB4804F0DDF8AB4C94F8D61074
:10C8500009B9AA4853E049B294F8D42094F8D530E5
:10C86000009194F8D710A648019194F9D810073494
:10C87000029194F9D210039194F8D31004912946AF
:10C880000135FBF757FC102DE0D1E2E720469D492A
:10C8900005220BF029F90546B8B929469A487022B5
:10C8A0000BF0D5F82846994B19680E2303FB0013AB
:10C8B00001300022082883F8232183F8242183F8FB
:10C8C000252183F82621F0D112E120469049042247
:10C8D0000BF00AF905462046002D4AD120210BF025
:10C8E000ECF8002800F00481461C30460BF0F3F809
:10C8F0002C460746874B53F824502DB986480FB075
:10C90000BDE8F040FBF716BC30462946FAB20BF002
:10C91000EBF801340028EDD1774A164602F1700198
:10C92000002382F8DA3082F8D63082F8D53082F8E7
:10C93000D43007328A42F3D1784901EBC40191F82F
:10C94000A022934210DAD1F8A472C3EBC302B0184C
:10C950003A44176800F1D401C0F8D47090880133CC
:10C96000888092798A71E7E729466D48FBF7E2FBF8
:10C970008FE06C4907220BF0B7F805462046002DE2
:10C9800049D120210BF099F806460BF0A4F8C4B267
:10C990006CBB6548FBF7CEFB214664480134FBF7CE
:10C9A000C9FB0E2CF8D15548FBF7C4FB00246048A6
:10C9B0002146FBF7BFFB0025544A012311680E22D4
:10C9C00002FB0412D2F82321AB401342594B5A49BF
:10C9D0005A4808BF19460135FBF7ACFB0E2DEBD1C9
:10C9E00046480134FBF7A6FB082CE0D180E0304636
:10C9F00053490BF0C9F82C4600284CD0022C4FD0DC
:10CA00000BF0BEF806AB43F824004D4900200BF0B4
:10CA1000BBF80134F0E74A490BF0B6F8002460B1E6
:10CA2000082C38D00BF0ACF806AB43F8240044498E
:10CA300000200BF0A9F80134F1E7082C2BD1069B5C
:10CA40000F2B28D8DDF81CE0BEF1070F23D8089F74
:10CA50000D2F20D8099E06F16402C82A1BD80A9D12
:10CA6000FF2D18D80B98642815D80C99642912D872
:10CA7000884210DA0D9C032C0DD8324AC3EBC30355
:10CA8000134483F804E05F719E71DD71187259726E
:10CA90009C722D4CD1E60FB0BDE8F040FAF73ABBDE
:10CAA000069B072B20D807990D291DD80278722ADA
:10CAB0000DD06E2A18D1154A0E20126800FB0323F0
:10CAC00001228A40D3F8231121EA020209E00F4A29
:10CAD0000E20126800FB032301228A40D3F82311A1
:10CAE0000A43C3F8232101E0FAF714FB0D4CA4E636
:10CAF0000FB0F0BD61CD01084C28002069D60108B7
:10CB00008CCD0108DEC90108202900202011002059
:10CB100009CA0108E8AD01080ECA010808AC0108FD
:10CB20001DCA010859CD01083ACC0108A8CD010859
:10CB30009FCB01089ED90108E4D80108ADCD0108BA
:10CB4000B1CD01081C29002064C701082DE9F74375
:10CB5000047805468CB9324D95F89B12B5F89822A9
:10CB600095F89A322F48009121460134FBF7E2FAFA
:10CB7000102C05F10405EFD14FE00BF001F80F2860
:10CB8000044636DC284620210AF097FF264EE4B200
:10CB9000D6F84480451CA400002728460AF0F0FF80
:10CBA0005FFA87F9B9F1010F83B208D0B9F1020F2A
:10CBB0000BD0B3F5B47F25D2726C13530AE0FF2B70
:10CBC00020D8736C2344987004E0FF2B1AD8736C40
:10CBD0002344D87028462C210AF06FFF054608B17F
:10CBE000013502E0B9F1020F0CD10137032FD4D186
:10CBF00013E00E480E4900220F2303B0BDE8F043B6
:10CC0000FBF798BA08EB0400002104220AF01FFF8A
:10CC100003B0BDE8F043FAF77DBA03B0BDE8F08396
:10CC20004C280020B3CD0108901C00207DC90108CC
:10CC30009CC901082DE9F04FAC498BB004460AF0BD
:10CC40000FFFAB49002820460CBF012507250AF03D
:10CC500007FFA8490028204608BF02250AF000FF68
:10CC6000002808BF0425E90740F1FB80A24803F033
:10CC7000C9FE002003F0D2FCA04CA14803F0C2FE84
:10CC8000A04803F0BFFE62799F4BA04803EB8203EC
:10CC9000D3F8DC11FBF74EFA9D48FBF74BFA26461A
:10CCA0000027D6F814800021404607F0EFFA20B1A3
:10CCB0009848FBF73FFA002669E039469648D6F8CF
:10CCC00018B0D6F81CA0D6F82090FBF733FA4046EF
:10CCD000002107F0E5FA10B1202003F08BFE06A931
:10CCE0004046FBF7ADF801468C48FBF723FA58465F
:10CCF000002107F0D5FA10B1202003F07BFE06A931
:10CD00005846FBF79DF801468448FBF713FA504656
:10CD1000002107F0C5FA10B1202003F06BFE06A930
:10CD20005046FBF78DF801467C48FBF703FA48466E
:10CD3000002107F0B5FA10B1202003F05BFE06A930
:10CD40004846FBF77DF8013701467548FBF7F2F9D5
:10CD50000C2F06F11006A4D1AAE749B294F8D4200A
:10CD600094F8D530009194F8D7106E48019194F959
:10CD7000D8100734029194F9D210039194F8D3108B
:10CD8000049131460136FBF7D5F9102E03D094F803
:10CD9000D6100029E1D100260E2777430024624AED
:10CDA0000123926CA3403A44D2F80A20134240F087
:10CDB000948001340E2CF2D10136082EECD15B4860
:10CDC00003F020FE4D4B5A4C9F6854F8041F19B1D4
:10CDD0005848FBF7AFF9F8E70E46574B53F8264093
:10CDE0004CB10123B3403B4203D054482146FBF7EA
:10CDF000A1F90136F1E7524803F004FE21463F4B0A
:10CE00000AAA0B4493F8883113444E4A8A5C0131D4
:10CE1000082903F8102CF2D1002306A94A488DF8FE
:10CE20002030FBF787F9494803F0ECFD4848FAF752
:10CE3000ADFC484803F0E6FD4548FAF771F946486D
:10CE400003F0E0FD4248FFF781FE4448FBF772F92A
:10CE50004020FFF7FFFB424803F0D4FD3C48FAF7BF
:10CE600037FDAA0726D53F4803F0CCFD3E4803F026
:10CE7000C9FD374803F012FC3C4803F0C3FD3448B9
:10CE8000FAF7CFF83A4803F0BDFD3148FAF7CEFB88
:10CE90003848FBF74FF92E48FAF750FA364803F0B6
:10CEA000B1FD2B48FFF726FC2C48FBF743F9802007
:10CEB000FFF7D0FB6B0716D5304803F0A3FD3048D1
:10CEC00003F0A0FD224803F0C3FB2448FBF732F92E
:10CED0004FF48070FFF7BEFB05E03146224629483B
:10CEE000FBF728F965E70BB0BDE8F08FC7CD010867
:10CEF00038D20108CECD0108D4CD01084C2800203D
:10CF0000E2CD0108F4CD010808AC010800CE01080B
:10CF10000BCE010818CE010825CE010839CC010836
:10CF20000DD501082DCE0108901C00204CCE010823
:10CF30004CAE01085CCE010850AE01086ACE010873
:10CF400077CE0108B4E0010883CE01088CCE010839
:10CF500064C701089BCE0108A7CE010869D6010865
:10CF6000B5CE0108C2CE0108D5CE0108E3CE010836
:10CF7000EDCE0108FCCE01080ACF010816CF01084A
:10CF800027CF010839CF010810B5204A18B9136816
:10CF900002221A8210BD1E481468002303802178E3
:10CFA000024611F07F010DD1637A990644BF022138
:10CFB000017013F0400F037814BF43F0010323F016
:10CFC000010314E0012920D002291DD1617901F06B
:10CFD0000F039B0003F1804303F5B84311F0800F6A
:10CFE0001B6806D003F03003102B07D10123137008
:10CFF00004E003F44053B3F5805FF6E7054B1B688C
:10D000001B699847024810BD184610BDD822002061
:10D01000E01C0020D020002010B5064C18B9236871
:10D0200001221A8210BD044B1B689B689847206838
:10D030000C3010BDD8220020D020002010B5064CA6
:10D0400018B9236801221A8210BD044B1B681B68A3
:10D05000984720680A3010BDD8220020D020002038
:10D06000084BDA68D10709D4DA68520708D4DB68BC
:10D0700013F0100F14BF03200420704701207047E5
:10D08000022070470020024003788B4283BF034B8D
:10D0900003EB410148880020704700BFE01C0020DE
:10D0A00070B5054601F082FD324CE369E061C31AB8
:10D0B000B3F5FA5F236282BF002384F8243084F83A
:10D0C000253094F824302BB9A12D02BF294A012123
:10D0D00082F8251094F82510264A31B1D118EDB206
:10D0E000013381F8265082F8243094F8245094F8C3
:10D0F0004730AB423CD11F4B93F84830052B02D050
:10D10000062B03D02FE0002005F03CFD94F82730DB
:10D110001E2B28D100200246C1B26B1E99421ADA9A
:10D12000214491F826300821DBB283EA0206F60793
:10D1300044BF83F01803C3F3460301F1FF3154BF2A
:10D140005B0843F0800311F0FF01C2F34702ECD10A
:10D1500001301A46E0E7234493F826309A4202D180
:10D16000032005F00FFD002384F8253084F82430D7
:10D1700070BD00BFE01C00202DE9F843324F3D6830
:10D180002A8A2E7AB2B9042E14D1304C3048237832
:10D19000012B0BD12F4B19682F4B89B20B445B002D
:10D1A00019681A6030230380227048E0102303803E
:10D1B000072644E0AC8AAB69A24294BF042602264B
:10D1C000944228BF14461FFA84F840469847214AE3
:10D1D00004F1010E13684FEA6E0E9BB203F1005387
:10D1E00003F540535B001B6800219BB203F1005321
:10D1F00003F540535B00714500F1020009D010F8BF
:10D20000019C10F802CC4CEA092C23F821C0013112
:10D21000F1E71268104B92B213445B001A681C606D
:10D220002B8A3022C8EB03032B826B8A9844084B6D
:10D23000A5F812801A80094B4FF440521A803B68BF
:10D240001E72BDE8F88300BFD8220020A83000205D
:10D25000CA200020505C004002300020C82000207E
:10D260000E4B0F4A1B683E299BB203EBC0000244E1
:10D270004FEA420209D94B09C80604BF03F1FF3344
:10D280009BB29B0243F4004304E04B08C90748BF2C
:10D2900001339B0211681360704700BF505C00406F
:10D2A000063000208A6810B50C6A036814430A69C6
:10D2B00023F4FF4314434A6923F0700314438A693B
:10D2C0001443CA6914434A6A14438A6A22431343C3
:10D2D0000360CB6843600B6883604B68C36010BD1C
:10D2E0004FF6FE730268134003600023036043603F
:10D2F0008360C360284B984201D1284A27E0284B1D
:10D30000984201D1254A2AE0264B984201D1234A6E
:10D310002DE0254B984201D1204A30E0234B984222
:10D3200001D11E4A33E0224B984204D11B4A536874
:10D3300043F470032EE01F4B984204D1174A536800
:10D3400043F0706326E01C4B984204D11B4A53689B
:10D3500043F00F031EE01A4B984204D1174A53685A
:10D3600043F0F00316E0174B984204D1134A536878
:10D3700043F470630EE0144B984204D10F4A536893
:10D3800043F4704306E0114B984204D10B4A5368B2
:10D3900043F47023536070470800024000000240CD
:10D3A0001C0002403000024044000240580002408D
:10D3B0006C00024080000240080402400004024069
:10D3C0001C0402403004024044040240580402405D
:10D3D0001F4A10B5536803F00C03042B03D0082B2D
:10D3E00004D01C4B14E01C4B1B6811E053685168BF
:10D3F000C3F38343C90303F1020301D4174906E0D1
:10D40000516811F4003F1449096818BF49084B439B
:10D41000036053681249C3F30313CC5C0368E34011
:10D4200043605468C4F302240C5D23FA04F484605E
:10D430005468C4F3C2240C5DE340C3605268C2F375
:10D4400081320A44127CB3FBF2F3036110BD00BFCA
:10D450000010024000127A004800002000093D0040
:10D4600038B0010810B50446FFF7FAFD012806D1CF
:10D470001CB1FFF7F5FD013CF8E7052010BD002CBD
:10D4800008BF052010BD0A88F0B54B888E88B1F81A
:10D4900008E0CC88002A3AD1028C43F0010322F044
:10D4A00001021204120C0284058B078CADB225F028
:10D4B000F30545EA0E1189B241EA06027A49BFB284
:10D4C000884212D001F5006188420ED0B0F1804F41
:10D4D0000BD0A1F59831884207D001F580618842D0
:10D4E00003D001F58061884202D127F0020701E0F4
:10D4F00027F00A071F4302830784038B23F00C03E2
:10D500001B041B0C0383038B9BB21C4344E0042AC3
:10D5100044D1028C22F010021204120C0284018BFE
:10D52000058C21F440721205120D42EA0E325E495A
:10D5300092B242EA06228842ADB292B212D001F50E
:10D54000006188420ED0B0F1804F0BD0A1F5983128
:10D55000884207D001F58061884203D001F58061DF
:10D56000884207D125F0200141EA03139BB243F022
:10D57000100304E025F0A00143F010030B430283E5
:10D580000384038B23F440631B041B0C0383038B72
:10D590009BB243EA0424A4B20483F0BD082A028C9F
:10D5A0003ED122F480721204120C0284828B3E4D12
:10D5B00092B222F0F307018C47EA0E1292B2A8420F
:10D5C00089B242EA060212D005F50065A8420ED0E3
:10D5D000B0F1804F0BD0A5F59835A84207D005F5DE
:10D5E0008065A84203D005F58065A84207D121F4E3
:10D5F000007141EA03239BB243F4807304E021F4F9
:10D60000206143F480730B4382830384838B23F074
:10D610000C031B041B0C8383838B9BB21C4341E0D4
:10D6200022F480521204120C0284858B018C25F4A2
:10D6300040752D052D0D45EA062545EA0E321A4D99
:10D6400089B2A84292B212D005F50065A8420ED068
:10D65000B0F1804F0BD0A5F59835A84207D005F55D
:10D660008065A84203D005F58065A84207D121F462
:10D67000005141EA03339BB243F4805305E047F67F
:10D68000FF5543F480530D402B4382830384838BE7
:10D6900023F440631B041B0C8383838B9BB243EAFC
:10D6A0000424A4B28483F0BD002C0140CA78F0B5F4
:10D6B000D40648BF8C780D8802F00F0348BF23437F
:10D6C00015F0FF0F1DD0016800240126A64006EAD0
:10D6D0000507B74211D14FEA840E0F2606FA0EF65F
:10D6E00021EA0601282A03FA0EF641EA060101D1D1
:10D6F000476102E0482A08BF07610134082CE4D1E1
:10D700000160FF2D1FD94168002404F1080701269C
:10D71000BE4006EA0507B74211D14FEA840E0F2634
:10D7200006FA0EF621EA0601282A03FA0EF641EA65
:10D73000060101D1476102E0482A08BF07610134B0
:10D74000082CE2D14160F0BD0F4B1A6842F0010293
:10D750001A6059680D4A0A405A601A6822F08472A9
:10D7600022F480321A601A6822F480221A605A6801
:10D7700022F4FE025A604FF41F029A60044B4FF0ED
:10D7800000629A60704700BF001002400000FFF87E
:10D7900000ED00E02DE9F843564C0368013AC4F867
:10D7A0004A3083880D46A4F84E30072A42D8DFE875
:10D7B00002F0040A101822292F35B4F84A300B80E1
:10D7C000B4F84C3013E0B4F84C300B80B4F84A3065
:10D7D00005E0B4F84A305B420B80B4F84C305B4251
:10D7E00005E0B4F84C305B420B80B4F84A306B80F3
:10D7F000B4F84E301DE0B4F84A305B420B80B4F808
:10D800004C3012E0B4F84C300B80B4F84A300CE0E5
:10D81000B4F84A300B80B4F84C3005E0B4F84C3022
:10D820005B420B80B4F84A305B426B80B4F84E30F8
:10D830005B42AB80304B1B79002B59D1B5F900000E
:10D8400006F03CFB8046B5F9020006F037FB0746C0
:10D85000B5F9040006F032FB216D0646404606F09D
:10D8600081FBE16D8146384606F07CFB0146484667
:10D8700006F070FAA16E8146304606F073FB014651
:10D88000484606F067FA0AF0EFFA616D28804046D4
:10D8900006F068FB216E8146384606F063FB0146C0
:10D8A000484606F057FAE16E8146304606F05AFBCC
:10D8B0000146484606F04EFA0AF0D6FAA16D688095
:10D8C000404606F04FFB616E8046384606F04AFB44
:10D8D0000146404606F03EFA216F0746304606F004
:10D8E00041FB0146384606F035FA0AF0BDFAA88039
:10D8F000BDE8F883E01C00204800002038B50F4B3D
:10D900001B689C890E4B186880F31000201A06F0E3
:10D91000D5FA0C4906F026FB0546204606F0CEFA5D
:10D920000146284606F0D2FB06F0E2FC6428A8BFB8
:10D93000642020EAE070C0B238BD00BFD0110020E2
:10D94000E01100200000C84244F6FB71084B1A6841
:10D95000137803EB431300FB03135078C0EB003044
:10D96000B3FBF0F39078B3FBF0F080B2704700BFE8
:10D97000D011002008B50A480A2290F8753000EB53
:10D980004303B3F88410903089B220F8041C01F0EE
:10D99000E3F980B2FFF7D8FF024B188008BD00BF43
:10D9A000E01C0020D41100202DE9F04F87B0039334
:10D9B000994B80461B889346980737D540F2E6324C
:10D9C000109B9648DC89B0F900301B1B03F2F3155D
:10D9D000954203D8002BB8BF5B4201E04FF4FA73C5
:10D9E000B0F9022040F2E630121B02F2F314844236
:10D9F00003D8002AB8BF524201E04FF4FA729342B2
:10DA0000B8BF13460522C3F5FA7393FBF2F30A225B
:10DA1000643B534398F81C20D2105343642293FB79
:10DA2000F2F3134423EAE373DBB200E06423C1465C
:10DA30000093CB1C02930025029B022D13F8016F6B
:10DA4000774F02934FEA450A05D1B7F904301B36E8
:10DA50005E43761149E0734B37F9152033F91530E1
:10DA600003EB4202CBF100039A4203DB5A45134613
:10DA7000A8BF5B466C4A32F90A40039A1B1B32F975
:10DA800015402344019305F075FC019B88B1674A5A
:10DA90001846545D06F012FA654906F017FB014678
:10DAA000204605F01FFA624906F05CFA06F020FCF9
:10DAB0000346594A1288D10713D437F90A401B3656
:10DAC000664392074FEA26160FD598F812409DF943
:10DAD000002063435343642293FBF2F306EB2316C7
:10DAE00003E098F808405C432611524B042433F9B4
:10DAF0000A3099F8017093FBF4F4341B67434E4EDF
:10DB000098F85120AB5D5F430193642397FBF3F7D3
:10DB1000FF1172B13846049206F0D0F9331D0C2182
:10DB200001FB0531049AB36AFAF7C4F806F0E0FB8A
:10DB30000746424B99F80B6019883F4B01FB04F2F2
:10DB400003F12C0E5EF82500D21206FB02063C4AB9
:10DB5000B6F5001FA8BF4FF40016964203F1380037
:10DB6000B8BF164650F8252040F825404FF6FF7004
:10DB70000909B0FBF1F1A21A4A4303F1440103F190
:10DB800050044EF8256051F825E054F8250044F87B
:10DB900025E098F85040921170444FEA850C7613B6
:10DBA000104441F8252094B1CDF810C0059306F03B
:10DBB00085F9059B0C2103F15C0201FB05219B6AA1
:10DBC0002246FAF777F806F093FBDDF810C099F8D3
:10DBD0001530BA195843019B013543431846642355
:10DBE00090FBF3F0174B0012024423F80A2003F1D4
:10DBF00008024CF80270032D03F1140203F1200314
:10DC00004CF802604CF8030009F101097FF414AFED
:10DC100007B0BDE8F08F00BFA81200202828002020
:10DC2000C8110020A0300020E22700204CB00108DD
:10DC30000000204108110020F81D0020E410002001
:10DC40000000E0FF781E00202DE9F04F8BB0079315
:10DC5000C04B0592B3F90220002682EAE279A9EBD3
:10DC6000E279B3F90020804682EAE273A3EBE27323
:10DC70009945B8BF9946B4463446B9F5FA7F06913E
:10DC8000A8BF4FF4FA79029001960396B24D2B8803
:10DC9000990755D0AF4B610033F91420AF4B33F9DE
:10DCA000143003EB4202059B5B429A4203DB059B67
:10DCB0009342A8BF1346AA4A8F5E079ADB1B32F92C
:10DCC00014001F1805F056FB90B1A64B384613F808
:10DCD00004A006F0F3F8A44906F0F8F9014650460E
:10DCE00005F000F9A04906F03DF906F001FB0746F2
:10DCF00098F8083064227B4393FBF2F398F81C20D9
:10DD00006FF0040101FB02FC634505DB02EB8202BC
:10DD10009342A8BF13469C4642F21072934B53F8AD
:10DD2000240038449042A8BF1046914A9042B8BFA0
:10DD3000104643F8240098F8123058430313039315
:10DD40002D8805F00303012B38D0824B894933F924
:10DD50001430A6000193029B51F8247093F801E05F
:10DD6000854B33F9140080EAE073A3EBE073B3F55D
:10DD7000206F16DC019A50235A4392FBFEF30422D3
:10DD800090FBF2F0181A0744B7F57A5F7B4BA8BFF7
:10DD90004FF47A579F42ACBF41F8247041F82430C9
:10DDA00002E0002341F824308B597D2693FBF6F6E0
:10DDB000029BDB7A7343402693FBF6F6AA0712D543
:10DDC000019B09FB06F509FB03F70398C9F5FA72F5
:10DDD00002FB0C7702FB00524FF4FA7197FBF1F350
:10DDE00092FBF1F505E0EB0755BF35466346019B15
:10DDF000039D614A042732F91420DFF884B192FBB5
:10DE0000F7F70BF1B402A25C4FEA440A57436FF0F4
:10DE10004F0297FBF2F798F851201F44A2B1384601
:10DE2000CDF810C0089206F049F80BF104030C215C
:10DE300001FB0431089ADBF82830F9F73BFF06F0C4
:10DE400057FA0746DDF810C04B4B4FEA840B3AF8FF
:10DE500003004B4B02B203F1B8013AF901E02AF892
:10DE60000100CEEB02024FF0040E92FBFEF203F132
:10DE7000BC0103F1C40E04925EF8240051F8242082
:10DE80001044049A104451F824204EF82420049A97
:10DE900041F8242098F85020A2B1CDF810C0099381
:10DEA000089206F00BF8099B4FF00C0E03F15C0191
:10DEB0000EFB0411089A9B6AF9F7FCFE06F018FAAB
:10DEC000DDF810C02E4B03F1CC02125D03F180018E
:10DED0005043202290FBF2F07A19121A2AF80120FE
:10DEE00003F188024BF8027003F194024BF80250E0
:10DEF000404203F1A0024BF80200029A0132029262
:10DF00000CB90124C2E6134A0420B2F90410069A9F
:10DF10005C6B92790F3252004A4317495511B1F99F
:10DF2000041085EAE57291FBF0F0A2EBE572322A6B
:10DF3000A5EB000098F80D1028DC01FB0041114A08
:10DF40008A42A8BF0A4610498A42ACBF5A63596345
:10DF50001EE000BFC8110020A8120020A030002041
:10DF6000E22700204CB0010800002041A41E002040
:10DF7000F0D8FFFF241E00200811002080C1FFFF01
:10DF8000F81D0020FEFFFF0F020000F000225A6380
:10DF900098F8031001FB00F2154992110978032942
:10DFA0000CD9B8F84E10B1F5FA7F07D24842824238
:10DFB00003DB8A42A8BF0A4600E00246596B6FF0B5
:10DFC000FF0041F34F31B1F5807FA8BF4FF480715E
:10DFD0008142B8BF0146C3F8902050180022A3F830
:10DFE0008400C3F89C10C3F8A8200BB0BDE8F08FE4
:10DFF000182100202DE9F04F87B00393BB4B8146D9
:10E000001D88029105F00205ADB2019295B1B84BA1
:10E01000B3F90250B3F90030002DB8BF6D42002BA8
:10E02000B8BF5B429D42B8BF1D46B5F5007FA8BF93
:10E030004FF40075CB460026AD4BAE4933F91620A0
:10E04000AD4B4FEA460A33F91630520083EAE374C7
:10E05000A4EBE374B4F5206F4FEA860851F826006C
:10E0600011DC042493FBF4F3D31A0344B3F57A5F71
:10E07000A248A8BF4FF47A538342ACBF41F8263080
:10E0800041F8260002E0002341F8263051F80870DC
:10E090009BF80B30FF119BF801405F43934B5443B7
:10E0A0001B88BF119B074FEAA41456D0944B3AF932
:10E0B00003301A44019B5B429A4203DB019B93426B
:10E0C000A8BF13468F4A3AF902209B1A039A32F9E5
:10E0D00016201A44049205F04DF9049A98B18A4B1F
:10E0E00010469B5D049305F0E9FE884905F0EEFFBC
:10E0F000049B0146184604F0F5FE844905F032FF02
:10E1000006F0F6F8024642F21070814958F80130E4
:10E1100013448342A8BF03467E488342B8BF0346E8
:10E1200048F8013099F8081099F81C004A4300EBB0
:10E130008000D21141428A4203DB8242A8BF0246DC
:10E14000114699F81220641A53431B13FF1A6F43A8
:10E150006C4303EB672701EB6424674B04223AF915
:10E16000033093FBF2F16C4B03F1B402925D4A432E
:10E17000A4EBA21499F8512082B120460593049291
:10E1800005F09CFE059B0C24191D04FB0611049A46
:10E190009B6AF9F78FFD06F0ABF80446564B3AF848
:10E1A00003005D4B02B203F1D0013AF901E02AF815
:10E1B0000100CEEB02024FF0040E92FBFEF203F1DF
:10E1C000D40103F1DC0E58F801C058F80E0048F8ED
:10E1D00001206044104499F8502048F80EC082B1E4
:10E1E0000593049205F06AFE059B4FF00C0E03F1B7
:10E1F0005C010EFB0611049A9B6AF9F75BFD06F0C1
:10E2000077F8454B0BF1010B03F1CC02925D03F162
:10E2100080015043E2194011121A2AF8012003F13B
:10E22000880248F8024003F1940248F80270404224
:10E2300003F1A00248F802000EB90126FCE62C4AC0
:10E240000420B2F90410029A5C6B92790F325200EA
:10E250004A4329495211B1F90410002A91FBF0F008
:10E26000A2EB0000B8BF5242322A99F80D100BDC25
:10E2700001FB0041294A8A42A8BF0A4628498A422E
:10E28000ACBF5A63596301E000225A6399F8031046
:10E2900001FB00F223499211097803290CD9B9F83E
:10E2A0004E10B1F5FA7F07D24842824203DB8A4220
:10E2B000A8BF0A4600E00246596B6FF0FF0041F329
:10E2C0004F31B1F5807FA8BF4FF480718142B8BF54
:10E2D0000146C3F8902050180022A3F88400C3F828
:10E2E0009C10C3F8A82007B0BDE8F08FA81200204A
:10E2F000C8110020241E00200811002080C1FFFF4B
:10E30000A0300020E22700204CB00108000020418E
:10E31000A41E0020F0D8FFFFF81D0020FEFFFF0F15
:10E32000020000F0182100202DE9F04F054690F87A
:10E3300050008DB008910592099318B13228A8BFFA
:10E34000322000E0012005F0B9FD0146AA4805F0A1
:10E35000BDFEAA4B04461888002808BF012005F01E
:10E36000ADFDA749069005F0FDFD019001992046FD
:10E3700005F0F0FC0146019805F0A8FEA14B0790BE
:10E380001B889A0724D5A049B1F90030B1F90200E1
:10E3900083EAE37280EAE071A2EBE372A1EBE07141
:10E3A00091420C46B8BF1446B4F5E17F12DA9142AF
:10E3B00003DD0028D8BF404203E0002BCCBF184645
:10E3C000584205F07BFD914905F080FE064603E0CA
:10E3D000002601E04FF07E564FF00009CA46039533
:10E3E0000024630004938A4B33F9140005F066FDA2
:10E3F000884905F0B7FD05F07BFF05F05FFD864914
:10E4000005F0B0FD804B029033F9140005F056FD85
:10E410007C4B07461B889B077ED0014605F09AFC83
:10E420007E4B804633F9140005F048FD0146404616
:10E4300005F090FC05F05CFF059B5B42984203DB16
:10E44000059B8342A8BF0346754A0499885E099AD2
:10E450001B1A32F91400184405F030FD804604F010
:10E4600089FF70B16F4B40466F4914F8039005F077
:10E470002DFE0146484604F035FD6B4905F072FD5E
:10E480008046287F05F016FD684905F06BFD824641
:10E49000287A05F00FFD0146404605F063FD64490A
:10E4A00005F060FD05F024FF81460AF1004005F00B
:10E4B0001FFF814505DB504605F01AFF4845A8BF00
:10E4C000484605F0FBFCDFF88C91019982464046F6
:10E4D00005F048FD59F8241005F03CFC55494FEA79
:10E4E000840B804605F0DCFE38B94046524905F001
:10E4F000F5FE20B1DFF8408101E0DFF8388149F80E
:10E500000B80A87C05F0D6FC0146404605F02AFDAC
:10E510004A4905F027FD81463A4BB3F800B01BF09D
:10E52000010F40F099803A4B049ADFF82081D35EC6
:10E53000002BB8BF5B42B3F5206F4FEA84030A9308
:10E5400003DD002348F824302AE03D49384605F031
:10E5500009FD039B0B90587805F0ACFC0B9A014623
:10E56000104605F0B3FD029905F0F2FB019905F0A4
:10E57000F9FC58F8241005F0EDFB3249804605F00F
:10E580008FFE38B94046304905F0A8FE20B1DFF8CB
:10E59000B88001E0DFF8AC802C4A0A9B42F8038087
:10E5A000039BD87A05F086FC284B53F8241005F01D
:10E5B000D9FC274905F0D6FC1BF0020F80464DD050
:10E5C0003846514605F0C4FB0146304605F0CAFC0A
:10E5D0000146504605F0BEFB49460746404605F059
:10E5E000B7FB0146304605F0BDFC0146484605F044
:10E5F000B1FB804632E000BF83F9223EE4100020E8
:10E60000BD378635A8120020C81100200000E14364
:10E61000081100200000A03ECDCC4C40A0300020CE
:10E62000E22700204CB00108000020410000A0407B
:10E630006F12033C0000F0C10000F0410AD7A33D77
:10E640000000A043000040C300004043E41E00203F
:10E650000AD7233CDC1E0020C8465746DFF830B2FC
:10E660000BF1B403185D05F029FC0146029805F092
:10E6700079FC864905F076FC0146384605F068FBD2
:10E6800095F8512003464AB10BF104030C2101FB1C
:10E690000431DBF82830F9F70DFB03467C4F029874
:10E6A00007F1F80B5BF824100A9305F051FB019970
:10E6B00005F00CFD029B07F580724BF8243052F8F0
:10E6C00024B00292594605F043FB0146079805F035
:10E6D00049FC0146584605F03DFB029A834642F844
:10E6E000240007F1CC02105D05F0E8FB0146584616
:10E6F00005F038FC674905F035FC83460A9B414626
:10E70000184605F027FB594605F022FB09F0ACFB43
:10E71000049B07F18002D0520A9B07F18802184639
:10E72000029205F0E5FD029A07F1940342F82400F5
:10E730004046029305F0DCFD029B07F1A00843F878
:10E7400024000BF1004005F0D3FD039B48F82400A2
:10E75000013303930CB9012443E6089A4E4B947994
:10E76000B3F90430640028345C434C4B6411B3F9B2
:10E77000040005F0A3FB4FF07A5105F0F3FB09F01C
:10E7800073FB201A05F09AFB002CB8BF6442322CB0
:10E79000064602DD00237B6324E0069805F0A8FD11
:10E7A00020F0030005F08AFB8046687B05F082FBC1
:10E7B0000146304605F0D6FB39490446404605F08F
:10E7C00085FC0146204605F0CDFB05F091FD7B6BF5
:10E7D0001844344B9842A8BF1846334B9842ACBFFC
:10E7E00078637B637B6B6FF0FF005B13B3F5807F17
:10E7F000A8BF4FF480739842B8BF184605F05EFB7F
:10E800008046304605F074FDEB785843801105F0E2
:10E8100055FB264B04461B78032B11D9B5F84E60E7
:10E82000B6F5FA7F0CD205F063FD7342984203DB24
:10E83000B0420346A8BF3346184605F03FFB0446E6
:10E8400095F851202AB120461949BB6AF9F732FAE6
:10E8500004464146204605F07DFA05F049FD00B228
:10E8600005F02CFB09F000FBA7F88400204605F01A
:10E870003FFDC7F89000404605F03AFD0023C7F879
:10E880009C00C7F8A8300DB0BDE8F08FA69B443BB4
:10E89000F81D0020F7CC9238C81100200811002084
:10E8A00000803B45FEFFFF0F020000F01821002012
:10E8B000141E0020034B4FF4004208B11A61704748
:10E8C0005A61704700080140034B4FF4004208B101
:10E8D0005A6170471A617047000801402DE9F74FEF
:10E8E0002F4C054627683846F9F7C6FC06463846D9
:10E8F000F9F74FFC676881463846F9F7BDFC01908F
:10E900003846F9F746FCD5F804A00746314650468C
:10E9100005F028FBD5F8088083464946404605F0B7
:10E9200021FB0146584605F013FA019B29688346EE
:10E93000184605F017FB49460546504605F012FB00
:10E94000394605F00FFB0146284605F003FA394623
:10E950000546404605F006FB314605F003FB01463F
:10E96000284605F0F7F90146584609F055FB0D49D0
:10E9700005F0F8FA0C4905F0A9FBA16805F0EAF9E1
:10E980000A4905F0A3FB09F06FFA83B21A0444BFE9
:10E9900000F5B47083B218B203B0BDE8F08F00BFC9
:10E9A000001F00200000E144DB0F4940000020412F
:10E9B00010B5084B0022196801EBC20393F902401D
:10E9C000844201D1981C10BD0132042AF4D10020E8
:10E9D00010BD00BFFC23002038B1438811EA0300BA
:10E9E00003D08B420CBF01200220704730B50A4B88
:10E9F0000A491C680A7B032A0AD81346551C04EBF3
:10EA0000C303EAB29D882842F5D00A73981C30BD32
:10EA10000A73002030BD00BFFC230020001F00202F
:10EA2000014B00221A73E1E7001F00202DE9F04797
:10EA3000877890F803C0BBB2C7F1640E03EB83067E
:10EA40005C42C3F178001C4D5FFA8EFE7600CCF17B
:10EA50006408A4B280B2A3B20FFA83F9B9F1000F2F
:10EA600004DC002B14BF3B46012300E0734609FB86
:10EA700009F25B4302FB0CF292FBF3F3434403FB0A
:10EA800009F30A2293FBF2F333449BB225F8023FC9
:10EA9000B1F800904A880A34C9EB020A1AB202FBA4
:10EAA0000AF24FF47A7392FBF3F3A4B24B4484421C
:10EAB0002B80D0D1BDE8F0870C1F002010B5447822
:10EAC0000078002240F6C41102FB02F3193B6343B5
:10EAD00003F6C4135343434393FBF1F3034921F873
:10EAE00012300132072AEDD110BD00BF261F0020D1
:10EAF000104B043033F91000B0F5617F05DB40F6B0
:10EB000033039842A8BF184601E04FF461700A78B9
:10EB100019235A4302F28332824208DA4A78534375
:10EB200003F283338342B4BF0020012070470020EA
:10EB3000704700BF2828002010B500F1500302786C
:10EB40008A4203D18478C278944204D30430984234
:10EB5000F5D1002010BD012010BD1FB5084B1B686A
:10EB60001B0309D58DF80400039101230D2001A991
:10EB70008DF80530FBF730FE05B05DF804FB00BFF3
:10EB8000EC2700201FB5084B1B681B0309D58DF827
:10EB90000400029100230D2001A98DF80530FBF738
:10EBA0001BFE05B05DF804FBEC27002010B5094AF8
:10EBB000094B11689B6812689142F8D1074A4FF4DB
:10EBC0007A70546B00FB04F2D31AB3FBF4F300FB2E
:10EBD000013010BD1028002010E000E0001F0020D0
:10EBE00038B50446FFF7E2FF0546FFF7DFFF401B9D
:10EBF000A042FAD338BD10B504462CB14FF47A7058
:10EC0000FFF7EEFF013CF8E710BD024A136801333D
:10EC10001360704710280020024B9B6B03B118470C
:10EC2000704700BF001F0020014B1B68184700BF42
:10EC30008430002010B50020FFF7F6FF064B0024BB
:10EC40001C7004F0DDF8054B83F83C401C64A3F80D
:10EC500044409C6410BD00BFD7270020001F002047
:10EC600010B510B9BDE81040E4E700230C225A4368
:10EC70000A4C1119125D824203D00133102BF5D1D9
:10EC800010BD074B986C18B14A784078824204D284
:10EC900000229964A3F844201A6410BD58B30108F7
:10ECA000001F002010B540001428A8BF1420002326
:10ECB000074A022199540B4499181424834201F8FD
:10ECC000014CF5DBFF21D1540F20BDE81040C7E710
:10ECD0006821002038B540F2DB156843104B08224C
:10ECE0001A61851E0B24013C14F0FF0411D00C4A5C
:10ECF0002846D36883F00803D360FFF77CFF012028
:10ED0000FFF792FF1920FFF776FF0020FFF78CFF37
:10ED1000E9E7044A044B1A60044A054BDA6038BD3F
:10ED2000000C0140EFBEADDEF04F00200400FA05FC
:10ED300000ED00E003685B69184703681B6918472A
:10ED40000368DB68184703689B68184703685B68BB
:10ED5000184703681B681847B0F902302DE9F74FD0
:10ED600093421CBF0023037090F800A004460E4697
:10ED70009146BAF1000F40F0AB80104605F09EF8C6
:10ED8000864905F0EFF8864905F0ECF84FF07C5124
:10ED900005F0E8F809F0C8F80146054605F0E2F884
:10EDA00080498346284605F0DDF803465846194653
:10EDB000019304F0CFFF4FF07E5104F0CBFF0146EA
:10EDC0004FF07E5005F082F92946804605F0CAF8DA
:10EDD000294605F0C7F807460146606004F0BAFF0F
:10EDE000E7604FF07E572946A0602761284604F06F
:10EDF000B1FF294605F0B6F84FF0804104F0A8FFB6
:10EE00000146404605F0AEF8019B60611946584640
:10EE100004F09EFF394604F09DFF0146404605F090
:10EE2000A1F840F2DC53A0462746554663651023FF
:10EE3000A4F852301823A061A4F850304FF0974145
:10EE4000D8F8100005F08EF80021824605F028FA67
:10EE500028B150464FF07C5104F07AFF04E0504650
:10EE60004FF07C5104F076FF05F0A4FAC7E90E01DB
:10EE70004FF09741D8F8040005F074F8002182465D
:10EE800005F00EFA28B150464FF07C5104F060FFB7
:10EE900004E050464FF07C5104F05CFF05F08AFA24
:10EEA0000135032DC7E9080108F1040807F1080737
:10EEB000C4D1A6F2DC531B042367E3676367C4F87D
:10EEC0008030A367C4F884300123A4F80290237033
:10EED000D4F85490B4F95280C9EB0606636A06FA76
:10EEE00008F67343276A4FEAE67B206F07FB0B3374
:10EEF0002667A7FB0667E26F1F44636CD4F840C027
:10EF000053434FEAE27B0CFB0B3ED4F88010C4F86D
:10EF10008020ACFB02237344B61A67EB0307E36A55
:10EF2000A26A43434FEAE07B02FB0B3EA2FB0023B5
:10EF30007344B6185F41E36C656F4B436067A06C28
:10EF40004FEAE17B00FB0B33C4F88410A0FB010106
:10EF50001944636B361A05FB03F3206B4FEAE57B1C
:10EF600000FB0B3367EB0107A0FB05018019194477
:10EF70007941B4F95020A56704F0D8FE08F1FF32BA
:10EF800001239340E067C01841EBE371424604F06F
:10EF9000CDFE484403B0BDE8F08F00BF6F12833A46
:10EFA000DB0F4940F404B53F2DE9F0410024234B29
:10EFB000E0B21E78B0420CD2214B33F81010214B36
:10EFC00053F820301BB10B2801D8DB689847013477
:10EFD000EDE71D4B1B685B032DD500242346E2B2F1
:10EFE000B24228D2174F4FEA840857F824205568B8
:10EFF0009D4218D02846FCF787FFEFF3128350227A
:10F0000082F3128811494FF0280EAA8C0EFB0010D3
:10F0100092B201320267AA8ADBB292B242F00102D6
:10F02000AA8283F3118857F8083000221B68013444
:10F030001A802B46D3E7BDE8F08100BF18210020DD
:10F04000241100201C210020EC270020001F00209C
:10F0500008B50E4B1B6813F4805F0D4B14BFD3F83B
:10F06000EC30D3F8F0309A880A4B19780023D8B2E4
:10F07000884204D2084820F813200133F7E7FFF74D
:10F0800093FFBDE808403220B5E500BFEC27002023
:10F09000001F002018210020241100200A4B30B549
:10F0A0001A680A4B02F48052D3F8EC40D3F8F050BF
:10F0B00000230AB1A18800E0A988054820F81310B0
:10F0C00001330C2BF5D130BDEC270020001F0020B0
:10F0D000FA20002070B5124D0024214605F1F500FC
:10F0E000702285F8F44008F0B2FC2146D5F868316A
:10F0F0000B4A0B4493F9020088B11E6802F1F50433
:10F100000E5108199C88073184809B79702983717E
:10F1100092F8F43003F1010382F8F430E6D170BDC7
:10F12000001F0020094B1A680E2303FB0020437ABE
:10F13000FF2B07D0064A12789A4203D9054A32F8C3
:10F14000130000E0808800B2704700BFD81C002088
:10F15000D4270020282800202DE9F04F91B0FFF798
:10F1600025FD8C4C0546D4F86C614FF00008831BDC
:10F170001846019304F09EFED4F87011029004F03A
:10F18000F1FEC4F86C514546D4F87471824E97F87C
:10F1900000B00390814A0DF11C0A32F9150004F009
:10F1A0008DFE039904F0DEFE4AF82500BBF1000F46
:10F1B0002BD0584604F082FE01464FF07E5004F0FA
:10F1C00085FF0246DFF8009211464FF07E5005920F
:10F1D00004F0BEFD59F8251004F0C4FE09F10C013D
:10F1E000049031F9150004F069FE059A114604F007
:10F1F000B9FEDDF810C00146604604F0ABFD49F8E9
:10F20000250005F075F8708003E0654A32F8152096
:10F21000728036F9022F0135032D02FB0288B9D125
:10F22000642303FB08F85F4B5F481B8807A95B4317
:10F2300098FBF3F8A8F149081FFA88F8F9F79AF84B
:10F24000B8F13B0F7D6810D9524BB3F99801D3F850
:10F25000945104F033FE0146284605F03FF8534B25
:10F2600068B31A7842F008022CE04FF07E5128462D
:10F2700004F070FD01464FF07E5004F027FF8146F8
:10F280004FF00008DFF820B128465BF8281004F0A2
:10F2900069FE474A039032F9180004F00FFE039B01
:10F2A0000146184604F056FD494604F05BFE4BF853
:10F2B000280008F10108B8F1030FE3D1C4E71A7878
:10F2C00022F008022946D4F890011A7008F0A4FE32
:10F2D00081462060D4F88C01D4F894B100F1004547
:10F2E000D4F89001014604F03DFE59468046584648
:10F2F00004F038FE0146404604F02CFD09F018F8F1
:10F300000146284608F088FE2A4980466060484643
:10F3100004F028FE08F0A8FD274D26492880404625
:10F3200004F020FE08F0A0FD244B68801B681B073A
:10F330004CD5234807A9F9F71DF8BD684FF07E5159
:10F34000284604F007FD01464FF07E5004F0BEFE53
:10F3500082464FF0000B1A4B284653F82B100493AB
:10F3600004F000FE1749039031F91B0004F0A6FDDC
:10F37000039A0146104604F0EDFC514604F0F2FDFC
:10F38000049B43F82B000BF1010BBBF1030FE2D1FF
:10F39000184652E0001F0020B01100200811002084
:10F3A000842000201C0000208C200020E811002078
:10F3B000B21100204C3D0F44E2270020E411002050
:10F3C0009C200020E0230020782000206C4D514636
:10F3D0002846F8F7CFFF28686B680146039304F0CE
:10F3E000C1FD039B82461946184604F0BBFD014649
:10F3F000504604F0AFFCD5F808B08246594658464E
:10F4000004F0B0FD0146504604F0A4FC08F090FF63
:10F410000021824604F03AFF70B92868514604F092
:10F4200055FE51462860686804F050FE51466860F9
:10F43000A86804F04BFEA8605148FFF74FFA514B03
:10F4400051491880029804F08DFD4E4B08F1004898
:10F45000054609F10049B3F90000CDF82C80CDF83C
:10F46000289004F02BFD494900F1004004F07AFD9A
:10F47000DFF82C810C90B8F9000004F01FFD0D900E
:10F48000B8F9020004F01AFD0E90B8F9040004F077
:10F4900015FD0AA90F900DA8F8F76CFF7B78012BDA
:10F4A0001AD13B4B3B4F1B7813F0040F0ED1D7F80A
:10F4B000A801402390FBF3F3C01A04F0FFFC0F995E
:10F4C00004F048FC04F014FFC7F8A801D7F8A8011D
:10F4D000402390FBF3F001E02F4B188804F0EEFC82
:10F4E00001460F9804F034FCD4F8B0110F90284670
:10F4F00004F030FC0146284604F0E8FDD4F8AC7175
:10F50000054639460F9804F023FC0146284604F0CE
:10F5100029FD0146384604F01DFC0746C4F8AC013D
:10F520000D9808F0A1FCD4F8B4512978F8F722FE20
:10F53000D4F8B8311844C4F8B8010E9808F094FC17
:10F540002978F8F717FED4F8BC311844C4F8BC0188
:10F55000384608F089FC6978F8F70CFED4F8C03119
:10F560000E4A184401991368C4F8C0011944D4F82C
:10F57000C43111600133C4F8C43111B0BDE8F08F5B
:10F5800050000020C0110020BD37863535FA8E3C72
:10F59000A6300020001F00201C000020803000202A
:10F5A000B211002001380A4B042804D8DFE800F02B
:10F5B0000507090B0D00074A08E0074A06E0074A5D
:10F5C00004E0074A02E0074A00E0074A1A60704771
:10F5D000FC00002099330108A9D9000899360108D8
:10F5E000F5DF000849DC000829E30008704708B58A
:10F5F0000B4B002093F82C10FDF732FE094B1B68D3
:10F60000187A082801BF084B4FF480521A80102244
:10F6100008BF5A80A0F109035842584108BD00BFF5
:10F62000C8000020D8220020C82000207047704762
:10F630007047FEE7FEE7FEE7704730B50024E3B20F
:10F6400093420DD2030F092B94BF3033373301F8A7
:10F650001430002501EB440300015D700134EEE736
:10F6600030BD30B5002240F60F7102F1805303F532
:10F67000B8539B001D6842F4004444F080042940C4
:10F6800001322143042A1960EDD1024B40F0800081
:10F69000186030BD4C5C00402DE9F347884D894C23
:10F6A0002B68894E9BB2A380A28831880A409705B7
:10F6B00007D54FF6FF53854A2B6013780133DBB231
:10F6C0001370A3880B40180440F100830023ADF8A9
:10F6D00002302B687B4F9AB21804A28040F1F68268
:10F6E000BB8803F00F03BB71002B40F0C182784A46
:10F6F00013689BB23B803B8803F030037B803B88E0
:10F7000003F440533B804BF6BF7311680B4083F406
:10F71000005383F0200343F4004343F0800313605D
:10F72000BB88D90621D448F60F7311680B4069498C
:10F7300013600B6888461A7A022A01D0042A02D183
:10F74000FDF71AFD59E2062A40F06B825A78052A25
:10F7500008D11A78520605D1D878FFF782FFBB6826
:10F760001B6A9847E3689B685AE213689BB2ADF83E
:10F770000230BDF802301F0540F1CF8140F68F7393
:10F780001168544F0B40544913600A68534B92B2AE
:10F7900013445B001A683B688846187A092817D01A
:10F7A00092B2520002F1804202F5C0421178197003
:10F7B000517859709188C8B2090A41EA00215980EC
:10F7C0001189C8B2090A41EA002199809289DA8038
:10F7D00001221A72DA8893F80190002A40F0DC8046
:10F7E0001A7812F07F024AD1B9F1090F0FD1DA78F5
:10F7F000012A00F2B8809978002940F0B4809988F5
:10F80000002940F0B0809A72A3685B68A9E0B9F162
:10F81000050F10D193F90320002A01DA0823B9E07B
:10F820009A78002AFAD19A88002AF7D19B7A002B7D
:10F8300000F0A280F2E7B9F1030F0ED1DA78012AC5
:10F8400040F091809A88002A40F08D805A7A42F0E8
:10F8500020025A72A368DB6983E0B9F1010F40F01E
:10F860008280DA78012A7ED19A88002A7BD15B7A5D
:10F87000980678D508F03EF800287DD073E0012A7C
:10F880002ED1B9F10B0F6ED1E26858799269D9780F
:10F8900090473B689A7A002A65D0002863D11A798C
:10F8A000002A60D19B78002B5DD1064B9B68DB68FA
:10F8B0009847084B1B685A79DA72DA781A735BE05A
:10F8C000445C0040C820002078300020A93000208F
:10F8D000005C0040D8220020505C00400430002032
:10F8E000022A40D1B9F1010FC4D0B9F1030F3AD1C6
:10F8F000587920F0800E4FEA8E0202F1804101F526
:10F90000B841096810F0800F14BF01F0300101F414
:10F910004051BEF1030F26D8B3F802E0BEF1000F4C
:10F9200021D101B39B7AF3B102F1804202F5B842D2
:10F93000136801064BBF23F4E04323F4804323F014
:10F94000400323F070034BBF9BB29BB283F01003C4
:10F9500083F4805343F4004343F080031360A368AF
:10F960009B69984708E0E36848465B699847032825
:10F970000FD000287FF452AFD8F80020A14B92B2EC
:10F9800013445B001A6800221A6030236380062348
:10F9900000E009233A6847E1B9F1060F12D11A785D
:10F9A000520677D19B78012B02D1E368DB6966E0D0
:10F9B000022B02D1E3681B6A61E0032B6AD1E36882
:10F9C0005B6A5CE0B9F1000F37D15988002961D139
:10F9D0005A6822F47F42B2F5003F5BD11A7812F0E8
:10F9E0007F0204D19B88002B00F0D58152E0012AD0
:10F9F00008D1E26858799269904700284AD13B685B
:10FA00009B7A16E0022A45D15A7902F00F018B0049
:10FA100003F1804303F5B8431B6812F0800F14BF55
:10FA200003F0300303F44053032933D812F0700F6E
:10FA300030D1002B40F0AF812CE0B9F1080F04D198
:10FA40001B785B0600F0A98124E0B9F10A0F21D1EF
:10FA50001A7802F07F02012A1CD19A7AD2B1598811
:10FA6000C1B95A6822F47F42B2F5803F12D1E268F0
:10FA7000587992699047002800F091810AE04BB1D3
:10FA80003A684FF00008A2F8128093614046984708
:10FA900040460BE0E3683A681B69507898470328B2
:10FAA00004D1594B09221B681A72BEE04FF6FF7150
:10FAB0003A68138A8B4201D10923B5E0022800D0AD
:10FAC0000BB90823B0E092F9001000291FDAD188A1
:10FAD00001910198834202D9019B138210E08B426D
:10FAE0000ED2E16891F82C00834201D2002105E09A
:10FAF00093FBF0F100FB113313B90121434B197053
:10FB0000E36893F82C309382FDF736FB8DE00323F6
:10FB100013724FF44053238087E0BDF802301BB2CC
:10FB2000002BBFF6D6AD40F68F7311680B40136003
:10FB3000354A176890463B7A022B72D0042B70D05E
:10FB4000032B01D0052B67D1BB693A8A8BB9398A5F
:10FB500000293BD04FF4405323802D4B1A68294B8A
:10FB600092B213445B001A6800221A60302363804B
:10FB70002CE0002AEBD0B7F81490914528BF9146AD
:10FB80001FFA89FA504698473B8A4FF0000ECAEB9D
:10FB900003033B827B8A53447B821D4B1A681D4BB7
:10FBA00092B213445B001B6809F101029BB203F19E
:10FBB000005303F5405352105B009645C7D053F8ED
:10FBC0002E1020F81E100EF1010EF6E7BB8A8B42B4
:10FBD000D8F8003001D8032201E011B105221A72D1
:10FBE0000BE006221A720A4B1A68064B92B21344B3
:10FBF0005B001A68196030236380D8F800301B7AE4
:10FC000010E000BF02300020D8220020A8300020E1
:10FC1000505C004004300020072B02D1E368DB6811
:10FC200098470823D8F800201372FFF7E0FC5E4BDA
:10FC30001A684BF6BF7313402288D704228848BF46
:10FC400083F480539004628848BF83F40053D10644
:10FC5000628848BF83F01003920648BF83F02003F8
:10FC600043F4004343F080034F4A9BB213602DE0FE
:10FC70009A0002F1804202F5B842116889B2ADF8EB
:10FC80000210BDF8021009B2002909DA40F68F719E
:10FC90001068013B01401160444A52F823309847F4
:10FCA000BDF802301F067FF514AD48F60F72A1793A
:10FCB0008B0003F1804303F5B843186802401A60D3
:10FCC0003A4B03EB81039B69984702E5A28833888E
:10FCD0001340590505D54FF6FF332B60344B5B6855
:10FCE0009847A28831880A40920444BF4DF6FF73BA
:10FCF0002B60A3882F4A0B40DB0452D54EF6FF73CE
:10FD00002B6000231374137C052B41D8DFE803F02C
:10FD1000030D1418222D6369264D1BB902F0B6FBA2
:10FD2000062300E005232B743BE002F0AFFB042325
:10FD300023740123636134E002236374032328E006
:10FD4000637C013BDBB26374637C53BB194B0422BD
:10FD50001A7426E0184A13689BB243F0100313602C
:10FD6000052323740A2363741BE0637C114A013B5F
:10FD7000DBB26374637C03F0FF0093B94FF6EF735B
:10FD80000D490C6823400B6006231374506108E092
:10FD90000623237405E0094B72E6094B70E6094B14
:10FDA0006EE602B0BDE8F087005C004050B001088C
:10FDB000C8000020C8200020405C004089CF000817
:10FDC0003DD0000819D0000837B5062204460321AB
:10FDD0006B461E20F5F7A0F99DF801309DF8000054
:10FDE000154D43EA002000B204F068F8296804F0D9
:10FDF000B9F804F07DFA9DF8033020809DF80200E8
:10FE000043EA002000B204F059F8A96804F0AAF807
:10FE100004F06EFA9DF80530A0809DF8040043EAD6
:10FE2000002000B204F04AF8696804F09BF804F07E
:10FE30005FFA608003B030BD5C0000202DE9F04720
:10FE4000664D2B686649581C0A788E4602F0FF06FC
:10FE50000AB10346F6E737462B60687BAB6895F836
:10FE60000C80AA7B39B2202900F09C80DFF880C189
:10FE70000CEB8103DC789B783CF82110C3F1FF0385
:10FE80009BB2002B65D04FF03C0CB1FBFCF9C3F1E9
:10FE9000FF0363431B12B9F1050F5DD8DFE809F0DA
:10FEA000030B1A293A4AE01A4143B1FBFCF0DAB2DB
:10FEB0001044C0B251E0B1FBFCF00CFB101189B250
:10FEC000DAB2C1F13C01E31A4B43B3FBFCFC204620
:10FED00094442CE0B1FBFCF00CFB1011E21A89B247
:10FEE0004A43B2FBFCF25FFA83F84244D2B22046A6
:10FEF00032E0B1FBFCF90CFB191189B2E01AC1F137
:10FF00003C014843B0FBFCF05FFA83F84044C0B2C8
:10FF1000224621E0B1FBFCF80CFB1811D8B289B2E3
:10FF2000E31A01FB03F2B2FBFCFC224684445FFAB5
:10FF30008CF412E0B1FBFCF80CFB181189B2D8B2BA
:10FF4000C1F13C01E31A4B43B3FBFCF20244D2B2D1
:10FF500003E02246204600E044464FEA042C4CEAE7
:10FF6000004C4CEA020C17234FF0010808FA03F882
:10FF700006F1170118EA0C0FA1EB0301DFF87480FA
:10FF800014BF4FF011094FF0090989B213F1FF3383
:10FF900008F80190E8D218360137B6B2BFB2114B5B
:10FFA000A0465FE7AB6001238EF8003040F22A33B1
:10FFB000AA730D4AE9800D4985F80C806873AE80FC
:10FFC000536000238B840B889BB243F001030B80AA
:10FFD000136843F001031360BDE8F087E0200020C0
:10FFE000A5300020EC2000206C00024000040040FE
:10FFF000C20E00206D030020F0B5B1F800E0002330
:020000040801F1
:100000004EFA03F2D50725D58E784FEAD30CF406C5
:1000100048BFCC7806F00F0203F0070748BF224321
:10002000BF0050F82C500F24BC4025EA0404BA400D
:100030002243282E40F82C2005D1C46801229A4082
:1000400024EA020205E0482E04D1C46801229A4045
:100050002243C2600133102BD2D1F0BD2DE9FF4104
:100060005B4B1B689BB11A681AB15A4988690243F5
:100070008A619A889868ADF8042002228DF80720DA
:1000800004220DEB02018DF80620FFF7B5FF3220A8
:10009000FEF7B1FD002111221E20F5F7FDF8012128
:1000A00060221E20F5F7F8F86420FEF7A4FD002476
:1000B00002A8FFF789FE274626460A2502210122CB
:1000C0001E20F5F7E9F83220FEF795FD02A8FFF7AC
:1000D0007BFEBDF90820BDF90A1014448A42A8BF6E
:1000E0000A46BDF90C300F4493421E44A8BF134684
:1000F00013F5805F04DD013DE0D14FF0010801E020
:100100004FF000081E2000211222F5F7C5F80A253D
:10011000022101221E20F5F7BFF83220FEF76BFD09
:1001200002A8FFF751FEBDF90820BDF90A10A41A74
:100130008A42A8BF0A46BDF90C307F1A9342A6EB4B
:100140000306A8BF134613F5805F02DD013DDFD132
:1001500001E04FF00008204603F0B0FE01461E48C3
:1001600003F0B4FF1D4D20F000402860384603F036
:10017000A5FE0146184803F0A9FF20F00040686082
:10018000304603F09BFE0146154803F09FFF20F028
:100190000040A860002170221E20F5F77DF80121A3
:1001A00020221E20F5F778F81E2002210022F5F704
:1001B00073F86420FEF71FFDB8F1000F04D14FF073
:1001C0007E532B606B60AB6004B0BDE8F08100BF74
:1001D0004C0300200010024000406F465C000020ED
:1001E00001C05E46104B73B518781C46A0B10523BC
:1001F0000E4D8DF800304FF4805600238DF80130FD
:100200000B486E6101A96A460223F5F7ADF82E612D
:100210009DF8050000F0010000F00100207080F062
:10022000010002B070BD00BFC1060020000C0140FB
:1002300000380040064B70B506461C461D68FFF7A7
:10024000D1FF18B923685B1BB342F8D970BD00BF5A
:1002500010280020F7B503238DF80430030C8DF827
:1002600005308DF80700030A06200F4614468DF866
:100270000630FFF7DFFF88B1094D4FF480560021AB
:1002800001AA04236E610748F5F76EF80548394660
:1002900000222346F5F768F820462E6103B0F0BD32
:1002A000000C014000380040024640213C20F4F799
:1002B000F3BF70B500EB8000094CA0F1A1059C389C
:1002C00025440444074B15F8010F1E787040FFF7D2
:1002D000EBFFA542F6D13046BDE87040E4E700BF31
:1002E0008CB00108AA30002010B5441E14F8010F8C
:1002F00010B1FFF7DEFFF9E710BD024680213C2078
:10030000F4F7CABF10B5D420FFF7F7FF8020FFF73E
:10031000F4FFA820FFF7F1FF3F20FFF7EEFFD32007
:10032000FFF7EBFF0020FFF7E8FF4020FFF7E5FFB6
:100330008D20FFF7E2FF1420FFF7DFFFA120FFF77A
:10034000DCFFC820FFF7D9FFDA20FFF7D6FF122025
:10035000FFF7D3FF8120FFF7D0FFCF20FFF7CDFFBE
:10036000D920FFF7CAFFF120FFF7C7FFDB20FFF717
:10037000C4FF4020FFF7C1FFA420FFF7BEFFA62067
:10038000FFF7BBFFAF20FFF7B8FFA620FFF7B5FFD1
:10039000AE20FFF7B2FF2020FFF7AFFF0020FFF7EE
:1003A000ACFFB020FFF7A9FF4020FFF7A6FF002019
:1003B000FFF7A3FF1020FFF7A0FF4FF48064013C7C
:1003C0000020A4B2FFF770FF002CF8D18120FFF7C6
:1003D00094FFC820FFF791FFAF20FFF78EFF0120A9
:1003E00010BD08B55038C0B2FFF787FF0020FFF7F7
:1003F00084FFBDE8084010207FE710B5044650395F
:10040000C8B2FFF77AFF04EB4400400000F00E0092
:10041000FFF773FF06206043BDE81040C0F30310F0
:1004200010306AE7012828BF01202DE9F04F064669
:10043000734F142000FB0671724BD1F8A4421E7555
:100440001C61714BD1F8B422DD69B1F8AC822A434A
:10045000DA61A288B1F8AEA222F44072D1F8A852B3
:10046000120489B0120C4AEA0809A28003A9C5F84F
:10047000109002228DF80E0028460193ADF80C90E2
:100480008DF80F20FFF7B8FD019B00971F464FF036
:10049000080BAA6818EA020F03D10A20FEF7A0FB96
:1004A000F7E70A20C5F81480FEF79AFBC5F810801C
:1004B0000A20FEF795FBBBF1010BEAD1C5F814A0A9
:1004C0000A20FEF78DFBC5F814800A20FEF788FB92
:1004D000C5F810800A20FEF783FB0222C5F810A0A1
:1004E000284603A98DF80F201C228DF80E20ADF8A8
:1004F0000C90FFF781FD454A03A894423A690BBF6F
:1005000042F4001242F480023A613A610BBF3A6948
:100510003A6922F4001222F480023A61A38823F49B
:1005200040731B041B0CA38023889BB243F0010380
:100530002380A588FCF74CFF0599354B25F03F0536
:10054000B1FBF3F32D042D0C1D43ADB2A580228821
:10055000002522F001021204120C22802D4A03A869
:10056000B1FBF2F100298AB208BF012242F4004136
:100570004FF4967253434FF47A7293FBF2F30133C4
:100580009BB22384A1832388009A9BB243F001038A
:100590002380238823F4816323F002031B041B0CB4
:1005A00023804FF480432381142303FB062696F80F
:1005B000B13201248DF80C308DF80D508DF80E50AD
:1005C0008DF80F4002F040FC96F8B0329DF80F20F5
:1005D0008DF80C308DF80D508DF80E501AB103A81F
:1005E00002F032FC08E05A0903F01F039C4002F1BC
:1005F0002003094A42F8234009B0BDE8F08F00BF4C
:100600008CB00108E020002000100240005400409F
:1006100040420F00804F120000E100E007B5064B9A
:1006200006490093064B074A01930748074BF7F723
:1006300081FD03B05DF804FB94C40108CDCA010834
:1006400069C40108C6CA01089CD4010888C401080D
:1006500008B5037833B90C4B0C481978BDE808404D
:10066000F7F768BD07F08CFA02280CD8064B0C226D
:100670001870074B02FB0030064B0230186001F087
:10068000ABF80548E5E708BDF8200020BCD4010818
:10069000EC2F00204811002064C7010808B503783A
:1006A0003BB90B4B0B4893F8A017BDE80840F7F790
:1006B00041BD07F065FA022808D8054B83F8A0076A
:1006C000F7F7FEFEF7F79EFF0348E8E708BD00BF17
:1006D0004C280020C0D4010864C7010838B503784D
:1006E00003BB214B1B6801330F2B07D81F490C227A
:1006F00002FB031295681C462DBB00E01C4601342A
:100700000F2C01DD002400E005D818490C2202FB63
:1007100004129568BDB99C42F1D11548BDE8384036
:10072000F7F708BD07F02CFA0F28044605D80F4A42
:100730000C2303FB00239D682DB92146BDE83840FA
:100740000C48F7F7F7BC084B1C60FEF773FA21461C
:100750002A460948F7F7EEFC0C235C43034B185D6F
:10076000BDE83840FEF77CBA6800002058B30108A5
:10077000CDD40108E3D40108FBD4010873B5037894
:1007800013B9F6F7C7FC3FE001AA204907F059FA70
:1007900000240246264625469AB134B1012C08D1E0
:1007A000104607F0EDF9064603E0104607F0E8F9B9
:1007B000054601AA0020154907F043FA0134024614
:1007C000EAE70B2D03D9124812490C230CE0022C46
:1007D00011D1A6F57A73B3F57A7F08D90C480E4982
:1007E0004FF47A724FF4FA63F7F7A4FC0CE00B4B6A
:1007F00003EB45035E80094B094803EB450329469B
:10080000B3F90220F7F796FC02B070BDB1CD010834
:100810007DC901089CC901085AD10108F8200020AF
:1008200012D5010838B50D4C05462368834206D120
:10083000F7F7C1F8204600214C2207F008F9E36CD5
:10084000AB4209D12846F7F7B6F8BDE8384004486E
:1008500000214C2207F0FBB838BD00BF3C2300202C
:1008600088230020034B1A68D379591C1344D17193
:10087000187A70478812002010B5FFF7F3FF84B292
:10088000FFF7F0FF04EB002080B210BD10B5FFF7BA
:10089000F3FF0446FFF7F0FF04EB004010BD10B576
:1008A0000446054B21461868FEF753FA034B1B68B4
:1008B00098796040987110BD8C1200208812002039
:1008C00038B504460D462420FFF7E9FF4D20FFF719
:1008D000E6FF002C084C14BF21203E20FFF7DFFF6D
:1008E0002368002228469A71FFF7D9FF236893F8FE
:1008F0004900BDE83840D2E78812002001460020B8
:10090000DEE710B50446C0B2FFF7C9FF200ABDE814
:100910001040C4E710B5044680B2FFF7F2FF200C88
:10092000BDE81040EDE737B58288836804461006BD
:100930000D4641BF29494FF4CC7091F8A01700FB38
:100940000133D10542BF26490C20097802F03F024D
:1009500048BF00FB0133042A12D006D8012A0DD06B
:10096000022A2FD193F900102DE0102A0AD0202A54
:100970000AD0082A26D1B3F9001024E0197822E021
:10098000198820E019681EE069461868F7F758FAD8
:1009900001461448F7F7CEFBF5B1E06803F08EFA94
:1009A0006946F7F74DFA01460F48F7F7C3FB206990
:1009B00003F084FA6946F7F743FA01460A48F7F765
:1009C000B9FB09E000210948F7F7B4FB25B1084855
:1009D000E1682269F7F7AEFB03B030BD4C28002078
:1009E000F820002039CC010832CC01089FCB010847
:1009F00021D50108024B0146D869FEF7AAB900BF0C
:100A0000F820002010B5441E14F8011F21B1034B3B
:100A1000D869FEF79EF9F7E710BD00BFF820002067
:100A20002DE9F04F037885B01BB96C48FFF7EAFF5A
:100A3000D1E007F0A5F805460628694C99BF69483A
:100A4000294669480621F7F775FB94F82020002312
:100A5000D9B2914207D26549002051F823100133E1
:100A600009680880F4E7013DEDB272B6604F6DB2DF
:100A700007EBC50149684FF001085E4B5E4E57F821
:100A80003590042208FA01FA5A611FFA8AF14FF4EC
:100A900080624FF4007372614FF0480B736130460F
:100AA000C9F8141003A9ADF80C2001938DF80EB00D
:100AB0008DF80F80FFF7A0FA019B3046ADF80C309F
:100AC00003A910238DF80E30ADB28DF80F80FFF71B
:100AD00093FA484603A9ADF80CA08DF80EB08DF836
:100AE0000F80FFF789FAE9007B185A6857F835300C
:100AF000D00803EB800E53F8203002F00702A36504
:100B00009200E36523660F239340DB43E06DC4F856
:100B100054E01840E065A06D0340A365E06D082334
:100B200093400343E365A06D08FA02F3034338469C
:100B3000A365B3685F05FCD4676DA36D08223B60B5
:100B40004FF40073C9F814A073612A4B1A6140F680
:100B5000B833B268520516D4013BFAD14FF4007392
:100B6000ADF80C3018238DF80E302348012303A96B
:100B70008DF80F30FFF740FA236E04223B601D4BC7
:100B80001A6162B627E0C9F810A0E36D50F835E0AD
:100B90003B604318D3F804C0DEF80C20012303FAAD
:100BA0000CF31343CEF80C30B268134B5205C4D586
:100BB000D9F808204FF4007C1AEA020F0D4A4FF0D2
:100BC000080E15BFC3F810C0C3F814C0C2F810E077
:100BD000C2F814E0E8E705B0BDE8F08F28D50108B9
:100BE000F82000206FD501089BD501081C210020AA
:100BF0006CD40108000C014000080140F7B52A49F7
:100C00002A4B08782A4D1C682A4B05EB80001A886D
:100C1000D0F8C010284B29481B7800914FF47A7106
:100C2000B4FBF1F1F7F786FA254B26481968264BF5
:100C30000026B1FBF3F1F7F77DFA244B1F68F3B2FE
:100C400005EB8302D2F8D010E9B101249C403C426C
:100C500017D0220715D01E4A0B20D25C00FB0323BD
:100C6000134A1C4802EB8303D3F8F020F7F762FA2B
:100C7000022C06D1184B93F86C1011B11748F7F7F6
:100C800059FA0136DBE71648FFF7BCFE154B16484C
:100C90001A88164B92B2198840F2CC7303B0BDE8A3
:100CA000F040F7F747BA00BF3412002010280020A8
:100CB00058B30108D4110020F8000020C6D501085F
:100CC0000401002009D6010840420F00E411002071
:100CD0000001002019D60108F820002021D60108C3
:100CE00069D60108E610002025D60108E41000208E
:100CF0002DE9F0410024804625460F4E4146A75974
:100D0000384606F025FF58B139460C48F7F712FA75
:100D100030190021FFF707FE0948FFF773FE013580
:100D20001434B4F5486FE8D11DB9BDE8F041054869
:100D300068E6BDE8F08100BFF8B40108C1CC010845
:100D400069D601080ECA01082DE9F74F824606F060
:100D5000C2FE054628B1012818D19AF800302A2B86
:100D600014D15848FFF74EFE0024574E5748A1595A
:100D7000F7F7E0F930192946FFF7D5FD1434544848
:100D8000FFF740FEB4F5486FEFD198E050463D21A3
:100D900006F093FE002800F08D8003461D4613F8F0
:100DA000012D202AFAD0441C204606F0E9FE814697
:100DB0002046F6F7AFFF0746CAEB05054FF0000BDC
:100DC000142404FB0BF4DFF8208108F5D073E658F7
:100DD0000193304606F07FFE844631466246504617
:100DE000CDF800C006F080FEDDF800C0019B0028B1
:100DF00056D1EAB2624553D11D194444D4F8AC012E
:100E000003F05CF80146384603F05EFA002845D04E
:100E1000D4F8B00103F052F80146384603F04AFA1C
:100E200000283BD0B4F8A4319A0658BF4F4614228C
:100E300002FB0B881C0648BF2648D8F8A82142BFF1
:100E400090F8A0074FF4CC7404FB0022D80542BFF1
:100E500021480C24007803F03F0348BF04FB002224
:100E6000042B39460BD004D8013B012B0CD817704A
:100E70000AE0102B05D0202B05D0082B04D11180BF
:100E800002E0176000E0176031461448F7F752F9A6
:100E90002846002103B0BDE8F04F44E5104805E0C6
:100EA0000BF1010BBBF1A00F8AD10E4803B0BDE8D6
:100EB000F04FA7E5504603B0BDE8F04F18E703B088
:100EC000BDE8F08F57D60108F8B40108C1CC01087D
:100ED00069D601084C280020F82000206CD60108B3
:100EE00077D601080ECA010858B3010808B50748AB
:100EF000FFF788FD064BD869F6F752FDFEF7A8F814
:100F0000F7F7B4FA034A044BDA6008BD97D6010834
:100F1000F82000200400FA0500ED00E008B50548BF
:100F2000FFF770FD00F09EFCF7F7CAFABDE8084035
:100F3000DCE700BFA3D6010808B50448FFF762FD4F
:100F4000F7F7BEFABDE80840D0E700BFB9D6010800
:100F500010B54B88DC0641BF2F4B14791B6853F842
:100F6000244044BF2D4B43F820404B889B0641BF93
:100F7000294B54791B6853F8244044BF274B43F84E
:100F800020404B881C070ED5254B0C781B78B3EB03
:100F9000141FA1BF204BD4781B6853F82440A4BF72
:100FA0001E4B43F820404B889B070ED51D4B0C78F9
:100FB0001B78B3EB141FDFBF174B54781B6853F833
:100FC0002440DCBF154B43F820404B88DC070FD58D
:100FD000154C0B78247803F00F03A342DFBF0E4BB0
:100FE00014781B6853F82440DCBF0C4B43F82040B6
:100FF0004B885B070FD50B780C4903F00F0309787A
:101000008B42A1BF044B92781B6853F82220A4BFE7
:10101000024B43F8202010BDD41C0020C20E00203B
:101020006316002061160020601600206216002062
:10103000254A0023F0B515681C461A462348244962
:1010400003700B702E1976884EB92F5D3FB903706F
:1010500000230A704B7007781C461A460CE03605D0
:1010600048BF013204F1040403F1010348BFD2B2C6
:10107000802CDBB2E6D1EAE7E0B2B8420CD215F838
:101080002400013406099E4200F00F00A8BF731C23
:101090009042A8BF421CEFE78A704B70C2F3470131
:1010A00002F001020A444C1E0A490B480A70C3F3BD
:1010B000470203F00103134404700849501E084A14
:1010C00008701370F0BD00BFAC120020581600204D
:1010D0008021002062160020601600206316002088
:1010E00061160020924B2DE9F04FDA68914D1A619C
:1010F0002A6891B0DA60904A0295136843F02003A1
:1011000013608E4B1A78012A0CBF002201221A703C
:101110008B4B1A78910740F14D838A49097804294D
:1011200040F248838849097801F0040101F0FF008A
:1011300011B922F001021A701B78DB0702D408B142
:10114000FAF766FB8149CA78531C052293FBF2F239
:1011500002EB82029A1A7E4BCA701F78920000231B
:10116000DFF81082DFF8109258F82310794C91FBC9
:10117000F9FE04F1080040F823E0774844F8231012
:1011800000FB0E1142F2107091FBF0F004F110061A
:1011900080B226F813004FF0140C04F114060CFB77
:1011A000036C04F13C0A5AF823605CF802504CF8D6
:1011B0000210761B314405264AF8231091FBF6F104
:1011C00009FB0E114434012F44F823104FEA830B1E
:1011D000444605D10238B0F5797F98BF4BF8081026
:1011E0000BB90123BCE7594E029BB2461868336D18
:1011F000C01A02F05FFE594902F068FF029B4FF0EF
:101200007E511B680746336503F04AF808B94FF072
:101210007E574B4BCAF854701B78514E13F00103A4
:10122000504D12D00DAA00924F4B0EAA01920CCB3A
:1012300094E80300FAF702FA0D9A6421B2FBF1F286
:101240000E9B328093FBF1F300E033802B809AF801
:1012500058303E4D002B35D0696D4FF07E5002F076
:1012600035FF0746EB6D2068C01A02F027FE3946AD
:1012700002F078FE03F03CF82B6E86B2606836B25E
:10128000C01A02F01BFE394B196802F06BFE39469A
:1012900002F068FE03F02CF8B5F9662000B2811860
:1012A000B5F964200220B31891FBF0F193FBF0F341
:1012B00089B29BB2A5F86A10A5F86830A5F8661047
:1012C000A5F8643001238AF85830294B61681B88DF
:1012D000206803F030031D4E264DCAF86010CAF88E
:1012E0005C00002B00F0668206F17403009306F1A7
:1012F00078030193F26E336FFAF7A0F96B68306FE1
:10130000C01A02F0DBFD194B196802F02BFE02F047
:10131000EFFFF36E2A68C6F880009B1AF3670C4B48
:101320001B78012B2AD0022B00F0E68042E200BF9E
:101330002808002010280020E41100204E11002071
:10134000E8110020EE110020A630002080210020AE
:10135000FC0F002084210020806967FF00007A4490
:101360006212002064120020501100206C00002046
:10137000A8120020F011002080969800D6F8843042
:10138000D6F8A0400293D6F8943004F100400393BD
:10139000D6F89830776D059302F0AAFF8146204673
:1013A00002F0A6FFD6F89C30BB4C0493BB4B0690D2
:1013B0001B684FF0000B0793B94E4FEA4B0356F8EA
:1013C0002B80A6F11402404632F81B50089302F01D
:1013D00075FD029902F0C6FD02F08AFF401B1FFA5C
:1013E00080FA283626F81BA00FFA8AFA504602F037
:1013F00065FD039902F0B6FD02F07AFF86B20AEBB2
:10140000080002F05BFD059902F0ACFD394602F0E0
:10141000A9FD216802F09EFC02F06AFF484504DB4A
:10142000069B9842A8BF184600E0484602F046FDD9
:10143000206002F05DFF079B304486B2987802F08E
:1014400039FD984902F08EFD01464FF07E5002F0C2
:101450003DFE394602F07EFC0146384602F036FE7B
:1014600009906068D4F808A0C0EB080002F026FDDF
:10147000394602F02BFE514602F06AFC099A0146F9
:10148000104602F06FFD0146504602F063FC313514
:10149000ADB2622D01462061C4F80480A0600ED96F
:1014A000049802F05FFD02F023FF7F4AB0F5FA6F67
:1014B000A8BF4FF4FA609042B8BF104600E0002089
:1014C00040F6B832064436B29642A8BF1646774A6E
:1014D000089B9642B8BF1646754A54F8140B9E52A4
:1014E000142202FB0BF273495050BBF1000F40F085
:1014F00061814FF0010B5FE7684BB6F8A8401F68A9
:10150000736F3D8902935B089D4228BF1D4623B23D
:101510009D4202DC1FFA85F90AE06749706D02F00E
:1015200021FD02F0E5FE20441FFA80F9A6F8A890FC
:10153000DAF87860DAF8AC40341B2046FAF7C0F8E5
:1015400041F293130028D8BF40429842CCBF0020FC
:10155000012078B3204602F0B1FC584902F002FDA8
:10156000F6F717FE0446029802F0A4FC0146204656
:1015700002F0F8FC02F0BCFE40F6B83380B2AAF8E4
:10158000B00000B29842A8BF1846484B9842ACBF82
:101590003018F01848F6A043984203DDA0F50C403F
:1015A000A03804E00028BCBF00F50C40A030CAF809
:1015B000B40001E0CAF8B460DAF8B4300026C3F52C
:1015C0000C502830039302F079FC3C4902F0CAFC2D
:1015D0000446F6F751FE0F902046F6F7DAFDDAF8EA
:1015E000B830DAF8C4400593DAF8BC300E9004F154
:1015F0000040089302F07CFE0490204602F078FE42
:10160000DAF8C030DAF854802A4C09900793730056
:1016100048460A9302F052FC0EAB53F8261002F033
:10162000A1FCDFF8A0A005463AF9160002F046FC3E
:101630000146284602F08CFB02F05AFE05B2204B10
:10164000B5F57A7FA8BF4FF47A759D42B8BF1D46A5
:101650000AF13C0AA8B22AF8160000B202F02EFCE9
:101660000599824602F07EFC02F042FE089983B2A0
:101670005046069302F076FC414602F073FC216866
:1016800002F068FB02F034FE049B98421CDB099BCD
:101690009842A8BF184618E038100020001000201B
:1016A000FC210020DB0FC94030F8FFFF48F4FFFFAA
:1016B0000A100020601000200000C842D302373911
:1016C00018FCFFFFE8210020049802F0F7FB2060DF
:1016D0008346B87802F0EEFB384902F043FC01463D
:1016E0004FF07E5002F0F2FC414602F033FB01461F
:1016F000404602F0EBFC0B906068D4F808A0281A72
:1017000002F0DCFB414602F0E1FC514602F020FB16
:10171000DDF82CC00146604602F024FC014650462C
:1017200002F018FB656001462061A060079802F096
:1017300019FC02F0DDFD069B1434034458469A461A
:1017400002F0D6FD40F6B832504400B29042A8BF35
:1017500010461B4A0A9B9042B8BF1046194A1A49C4
:1017600098521422724342F801B00EB901264EE796
:101770003B792BB1039A642392FBF3F3134A138052
:101780003B88029A124C9A420DD9D4F8AC30A06F23
:10179000C01AF9F795FF42F2107380EAE072A2EBEB
:1017A000E0729A4206DD0B4B01221A70B4F8C82091
:1017B000064B1A8011B0BDE8F08F00BFDB0FC940A7
:1017C00048F4FFFF0A10002038100020F80F002016
:1017D00080210020FC0F002010B50E4C2068FDF782
:1017E0006DF920680022047A02FB02F3193B63437F
:1017F00003F6C4135343192193FBF1F3064921F86F
:1018000012300132072AEFD1BDE810400349FDF73D
:101810000DB900BF48110020480F0020902900207A
:101820000E4B1A78682A16D140F2CC725988914230
:1018300011D11A79BE2A0ED193F8C9270020EF2AB8
:101840000BD113F8012B5040054A9342F9D1B0FA5D
:1018500080F04009704700207047704700F8010889
:10186000CCFF01082DE9F74FEB4C002140F2CC7280
:10187000204606F0ECF8E94B04F536721A60E84BA6
:1018800000221A70E74B04F2A271196068232370DA
:10189000032363714FF48073A3604FF41673A4F8AD
:1018A0006631FA23A4F868312A23A4F864314FF48E
:1018B000FA73A4F86C31012384F8623184F87C3126
:1018C00084F88431052384F8173240F2DC53A4F8FD
:1018D000963140F24C43A4F8983140F26C73A4F86E
:1018E0009A3140F27533A4F89C3140F64303A4F8D2
:1018F0009E312346202184F86A116E2184F87A11E2
:101900000A2184F87B112B2184F87D11212184F890
:101910007E11232184F87F114FF4C871A4F880113F
:101920009918023200254FF01E0A1C2ABA4C81F881
:10193000A05181F8A1A1F3D140F27E41A4F8441155
:1019400040F23A71A4F8461140F27E51A4F84C11CD
:1019500040F2EA5140F2DC50A4F84E1140F2B4518A
:10196000052384F8D431C82301264FF47A774FF445
:10197000FA684FF0320BA4F8D831DFF8A0924FF498
:10198000C8731922A4F8BE81A4F8C281A4F8C68144
:10199000A4F8CA81A4F8DC31A4F84A01A4F85011D3
:1019A000A4F8BC71A4F8C071A4F8C471A4F8C871FB
:1019B00084F8D66184F8D76184F8DA61A4F84871B4
:1019C000A4F852B184F893A184F8D5210092019033
:1019D000A4F8543184F8D36184F8E061A4F856B1D6
:1019E00084F8E36100F02AFCD9F80030009A4FF047
:1019F0000F0E2674E673A4F80C80A57383F805E037
:101A00004FF0220E172183F806E0DA714FF00E0E28
:101A100021225975997583F810E05A7455214FF0B9
:101A2000350E53224FF0640C4FF02808D97083F81C
:101A30001AE02D21DA764FF05A0E0A2283F81CC0E4
:101A40004FF0780C83F80BA083F80CA0597383F83F
:101A500008E09A7400921D7083F8018083F8028078
:101A6000DD7583F804B09D731D76DD735D7683F8B4
:101A7000098083F80AC019754FF4FA71A3F84E1063
:101A80006949DFF8C4C19963D9636849C3F82CC0B8
:101A9000C3F830C09962DFF8B4C14FF07E5159638A
:101AA0004FF07F5A62490198C3F820A0C3F824A0E0
:101AB000C3F848C04FF0000A4FF04B0C59649E77B2
:101AC00083F8525083F8515083F85050C3F840A027
:101AD00083F84CC084F8A2E7A4F8AC074FF0410E9D
:101AE000042084F8A3E784F8A4B784F8A55784F801
:101AF000A95784F8AA5784F8A65784F8A75784F8FA
:101B0000A85783F85C00A3F85850A3F85A50A3F8DC
:101B100056501966152183F8681046494648D9661B
:101B2000464983F864801967454983F86580596799
:101B300083F8786000F0AEFBD9F80030009A1846C0
:101B40004FF4487183F8115183F8125183F81381CF
:101B500083F8146183F81851A3F8161184F8CE2184
:101B6000C82284F8CF21A4F8D0710E2202FB0532DE
:101B70006FF0170482F81941032482F81A416FF0BC
:101B80002F0482F81B41072482F81C416FF02304C4
:101B900082F81D41052482F81E4101355A2480F83F
:101BA000204180F821416422FF24082D80F81F2164
:101BB00080F822414FF0000100F10E00D5D1C8207D
:101BC000A3F88A01142083F88C01A3F890211E2029
:101BD0004FF4967283F88D01A3F8922101202822F8
:101BE00083F8891183F88E01A3F894210B460A4DDE
:101BF0005A191033C02BC2F814A0F8D105F526707D
